:020000040000FA
:10000000040004008BEF09F01200166A176A079AC1
:100010005AD9D8A01200D30FD8B4078A2D0FC60F13
:1000200003E20A0FF5E305D0F30FF2E2060FF0E367
:100030000A0F126E040E136ED89016361736132E52
:10004000FBD71250161204060EE03DD9D8A01200BC
:10005000C60F03E20A0F07E3ECD7F30F04E2060F23
:1000600002E30A0FE6D707AA04D0161E171E164A87
:10007000172A1650D8801200046A166E176A009666
:100080000450D8B40086100E036E000E16361736D4
:10009000D8B0010E3BD80366F8D71200046A166E7A
:1000A000176A00960450D8B40086040E036E173801
:1000B00005D8175003D8163801D816500F0BF60F75
:1000C000D8B0070F0A0F22D031D803D0046A166EB9
:1000D000176A00960450D8B40086050E036E270EEA
:1000E000136E100E0CD8030E136EE80E08D8136AA8
:1000F000640E05D8136A0A0E02D8165007D0126E85
:1001000017500F6E16500E6EAFD90E500E6E034E76
:100110000096045003E0035CD8B007D00E50D8A47A
:10012000009600B602D0300FC5D0120017AE1200F4
:1001300016501710D8B41200161E171E164A172A8A
:100140002D0EB8D0386E21AE02D02D0EB3D8233E7E
:1001500004D0223E02D0214A212A2C6A2D6A2E6A1E
:100160002F6A218E6A0E2026D89021322232233225
:100170002F322E322D322C32203EF6D72350205CE7
:100180002326205E2250215C2226215E046A38D874
:100190002E0E90D8396AD8902C34236E2D34226ECE
:1001A0002E34216E2F34206E3936D89023362236E5
:1001B0002136203639362C5023262D50D8B02D3CF0
:1001C00022262E50D8B02E3C21262F50D8B02F3CBE
:1001D0002026D8B0393ED890233622362136203614
:1001E00039363950300F66D823C02CF022C02DF09C
:1001F00021C02EF020C02FF0382ECCD7D89012007E
:100200000096045003E100860A0E046E23C011F02C
:1002100022C010F021C00FF020C00EF0036A196A4E
:10022000186A176A0A0E166EF4D8032A0350045C83
:10023000D8A4F5D71650D8A4009600A602D0042C56
:1002400003D01650300F36D8042EE0D71200ABB2D0
:10025000AB98AB8802C00EF005C00FF0126A136AAB
:10026000040000D004009EBA15D0E86812261322BC
:100270000E220F22D8A012001248133CF1D7D00E44
:10028000126E030E136EEED7ABB2AB98AB880400C0
:100290009EAAFED7AE50D8801200A66AA68E09008C
:1002A000F55002E002D8FBD7120004009EA8FED74A
:1002B000AD6E120001B4F9D701A205D001B003D090
:1002C00001B2EE6E12003652C2E03604DDE0080ED6
:1002D00007B4010E136E126AEA6802C0E9FF055006
:1002E0003DD90550EF120C0E86D8055002C0E9FF2B
:1002F000EF14FF0F07A4123207B412363C0E7BD85E
:10030000132EEDD71250D8801200126E080E07B4CB
:10031000010E136EEA6802C0E9FF05501FD9040000
:1003200005501232D8B0EF123C0E65D80550EF12CE
:10033000132EF1D7D8801200076E07A01200EA68CA
:1003400002C0E9FF05500AD9010E0F6EF40E54D811
:100350000550EF12010E0F6EF40E4ED0AA6AA96E70
:10036000A66AA680A850A94AAA2A1200AA6AA86E5C
:10037000A66AA684550EA76EAA0EA76EA6820400D2
:10038000A6B2FED7A694A94AAA2A1200E836E836F1
:10039000FC0B0109C2128009C216C050F80B0309F8
:1003A000C06E640E28D8C2820400C2B2FED7C4CF89
:1003B00021F0C350206E120035503410D8B4342AC6
:1003C00035343518E836353A3438E8463518353A94
:1003D000010B3436341A353634501200136A126E5B
:1003E000FF0E1226132200D0D8A01200030E0F6EAB
:1003F000E60E02D8F5D70F6AFE0F0E6E040000D08D
:1004000000D0E86A0F5AD8A012000E0600D000D023
:10041000F5D7286A296A2A6A2B6A210E146E15D02C
:10042000283629362A362B361650285C175029587C
:1004300018502A5819502B5808E32B6E1650285E76
:100440001750295A18502A5AD8800E360F361036AF
:100450001136142EE5D72BC019F02AC018F029C088
:1004600017F02850166E1200176A166A100EF36EF7
:100470000F34163617361250165C1350175805E312
:100480001250165E1350175AD8800E360F36F32EC0
:10049000EFD70E5012001D501718800BF46E1DAED2
:1004A00005D01C1E1D1E1C2AD8B41D2A17AE05D04F
:1004B000161E171E162AD8B4172A126A0E6A0F6A59
:1004C000136A175002E1165018E0100EF36ED89020
:1004D0001C361D36123613361750135C02E11650C7
:1004E000125C07E31650125ED8A013061750135E75
:1004F000D8800E360F36F32EEAD7F4AE05D00E1E96
:100500000F1E0E2AD8B40F2A0E50120012501A02D3
:10051000F4CF17F0F3CF16F013501B02F4CF0FF007
:10052000F3CF0EF012501B02F3501726F4500E2298
:10053000E86A0F2213501A02F3501726F4500E22C5
:10054000E86A0F22165012000E6E0FBE02D80E502F
:1005500012000E1E0F1E0E4A0F2A1200FF0AEF167F
:1005600000D0E988E92AEC161200A66AA68E0900D6
:10057000F55002E0EE6EFBD71200E9CFE1FFEACFC3
:10058000E2FF610EE75C07E67B0EE75C04E7DF0E47
:10059000E714E65201D0E650EE6EF3E11200A66ACF
:1005A000A68EEE500900F55C02E1F566FAD712005E
:1005B000336A326A7E0E306E800E2DAE000E316EC2
:1005C00001D842D130502C5C396E11E2396C2C507C
:1005D00030C02CF0306E2D5031C02DF0316E2E50C9
:1005E00032C02EF0326E2F5033C02FF0336E1A0E01
:1005F000396074D0305272E0386A2D503B6E311839
:100600003C6E2D8E318E080E395E08E333C038F013
:1006100032C033F031C032F0316AF5D7392607E005
:10062000D8903132323233323832392EF9D73CAEAB
:1006300033D033502F5E32502E5A31502D5A07E2AC
:10064000D880000E2F562E562D56800E3B1A386C31
:1006500004E02F06000E2E5A2D5A040E396E2D6618
:100660000DD02EC02DF02FC02EF038C02FF0386ADC
:10067000080E2C5E29E3392EF2D726D02DBE08D0E5
:10068000D89038362F362E362D362C2EF7D71CD054
:1006900038AE22D0386A0FD033502F2632502E2257
:1006A00031502D2206E32D322E322F3238322C4A91
:1006B0000DD038AE11D02F3E0FD02E3E0DD02D3E96
:1006C0000BD0D8802F90EFD72C6A02D03A822C68BA
:1006D0002F6A2E6A800E2D6E3BAE2D9E2F5012007B
:1006E0002D502A6E31183C6E305051E02C5252E0A1
:1006F0002C5E7F0E03E22C2603E24BD02C264CE22C
:100700002FC028F02EC029F02A8E318E180E3B6E95
:100710002F6A2E6A2D6A0BD03350285C325029582C
:1007200011E3296E2A6A3350285E0BD004E231505F
:100730002A5CF2E007E33350285E3250295A3150E8
:100740002A5AD8802F362E362D36283629362A3684
:100750003B2EECD72DBE07D02C521BE03C322C0692
:100760003B2A3C36E3D707E23350285E3250295A01
:1007700031502A5A17E32F3E15D02E3E13D02D3E6E
:1007800011D02D322E322F322C3E0CD005D03A868D
:1007900004D03A842C6A02D03A822C682F6A2E6ADE
:1007A000800E2D6E3CAE2D9E2F5012002D502A6EC5
:1007B00031183C6E2C50D8A430503AE02C267E0ED6
:1007C00003E32C5E03E336D02C5E31E32FC028F028
:1007D0002EC029F02A8E318E2F6A2E6A2D6A180EAD
:1007E0003B6E2A322932283206E333502F2632500C
:1007F0002E2231502D222D322E322F323B2EF1D788
:100800002DBE07D02F362E362D362C5210E02C065A
:100810002A3416E32F3E14D02E3E12D02D3E10D097
:10082000D8802D322E322F322C3E0AD003D03A847B
:100830002C6A02D03A822C682F6A2E6A800E2D6EA6
:100840003CAE2D9E2F5012002CC03BF02D502FC0DF
:100850002DF02F6E2F363B322F323A6A2F363B3631
:1008600002E33A843A7E06E13A803B6A2F6A2E6AB6
:100870002D6A0BD03B2803E0D8802F3206D0D890C9
:100880002F3202E13A8201D03A863AB604D03AA237
:100890000FD03AB407D07F0E2F6EFF0E2E6E2D6E46
:1008A0002C6E23D0800E2F6E01D02F6A000EF6D74B
:1008B0003AB0FBD72C6A9F0E3B60EBD77E0E3B64B1
:1008C000F4D79E0E3B5C07E0D8902F322E322D32AB
:1008D0002C323B2AF6D73AA408D0D880000E2C56EA
:1008E0002D562E562F562FAEE0D72C501200000E4C
:1008F0002DBEFF0E2E6E2F6E06D02C6E2D6A2E6A28
:100900002F6A3C9E0AD03C9E2FAE07D0D880000EA6
:100910002C562D562E562F563C8E960E3B6E2F5231
:1009200009E0080E3B262DC02CF02EC02DF02FC064
:100930002EF011D02E520FE1080E3B5E2D5007E134
:10094000080E3B5E2C5002E12F5010D02C6A2E6E08
:100950002CC02DF02C6A2EBE06D0D8902C362D3609
:100960002E363B06F8D73CAE2E9E3B502CC02FF0C7
:100970002C6E2E502DC02EF02D6E12004150525371
:1009800020444947495045415445522056200000D3
:100990004259204F4D334243205749544820504933
:1009A0004331384632364B32320054797065204834
:1009B000454C5020666F7220496E666F000054658A
:1009C0006D70657261747572652053656E736F72B8
:1009D0002000445331383230000044533138423221
:1009E000300020436F6E6E6563746564000054458B
:1009F0004C454D45545259204D4F4445204F4E00D3
:100A0000434F4E5645525345204F464600005749E6
:100A100044452020000057494445312000005749F3
:100A200044453220000042454100424541434F4E7B
:100A3000000042544558540043414C00434F4E007F
:100A400052454D4F54450000444947490000454335
:100A5000484F000046494C5445520000475053004F
:100A60004D4F4E004D4F4E49544F52004D5943008B
:100A70004D5943414C4C00005452000054524143E4
:100A8000450054454D5000005458440054584445C6
:100A90004C415900554E5000554E50524F544F0046
:100AA00044495350000048454C50000053455243C0
:100AB0004F4D000053455247505300005454455881
:100AC00054005441494C000053594D424F4C0000D2
:100AD000484F4C4400005458540054585441494C19
:100AE000000050455253000055430000564300009B
:100AF00057430000584300005041524D0000554EEE
:100B00004954000045514E530000424954530000DF
:100B10004445465300004443414C4C00535550500B
:100B20000000504152414D005645520046494C4C40
:100B3000000052444154410044535100494741543C
:100B40004500544E4300436F6D6D616E64206973C0
:100B5000206E6F742076616C6964000042454143E9
:100B60004F4E20544558545320455241534544005C
:100B700043414C494252415445204F4E0000534599
:100B800054204652455155454E4359204F4E205012
:100B90004F5254422E3620544F2036303020487A5F
:100BA0000000747970652055287029206F722044E8
:100BB000286F776E292C20726573702E2045286E61
:100BC000642900004F4E4C5920584D49542C524333
:100BD00056206F72204F464600004E45572042492E
:100BE0005452415445204146544552205245535495
:100BF00041525400414C4C00584D495400004F465E
:100C0000460052435600474F4E00474F4600474F5D
:100C1000464600004F4E4C5920414C4C2C584D49F3
:100C2000542C5243562C474F4E2C474F46206F7240
:100C3000204F46460000524553004E4F204D4F5224
:100C40004520504C4143455320464F522044454196
:100C5000442043414C4C5300526570656174657289
:100C60002072756E6E696E673A20000046494C54DA
:100C70004552200054454D5065726174757265206F
:100C8000000050455253697374656E63652000001F
:100C9000545844656C617920000054585461696C63
:100CA0002000244750524D430000244750474741FD
:100CB0000000244750474C4C0000545261636520AB
:100CC00000004D4F4E69746F722000002B47415455
:100CD00045574159000044494749706561742000F7
:100CE00046494C4C20696E20646967692000535561
:100CF00050507265737320005244415441200000EB
:100D0000504152414D20000044535175656C636859
:100D10002000424541636F6E200045766572792060
:100D2000000053594D424F4C2000484F4C446F66D1
:100D3000662000004947415445200000544E43209E
:100D400041444452455353200000534552434F4DB4
:100D500020005345524750532000554E50726F7437
:100D60006F2000004D5943616C6C20004443414C9E
:100D70004C73200042544558542031200000425406
:100D80004558542032200000545445585420000047
:100D9000313135323030000035746820696E70753D
:100DA00074206973206E6F7420616E616C6F6700D0
:100DB00056455253494F4E3A2042434449474920F1
:100DC0000000436F6D6D616E6473202877697468ED
:100DD000206578616D706C65293A20004449535054
:100DE00020446973706C617920616C6C2073657448
:100DF00074696E670000424541636F6E202862652A
:100E000061636F6E206576657279206E292D206E84
:100E10003D30206973206F666620616E6420313C2E
:100E20006E3C3630206D696E730042544558542034
:100E3000312028323030206368617273206D617810
:100E40002900425445585420322028323030206343
:100E500068617273206D617829005441494C2028E3
:100E60007461696C2074657874206F722062746597
:100E7000787432206576657279204E292D284F4E80
:100E80002C4F46462C4E292D204E3D302069732094
:100E90006F666620616E6420313C6E3C3920657659
:100EA000657279204E2D7468206D65737361676576
:100EB00000005454455854202D207461696C2074EE
:100EC000657874202D203130302063686172732082
:100ED0006D61780043414C696272617465202843FA
:100EE000616C69627261746520313230304264290C
:100EF0000000434F4E766572736520286F6E29009F
:100F0000444947497065617420286F6E2F6F66668B
:100F1000290046494C4C696E6469676920286F6EE8
:100F20002F6F666629004543484F20286F6E2F6F4C
:100F300066662900445351206469676974616C20B6
:100F4000737175656C636820286F6E2F6F666629F4
:100F5000000046494C54455220286F6E2F6F66663C
:100F6000292D2066696C74657220756E7072696EC9
:100F70007461626C65207465726D696E616C20636A
:100F800068617273000047505320286770732024F3
:100F900047504747412F244750474C4C2F24475038
:100FA000524D432900004D4F4E69746F72202861E5
:100FB0006C6C2F6F66662F7263762F786D69742F55
:100FC000676F6E2F676F662900004D5943616C6C27
:100FD00020286D7963616C6C204F4D3342432D3274
:100FE000290054454D50657261747572652028431F
:100FF0002F46290054526163652028786D69742F4B
:101000007263762F6F66662920666F722064656250
:10101000756767696E67206F6E6C79005045525333
:10102000697374656E636520286E207820313020E6
:101030006D732900545844656C6179207478646537
:101040006C6179206E20303C6E3C31303020286E4F
:101050002078203130206D73290054585461696C18
:10106000205458207461696C2074696D6520286E65
:101070002078203130206D732900554E50726F74E6
:101080006F2028756E70726F746F2061707273209C
:10109000762077696465312D3129202D2033206435
:1010A00069676973206D61780000534552434F4D65
:1010B000206E2073657269616C20706F727420738A
:1010C0007065656420666F7220544E432028343862
:1010D0002C39362C3139322C3338342C3537362CE8
:1010E000313135290000534552475053206E20734B
:1010F0006F6D6520617320534552434F4D206275DB
:101100007420666F72204750530053594D424F4C24
:10111000203220415052532073796D626F6C7320DE
:101120002D2064656661756C74206973204341529B
:1011300020282F3E2900484F4C444F4646206E2021
:1011400073657420484F4C44204F46462074696DA7
:101150006520696E207365632E286D696E2E2031BF
:1011600030290000535550507265737320286F6EFC
:101170002F6F666629207375707072657373206DAA
:10118000756C7469706C65207061636B6574730055
:101190005543616C20766F6C746167652063616C88
:1011A0006962726174696F6E20666F7220553120BA
:1011B000696E707574005643616C20666F722055BD
:1011C00032005743616C20666F72205533005843DC
:1011D000616C20666F72205534005041524D20736F
:1011E000657420706172616D657465727300554E2F
:1011F00049542073657420756E69747300004551FD
:101200004E5320736574206571756174696F6E73D8
:1012100020412C422C43202D2046696E616C2076A3
:10122000616C7565203D20412A585E322B422A5858
:101230002B43000042495453207365742062697443
:1012400020706172616D657465727320616E6420D7
:1012500070726F6A656374207469746C65004445CC
:10126000465320646566696E6520696E7075747397
:101270003A2041202D20616E616C6F672C20542034
:101280002D2074656D702E28445331383230292C4E
:101290002030202D206E6F742075736564005244D9
:1012A00041544120736574207261772074656C65C8
:1012B0006D657472696320646174610050415241CC
:1012C0004D20286F6E2F6F666629202D20504152C9
:1012D0004D2C554E49542C45514E5326424954539A
:1012E00020617320626561636F6E00005645527322
:1012F000696F6E20736F66747761726520766572B0
:1013000073696F6E000042434449474920004243DD
:10131000444947490000400E3A6E006AA00EAF6E85
:10132000200EAC6E900EAB6E00010FEE37F0ED6A42
:10133000E950EA10FCE1EF6A030E356E450E346E9B
:10134000F28E04D0F2BE12008EEF6CF00001FADFD4
:10135000F9DFDF0E926EF6DFF5DFBF0E936EF2DF80
:10136000F1DF8E0E946EEEDFEDDF806AEBDFEADFF9
:10137000826AE8DFE7DF900EAB6EE4DFE3DF200E8A
:10138000AC6EE0DFDFDFAC94DDDFDCDF716ADADF7B
:10139000D9DF726AD7DFD6DFF40ED36ED3DFD2DFA8
:1013A000D26AD0DFCFDFC00E9B6ECCDFCBDF796A95
:1013B000C9DFC8DF786AC6DFC5DFE00EF26EC2DFC4
:1013C000C1DFF16ABFDFBEDFF06ABCDFBBDFBF0E8B
:1013D000616EB8DFB7DF816AB5DFB4DF010EC26EC0
:1013E000B1DFB0DF080EC16EADDFACDFAB0EC06E9B
:1013F000A9DFA8DF030E0F01386FA4DFA3DF396B6D
:10140000A1DFA0DF3A6B9EDF9DDFF00E426F9ADF17
:1014100099DF040E9D6E96DF95DFA06A93DF92DF61
:10142000040E9F6E8FDF8EDFA26A8CDF8BDF870E4C
:10143000D56E88DF87DF300ECD6E84DF83DFBD6A37
:1014400081DF80DF2F0EBA6E7DDF7CDF910E4E6F65
:1014500079DF78DF4D6B76DF75DF230EAEEC01F0C0
:101460000301FD6F6FDF6EDF240EAEEC01F0FE6F47
:1014700069DF68DF250EAEEC01F0FF6F63DF62DF2E
:10148000260EAEEC01F00401006F5CDF5BDF270E7F
:10149000AEEC01F0016F56DF55DF990EAEEC01F0B6
:1014A000026F50DF4FDF9A0EAEEC01F0826F4ADF21
:1014B00002510001E8A214D045DF44DF0301FF918F
:1014C00041DF40DFFF933EDF3DDFFF953BDF3ADF4B
:1014D000FF9738DF37DFFF9935DF34DF04010095F0
:1014E000000130DF2FDFAA0EAEEC01F004010B6F1C
:1014F00029DF0B29000104E125DF24DF0301FD9F23
:10150000000120DF1FDF010EAA6E4C0EA96EB0ECA9
:1015100001F004010B6F16DF0B29000104E112DF5B
:1015200011DF0301FD9B00010DDF0CDF020EAA6E2F
:10153000170EA96EB0EC01F004010B6F03DF0B294D
:10154000000104E1FFDEFEDE0301FD9D0001FADE85
:10155000F9DE010EAA6E0F0EA96EB0EC01F00401C7
:101560000B6FF0DE0B29000108E1ECDE010EAA6E24
:101570000F0EA96E0D0EB7EC01F0E4DEE3DE020EF5
:10158000AA6EE20EA96EB0EC01F004010B6FDADE78
:101590000B29000108E1D6DE020EAA6EE20EA96E4A
:1015A0000D0EB7EC01F0CEDECDDE030EAA6E410EBD
:1015B000A96EB0EC01F004010B6FC4DE0B29000131
:1015C00008E1C0DE030EAA6E410EA96E0D0EB7EC47
:1015D00001F0B8DEB7DE030EAA6EA00EA96EB0EC65
:1015E00001F004010B6FAEDE0B29000108E1AADE59
:1015F000030EAA6EA00EA96E0D0EB7EC01F0A2DECE
:10160000A1DE430E04010C6F9DDE9CDE2A6B296B6C
:1016100099DE98DE896B96DE000182A203D092DE0D
:10162000949A8B8A8FDE8EDE0401059F8BDE8ADE24
:10163000059988DE87DE059385DE84DE056B82DE14
:1016400081DE066B7FDE7EDE036B7CDE7BDE046B81
:1016500079DE78DE426B416B75DE74DE886B876BFA
:1016600071DE70DEB8866EDE6DDEAC986BDE6ADE33
:10167000AC8468DE67DE0F0E821764DE63DE266BE5
:101680003A0E256F5FDE5EDE000E82B2010E25256A
:10169000A96E2651D8B0010FAA6EB0EC01F00B6F05
:1016A00051DE0B53000109E14DDE4CDE0D0EB06E34
:1016B00049DE48DE050EAF6E44D0010E04010B5D1D
:1016C000000109E13FDE3EDE060EB06E3BDE3ADE93
:1016D000820EAF6E36D0020E04010B5D000109E1EF
:1016E00031DE30DE030EB06E2DDE2CDE400EAF6E2E
:1016F00028D0030E04010B5D000109E123DE22DE88
:10170000010EB06E1FDE1EDE9F0EAF6E1AD0040EED
:1017100004010B5D000109E115DE14DE010EB06E5F
:1017200011DE10DE150EAF6E0CD0050E04010B5D40
:10173000000107E107DE06DEB06A04DE03DE8A0E82
:10174000AF6E00DEFFDD380EAEEC01F00301FC6F82
:10175000F9DDF8DD400EAEEC01F00401836FF2DD3F
:10176000F1DD410EAEEC01F0846FECDD000126EC02
:1017700051F0E8DDA2EC09F03F0EAEEC01F00401FF
:101780007D6FA2EC09F0A2EC09F07D517DEC04F034
:10179000336A326A400E316E7F0E306ED6EC03F043
:1017A00024EC04F07E6F0001A2EC09F0A2EC09F039
:1017B000390EAEEC01F00401086FA2EC09F0A2ECC6
:1017C00009F03E0EAEEC01F0796FA2EC09F0A2EC4C
:1017D00009F03C0EAEEC01F07B6FA2EC09F0A2EC3C
:1017E00009F03D0EAEEC01F07C6FA2EC09F0A2EC2A
:1017F00009F0420EAEEC01F0856FA2EC09F0A2EC0C
:1018000009F0430EAEEC01F0866FA2EC09F0A2ECF9
:1018100009F04E0EAEEC01F00B6FA2EC09F00B29B3
:10182000000128E1A2EC09F0AA6A4E0EA96E410E51
:10183000B7EC01F0A2EC09F0AA6A4F0EA96E410EB6
:10184000B7EC01F0A2EC09F0AA6A500EA96E410EA5
:10185000B7EC01F0A2EC09F0AA6A510EA96E410E94
:10186000B7EC01F0A2EC09F0AA6A520EA96E540E70
:10187000B7EC01F0A2EC09F0A2EC09F086C465F423
:10188000A2EC09F0A2EC09F0040108057A6FA2ECC1
:1018900009F00301FD3100011CE3A2EC09F0A2EC08
:1018A00009F00401266B256BA2EC09F0000196EC0F
:1018B00054F0A2EC09F0A2EC09F000EE4DF010EEAD
:1018C000B9F00F0EE75204E0E6CFEEFFE82EFAD7AC
:1018D000EF6AA2EC09F00301FD510001E8A21DD05E
:1018E000A2EC09F0A2EC09F00401266B070E256FAB
:1018F000A2EC09F0000196EC54F0A2EC09F0A2EC85
:1019000009F000EE56F010EEB9F00F0EE75204E0C9
:10191000E6CFEEFFE82EFAD7EF6AA2EC09F003015A
:10192000FD510001E8A41DD0A2EC09F0A2EC09F0E1
:101930000401266B0E0E256FA2EC09F0000196EC57
:1019400054F0A2EC09F0A2EC09F000EE5FF010EE0A
:10195000B9F00F0EE75204E0E6CFEEFFE82EFAD71B
:10196000EF6AA2EC09F00301FD510001E8A61DD0C9
:10197000A2EC09F0A2EC09F00401266B150E256F0C
:10198000A2EC09F0000196EC54F0A2EC09F0A2ECF4
:1019900009F000EE68F010EEB9F00F0EE75204E027
:1019A000E6CFEEFFE82EFAD7EF6AA2EC09F00301CA
:1019B000FD510001E8A81DD0A2EC09F0A2EC09F04D
:1019C0000401266B1C0E256FA2EC09F0000196ECB9
:1019D00054F0A2EC09F0A2EC09F000EE71F010EE68
:1019E000B9F00F0EE75204E0E6CFEEFFE82EFAD78B
:1019F000EF6AA2EC09F00401096B0A0E0401095D0B
:101A0000000119E2A2EC09F0A2EC09F0AA6A440E66
:101A100004010925A96ED8B0AA2AB0EC01F00A6E1B
:101A200000EE7AF009510AC0EBFFA2EC09F00401C4
:101A3000092B0001E2E3A2EC09F0A2EC09F00F018E
:101A4000386BA2EC09F0A2EC09F04E0EAEEC01F0FE
:101A500004010B6FA2EC09F0540E0B5D000132E1A2
:101A6000A2EC09F0800E026E010E056E076E9CEC72
:101A700001F0330E85EC01F0A2EC09F0800E026E4D
:101A8000010E056E076A67EC01F004015F6FA2ECBE
:101A900009F0000133EC69F0A2EC09F0A2EC09F0C6
:101AA00004015B31E832D8B05B85D8A05B95A2EC2D
:101AB00009F0A2EC09F05B35D8B05C81D8A05C914C
:101AC00000010ED0A2EC09F0410E04010B5D0001F3
:101AD00006E1A2EC09F0A2EC09F00F013881000147
:101AE000A2EC09F0A2EC09F0AA6A4F0EA96EB0ECC4
:101AF00001F004010B6FA2EC09F0540E0B5D000124
:101B000033E1A2EC09F0800E026E020E056E010EAA
:101B1000076E9CEC01F0330E85EC01F0A2EC09F0AD
:101B2000800E026E020E056E076A67EC01F004017A
:101B30005F6FA2EC09F0000133EC69F0A2EC09F050
:101B4000A2EC09F004015B31E832D8B05B87D8A081
:101B50005B97A2EC09F0A2EC09F05B35D8B05C838E
:101B6000D8A05C9300010ED0A2EC09F0410E040154
:101B70000B5D000106E1A2EC09F0A2EC09F00F01F7
:101B800038830001A2EC09F0A2EC09F0AA6A500E19
:101B9000A96EB0EC01F004010B6FA2EC09F0540E39
:101BA0000B5D000133E1A2EC09F0800E026E040E21
:101BB000056E010E076E9CEC01F0330E85EC01F012
:101BC000A2EC09F0800E026E040E056E076A67EC47
:101BD00001F004015F6FA2EC09F0000133EC69F041
:101BE000A2EC09F0A2EC09F004015B31E832D8B0B4
:101BF0005B89D8A05B99A2EC09F0A2EC09F05B35F7
:101C0000D8B05C85D8A05C9500010ED0A2EC09F09C
:101C1000410E04010B5D000106E1A2EC09F0A2EC0B
:101C200009F00F0138850001A2EC09F0A2EC09F0DF
:101C3000AA6A510EA96EB0EC01F004010B6FA2EC80
:101C400009F0540E0B5D000133E1A2EC09F0800EA7
:101C5000026E080E056E010E076E9CEC01F0330E4D
:101C600085EC01F0A2EC09F0800E026E080E056E04
:101C7000076A67EC01F004015F6FA2EC09F0000154
:101C800033EC69F0A2EC09F0A2EC09F004015B313D
:101C9000E832D8B05B8BD8A05B9BA2EC09F0A2EC39
:101CA00009F05B35D8B05C87D8A05C9700010ED0F6
:101CB000A2EC09F0410E04010B5D000106E1A2EC6B
:101CC00009F0A2EC09F00F0138870001A2EC09F03D
:101CD000A2EC09F0AA6A520EA96EB0EC01F0040160
:101CE0000B6FA2EC09F0540E0B5D010ED8A4000E90
:101CF000376E010E05B9000E3712000131E0A2EC7B
:101D000009F0800E026E100E056E010E076E9CEC3F
:101D100001F0330E85EC01F0A2EC09F0800E026EAA
:101D2000100E056E076A67EC01F004015F6FA2EC0C
:101D300009F0000133EC69F0A2EC09F0A2EC09F023
:101D400004015B31E832D8B05B8DD8A05B9DA2EC7A
:101D500009F0A2EC09F05B35D8B05C89D8A05C9999
:101D60000001A2EC09F00301FF510001E8AA0BD029
:101D7000A2EC09F0A2EC09F00301FF9FA2EC09F02C
:101D8000A2EC09F0FF9D0001A2EC09F0A2EC09F021
:101D90000401068FA2EC09F0A2EC09F0AECF0BF41F
:101DA000A2EC09F000510001E8B209D0A2EC09F060
:101DB000A2EC09F0430E04010C6F000107D0A2EC65
:101DC00009F0A2EC09F0460E04010C6F0001A2EC30
:101DD00009F0A2EC09F00F01506BA2EC09F0A2ECA3
:101DE00009F04F6BA2EC09F004015C510001E8A876
:101DF00086D0A2EC09F0800E026E100E056E010E68
:101E0000076E9CEC01F0CC0E85EC01F0440E85ECE5
:101E100001F0A2EC09F0030E136E200EEFEC01F0BE
:101E2000A2EC09F0800E026E100E056E010E076E18
:101E30009CEC01F0CC0E85EC01F0BE0E85EC01F0BF
:101E4000A2EC09F0800E026E100E056E076A67ECB8
:101E500001F00401396F67EC01F03A6FA2EC09F070
:101E6000A2EC09F05B35E836D8B05E89D8A05E995F
:101E7000A2EC09F0000185EC68F0A2EC09F0A2ECFC
:101E800009F038C430F437C42FF436C42EF435C406
:101E90002DF4A2EC09F0A2EC09F02F6A2E6A200EB4
:101EA0002D6E820E2C6E38C433F037C432F036C437
:101EB00031F035C430F0D6EC03F024EC04F004012A
:101EC000336F2DC034F4A2EC09F0096B0F0E04013E
:101ED000095D000114E2A2EC09F0A2EC09F000EEA9
:101EE000CFF0D8900401093533C4EBFFE82A34C49D
:101EF000EBFFA2EC09F00401092B0001E7E3A2ECDF
:101F000009F082A21BEF29F0A2EC09F081B80BD0F6
:101F1000A2EC09F0A2EC09F004010589A2EC09F099
:101F2000A2EC09F005830001A2EC09F00D0E55ECBE
:101F300001F0090EF76E7C0EF66E4DEC01F0040E0A
:101F4000016E046A176A166E69EC00F02E0E55ECED
:101F500001F0010E046E310E67EC00F00D0E55EC31
:101F600001F0A2EC09F0090EF76E900EF66E4DEC42
:101F700001F00D0E55EC01F0A2EC09F0090EF76E20
:101F8000AA0EF66E4DEC01F00D0E55EC01F0A2EC30
:101F900009F0090EF76EBE0EF66E4DEC01F0A2ECE4
:101FA00009F004015C510001E8A879D0A2EC09F025
:101FB00004015B510001E8BC09D0A2EC09F0090E54
:101FC000F76ED20EF66E4DEC01F008D0A2EC09F0DF
:101FD000090EF76EDA0EF66E4DEC01F0A2EC09F088
:101FE000800E026E100E056E010E076E9CEC01F065
:101FF000CC0E85EC01F0440E85EC01F0A2EC09F06A
:10200000030E136E200EEFEC01F0A2EC09F0800E2F
:10201000026E100E056E010E076E9CEC01F0CC0EE8
:1020200085EC01F0BE0E85EC01F0A2EC09F0800E0B
:10203000026E100E056E076A67EC01F00401396F3D
:1020400067EC01F03A6FA2EC09F0A2EC09F03A3526
:10205000D8B05C8BD8A05C9BA2EC09F0A2EC09F094
:102060003AAF03D0396DE86A3A570001A2EC09F0A3
:1020700004015B510001E8AC05D0A2EC09F085EC4D
:1020800068F00BD0A2EC09F0A2EC09F00401395180
:10209000050DF3CF2BF4F4CF2CF400010BD0A2EC00
:1020A00009F04E0E55EC01F06F0E55EC01F0740E78
:1020B00055EC01F0A2EC09F0090EF76EE20EF66E97
:1020C0004DEC01F0A2EC09F0A2EC09F0040105814D
:1020D000A2EC09F005510001E8A815D0A2EC09F026
:1020E00049EC61F0A2EC09F00D0E55EC01F0090E7F
:1020F000F76EEE0EF66E4DEC01F0A2EC09F0A2ECDC
:1021000009F0040105910001A2EC09F00D0E55EC57
:1021100001F00D0E55EC01F0630E55EC01F06D0E63
:1021200055EC01F0640E55EC01F03E0E55EC01F05B
:10213000A2EC09F0A2EC09F004010587A2EC09F079
:10214000A2EC09F006810001A2EC09F0040105519E
:102150000001E8A604D0A2EC09F099EC60F0A2EC32
:1021600009F004010631000104E3A2EC09F0C5EC1A
:102170002BF0A2EC09F0040106510001E8A203D003
:10218000A2EC09F042D8A2EC09F0040105310001EB
:1021900003E3A2EC09F0D8D9A2EC09F0040106355A
:1021A000000104E3A2EC09F0FEEC16F0A2EC09F049
:1021B000040106510001E8AA04D0A2EC09F0FFECEA
:1021C0001AF0A2EC09F0040106510001E8AC04D0B9
:1021D000A2EC09F026EC27F0A2EC09F0040105516D
:1021E0000001E8A204D0A2EC09F03BEC62F0A2EC02
:1021F00009F0040105510001E8AC04D0A2EC09F09B
:10220000CAEC29F0A2EC09F09ED7A2EC09F09EAA34
:10221000A2EF09F0A2EC09F0A2EC09F00401069B80
:102220000001A2EC09F0056A010E026E27EC01F034
:10223000F7E3466EA2EC09F0030E465CD8B491D0E9
:10224000A2EC09F0D9EC2BF0A2EC09F0C0D8A2EC7A
:1022500009F04C6A0A0E4C5C11E2A2EC09F0A2EC07
:1022600009F000EE7AF04C50EB50476EA2EC09F00A
:10227000C8EC15F0A2EC09F04C2AECE3A2EC09F052
:10228000A2EC09F0200E476EA2EC09F0C8EC15F0A4
:10229000A2EC09F0A2EC09F04C6AA2EC09F0FD0EE8
:1022A0004C5C21E2A2EC09F0A2EC09F001EE66F030
:1022B0004C50E926000EEA22EF50476EA2EC09F0DE
:1022C000C8EC15F0A2EC09F001EE66F04C50E926DE
:1022D000000EEA22EF500A6E0D0E0A5C04E0A2EC3A
:1022E00009F04C2ADCD7A2EC09F049EC23F0A2EC6F
:1022F00009F0A2EC09F09E9AA2EC09F0A2EC09F018
:10230000AECF0BF4A2EC09F0A2EC09F00401266BAD
:10231000256BA2EC09F0000181BA15D0A2EC09F0FE
:102320000401252B000E2623A2EC09F026510B0AEE
:10233000B80ED8B42519000106E0A2EC09F0010E90
:10234000EEEC01F0E8D7A2EC09F0FEEC16F0A2ECFE
:1023500009F0A2EC09F00401069DA2EC09F00001CD
:102360005FD7A2EC09F00D0E55EC01F00A0EF76EE6
:10237000000EF66E4DEC01F0A2EC09F0A2EC09F0B3
:10238000230EAEEC01F00301FD6FA2EC09F0A2EC0C
:1023900009F0240EAEEC01F0FE6FA2EC09F0A2EC05
:1023A00009F0250EAEEC01F0FF6FA2EC09F0A2ECF3
:1023B00009F004010693A2EC09F0A2EC09F00681F1
:1023C000A2EC09F000010AEC50F0A2EF09F0A2EC37
:1023D00009F0A2EC09F00401059DA2EC09F000014E
:1023E00026EC51F0A2EC09F0D8EC22F0A2EC09F0B6
:1023F000A2EC09F000EEB9F010EE56F0080EE7522C
:1024000004E0E6CFEEFFE82EFAD7EF6AA2EC09F07F
:10241000A2EC09F0610E4B6EA2EC09F00301FD5134
:102420000001E8A805D0A2EC09F0A2EC09F04B905D
:10243000A2EC09F0E0EC4EF0A2EC09F0A2EC09F0FD
:1024400000EEB9F010EE4DF0080EE75204E0E6CFD2
:10245000EEFFE82EFAD7EF6AA2EC09F0E0EC4EF0BE
:10246000A2EC09F04BB05AD0A2EC09F00301FD51E7
:102470000001E8A41BD0A2EC09F0A2EC09F0600E68
:102480004B6EA2EC09F0A2EC09F000EEB9F010EEF0
:102490005FF0080EE75204E0E6CFEEFFE82EFAD731
:1024A000EF6AA2EC09F0E0EC4EF003D0A2EC09F0E8
:1024B0001BD0A2EC09F00301FD510001E8A614D0E5
:1024C000A2EC09F0A2EC09F000EEB9F010EE68F011
:1024D000080EE75204E0E6CFEEFFE82EFAD7EF6AE7
:1024E000A2EC09F0E0EC4EF0A2EC09F0A2EC09F04D
:1024F000610E4B6EA2EC09F0A2EC09F000EEB9F00F
:1025000010EE71F0080EE75204E0E6CFEEFFE82E81
:10251000FAD7EF6AA2EC09F0E0EC4EF0A2EC09F079
:10252000A2EC09F0030E476EA2EC09F0C8EC15F01E
:10253000A2EC09F0A2EC09F0F00E476EA2EC09F053
:10254000C8EC15F0A2EF09F0A2EC09F0A2EC09F03A
:1025500004010591A2EC09F00301FE510001E8BC61
:1025600002D0A2EF09F0A2EC09F0010E0301FDB1C7
:10257000000E376E010EFDB3000E37120001D8A415
:10258000A2EF09F0A2EC09F0010E0301FDBB000E61
:10259000376E010EFDBD000E37160001D8A4A2EF64
:1025A00009F0A2EC09F0A2EC09F004010697A2ECF4
:1025B00009F00301FD510001E8AA51D0A2EC09F095
:1025C00004017A2BA2EC09F079517A5D000102E353
:1025D000000E01D0010E376E010E0301FEBB000E8E
:1025E0003712000110E0A2EC09F0A2EC09F0010E94
:1025F00004013E6F4C0E3D6FA2EC09F0A2EC09F015
:102600005E9100012BD0A2EC09F00301FD51000105
:10261000E8AC15D0A2EC09F0A2EC09F0020E04011E
:102620003E6F170E3D6FA2EC09F0A2EC09F07A6B39
:10263000A2EC09F0A2EC09F05E8100010ED0A2EC40
:1026400009F0A2EC09F0010E04013E6F4C0E3D6F43
:10265000A2EC09F0A2EC09F05E9100010ED0A2EC10
:1026600009F0A2EC09F0020E04013E6F170E3D6F57
:10267000A2EC09F0A2EC09F05E810001A2EC09F0E5
:1026800004010A6BC80E04010A5D000126E2A2ECF7
:1026900009F0A2EC09F004010A513D25A96E000ED3
:1026A0003E21AA6EB0EC01F00B6FA2EC09F00D0E0A
:1026B0000B5D000112E0A2EC09F05C0E04010B5D61
:1026C000000105E1A2EC09F007EC55F006D0A2EC00
:1026D00009F004010A2B0001D5E3A2EC09F077DE32
:1026E000A2EC09F00401626BC80E0401625D0001F6
:1026F000D8B09CD1A2EC09F0A2EC09F03EC4AAFF2C
:102700003DC4A9FFB0EC01F0476EA2EC09F00D0E3C
:10271000475CD8B48BD1A2EC09F05C0E475CD8A41E
:1027200075D1A2EC09F004013D2B000E3E23A2EC72
:1027300009F0A2EC09F00A6BA2EC09F0A2EC09F096
:102740003EC4AAFF3DC4A9FFB0EC01F0476EA2EC65
:1027500009F0A2EC09F0479AA2EC09F0550E475C8B
:1027600000010EE1A2EC09F0A2EC09F0010E040157
:10277000266F030E256FA2EC09F0000165D99CD0ED
:10278000560E475C0EE1A2EC09F0A2EC09F0010E36
:102790000401266F0E0E256FA2EC09F0000154D93A
:1027A0008BD0570E475C0EE1A2EC09F0A2EC09F0C9
:1027B000010E0401266F190E256FA2EC09F000012D
:1027C00043D97AD0580E475C0EE1A2EC09F0A2EC96
:1027D00009F0010E0401266F240E256FA2EC09F00A
:1027E000000132D969D0590E475C0EE1A2EC09F024
:1027F000A2EC09F0010E0401266F2F0E256FA2EC4A
:1028000009F0000121D958D0520E475C0EE1A2EC2C
:1028100009F0A2EC09F0010E0401266F5B0E256F92
:10282000A2EC09F0000110D947D0460E475C1DE12B
:10283000A2EC09F0A2EC09F000EEB9F0020E016E74
:10284000046A58C417F057C416F069EC00F0EF6A38
:10285000A2EC09F0A2EC09F00401266BB90E256F79
:10286000A2EC09F00001F0D827D05A0E475C24E111
:10287000A2EC09F0A2EC09F000EEB9F0020E016E34
:10288000046A176A040E166E69EC00F02E0EEE6EE6
:10289000020E016E010E046E310E67EC00F0EE6A5E
:1028A000A2EC09F0A2EC09F00401266BB90E256F29
:1028B000A2EC09F00001C8D8A2EC09F004015C51B7
:1028C0000001E8A8A0D0A2EC09F0540E475C0DE18D
:1028D000A2EC09F0A2EC09F00401266BF80E256FBA
:1028E000A2EC09F00001B0D88ED04C0E475C0EE18E
:1028F000A2EC09F0A2EC09F0010E0401266F450ECE
:10290000256FA2EC09F000019FD87DD0480E475CEE
:102910000EE1A2EC09F0A2EC09F0010E0401266F11
:10292000500E256FA2EC09F000018ED86CD0530E2A
:10293000475C0EE1A2EC09F0A2EC09F0010E0401E3
:10294000266F3A0E256FA2EC09F000017DD85BD00E
:10295000410E475CD8A457D0A2EC09F0A2EC09F0D4
:1029600030C42FF02FC42EF02EC42DF02DC42CF027
:10297000D8EC02F00401316F2DC032F4A2EC09F062
:10298000A2EC09F032AF03D0316DE86A3257000192
:10299000A2EC09F004012D53000117E004012E51AF
:1029A0000001E8BE12D0A2EC09F0A2EC09F000EEA2
:1029B000B9F0020E016E030E046E32C417F031C47A
:1029C00016F069EC00F0EF6A12D0A2EC09F0A2EC6C
:1029D00009F000EEB9F02D0EEE6E020E016E046EDF
:1029E00032C417F031C416F069EC00F0EF6AA2ECC3
:1029F00009F0A2EC09F00401266BB90E256FA2ECD8
:102A000009F0000121D8A2EC09F003D0A2EC09F0F2
:102A1000BFD8A2EC09F004013D2B000E3E23A2EC2E
:102A200009F00401622B0001D8A05ED6A2EC09F0E7
:102A300049EC23F0A2EC09F0A2EC09F00401068FA6
:102A4000A2EC09F000011200A2EC09F0A2EC09F0DE
:102A5000A2EC09F026C4E2FF25C4E1FFE6CF47F06F
:102A60000401252B000E2623A2EC09F04752000199
:102A700004E0A2EC09F08CD8E9D7A2EF09F0A2ECAF
:102A800009F0E7EC11F0A2EC09F0A2EC09F0600EFD
:102A9000476EA2EC09F081B006D0A2EC09F0A2ECDE
:102AA00009F0240E476EA2EC09F072D8A2EC09F0EE
:102AB000A2EC09F004010A6BA2EC09F0000101EE9E
:102AC00066F004010A51E926000EEA22EF500A6E70
:102AD0000D0E0A5CD8A4010E376EC70E0A5D010EFA
:102AE000D8B0000E3716000117E0A2EC09F0A2ECF6
:102AF00009F001EE66F004010A51E926000EEA220F
:102B0000EF50476EA2EC09F0000142D8A2EC09F0A8
:102B100004010A2B0001D2D7A2EC09F004017A2BA0
:102B2000A2EC09F079517A5D000ED8B0010E376E33
:102B3000000E0301FEBB010E3716000126E0A2ECD9
:102B400009F0A2EC09F004017A6BA2EC09F0000193
:102B500081A80DD0A2EC09F0A2EC09F004013E6BB3
:102B6000AA0E3D6FA2EC09F00001BAD50ED0A2EC7E
:102B700009F05CDFA2EC09F0170E136E700EEFEC9B
:102B800001F0A2EC09F077EF61F0A2EC09F04ED76A
:102B9000A2EC09F00301FF510001E8B60BD1A2EC51
:102BA00009F0A2EC09F004011551B10FE96E020E13
:102BB0001621EA6E47C0EFFFA2EC09F0152B000EBC
:102BC0001623A2EC09F0A2EC09F0F29AA2EC09F0AB
:102BD000446A0001080E445C4BE2A2EC09F0A2EC4E
:102BE00009F004015D8947A05D99A2EC09F000019C
:102BF0006DD8A2EC09F047B010D0A2EC09F0A2EC1D
:102C000009F0436AA2EC09F0A2EC09F00401048780
:102C1000A2EC09F0000133D821D0A2EC09F0A2EC1B
:102C200009F004010497A2EC09F0432AA2EC09F090
:102C3000000125D8A2EC09F0050E435C0FE1A2ECDF
:102C400009F0A2EC09F0436AA2EC09F0A2EC09F049
:102C500004010487A2EC09F0000111D8A2EC09F0EC
:102C6000A2EC09F0D8904732A2EC09F0442AB1E373
:102C7000A2EC09F0A2EC09F0F28AA2EF09F0A2ECB2
:102C800009F09EA2FED7A2EC09F0A2EC09F09E92F8
:102C9000A2EC09F0A2EC09F0E86A040104B9010F02
:102CA00004B7010AD8B40499D8A40489A2EC09F0A5
:102CB000A2EC09F0E86A04B9010E010AD8B4819CBB
:102CC000D8A4818CA2EC09F000011200A2EC09F05A
:102CD00004015D510001E8A806D0A2EC09F0A2ECC5
:102CE00009F0010E491AA2EC09F0A2EC09F0040166
:102CF0005D8949A05D99A2EC09F0A2EC09F0D89099
:102D00004A324932A2EC09F05D510001E8B802D024
:102D1000A2EF09F0A2EC09F0A2EC09F0080E491AA2
:102D2000A2EC09F0A2EC09F0840E4A1AA2EF09F015
:102D3000A2EC09F00301FF510001E8A602D0A2EFC6
:102D400009F0A2EC09F00401096B040109510B5DC3
:102D500000012EE3A2EC09F0A2EC09F004010487C3
:102D6000A2EC09F000018BDFA2EC09F0446A060E28
:102D7000445C0EE2A2EC09F0A2EC09F00401049715
:102D8000A2EC09F000017BDFA2EC09F0442AEFE39A
:102D9000A2EC09F0A2EC09F004010487A2EC09F00E
:102DA00000016DDFA2EC09F00401092B0001CDE365
:102DB000A2EF09F0A2EC09F0040E016E020E046EFF
:102DC00047504FEC00F0200E55EC01F0A2EC09F05A
:102DD0000401812BA2EC09F0100E815D00010BE1D2
:102DE000A2EC09F0A2EC09F00401816BA2EC09F05D
:102DF0000D0E55EC01F00001A2EF09F0A2EC09F074
:102E0000A2EC09F00401146B136BA2EC09F0A2EC24
:102E100009F0076BA2EC09F0A2EC09F00D6BA2EC33
:102E200009F0A2EC09F0069BA2EC09F0000181AACE
:102E3000A2EF09F0A2EC09F0A2EC09F00401048B66
:102E400081AE049B0001A2EC09F081AA11EF1AF0F7
:102E5000A2EC09F0040102310001D8A0C9D0A2EC13
:102E600009F0A2EC09F03E6A3D6AA2EC09F0A2EC7E
:102E700009F0406A3F6AA2EC09F0E86A81BE010FDE
:102E8000040104BB01080001D8B4F7D7A2EC09F093
:102E9000E86A81BE010F040104BB0108000119E0CA
:102EA000A2EC09F03D4A3E2AA2EC09F0010E3E5C7C
:102EB00008E3D8A411EF1AF0FF0E3D5CD8B011EF73
:102EC0001AF0A2EC09F0350EE82EFED70000000142
:102ED000DFD7A2EC09F0E86A81BE010F040104BB50
:102EE0000108000119E1A2EC09F03F4A402AA2ECD6
:102EF00009F0010E405C08E3D8A411EF1AF0FF0EB0
:102F00003F5CD8B011EF1AF0A2EC09F0350EE82EB4
:102F1000FED700000001DFD7A2EC09F03E5205E128
:102F20003D0E3D5C02E2000E01D0010E376E3E52B6
:102F300003E1500E3D5C02E3000E01D0010E371696
:102F4000010E405C000104E305E1D70E3F5C02E2A4
:102F5000000E01D0010E3716010E405C000106E3A1
:102F600003E1F40E3F5C02E3000E01D0010E3716C0
:102F70000001D8A448D0A2EC09F0010E3E5C04E3A5
:102F800005E1D70E3D5C02E2000E01D0010E376E66
:102F9000010E3E5C000106E303E1F40E3D5C02E33A
:102FA000000E01D0010E37164052000105E13D0E22
:102FB0003F5C02E2000E01D0010E3716405203E1E1
:102FC000500E3F5C02E3000E01D0010E37160001E7
:102FD0001AE1A2EC09F00401072BA2EC09F0050E9E
:102FE000075D0001D8A02ED7A2EC09F01AD20BD0B1
:102FF000A2EC09F0E86A040104BB010F81BE0108DC
:103000000001D8B41FD7A2EC09F0A2EC09F07EC4ED
:10301000BBFFA2EC09F0A2EC09F0BC6AA2EC09F03B
:10302000A2EC09F09E92A2EC09F0A2EC09F00401D6
:10303000048B81AE049BA2EC09F000019EA2FDD797
:10304000A2EC09F0E86A040104BB010F81BE01088B
:103050000001D8B4F7D6A2EC09F0A2EC09F07DC4C7
:10306000BBFFA2EC09F0A2EC09F0BC6AA2EC09F0EB
:10307000A2EC09F0D8904832A2EC09F07ADAA2EC7E
:1030800009F0A2EC09F00401488E5DAF489EA2EC65
:1030900009F0000181AAC5D1A2EC09F07E0E485CBE
:1030A000E5E1A2EC09F07E0E485C04E1A2EC09F037
:1030B000BED9F9D7A2EC09F0A2EC09F048C066F13C
:1030C000A2EC09F0929A898AA2EC09F0A2EC09F02C
:1030D000436AA2EC09F00401146B010E136F010E98
:1030E0000401145D000106E344E14A0E0401135D8E
:1030F00000013FE2A2EC09F0000199D9A2EC09F02D
:1031000004015D510001E8BCB1D7A2EC09F0040153
:103110005D510001E8AA12D0A2EC09F00401145399
:10312000000109E10F0E0401135D000104E2A2ECAD
:1031300009F09CD703D0A2EC09F01BD0A2EC09F057
:10314000A2EC09F004011351660FE96E010E14217F
:10315000EA6E48C0EFFFA2EC09F0000181AA61D13C
:10316000A2EC09F00401132B000E14230001D8A0D7
:10317000B6D7A2EC09F0929A899AA2EC09F0A2ECD7
:1031800009F0030E0401135F000E145BA2EC09F0BA
:10319000A2EC09F05D9DA2EC09F0A2EC09F04A68EE
:1031A0004968A2EC09F0266B256B04012551135DDB
:1031B00026511459000139E3A2EC09F0A2EC09F000
:1031C00004012551660FE96E010E2621EA6EEF50CB
:1031D000806FA2EC09F0096B080E0401095D000183
:1031E0001CE2A2EC09F0A2EC09F004018031D8B095
:1031F0005D89D8A05D99A2EC09F0000166EC16F09B
:10320000A2EC09F0A2EC09F0D89004018033A2EC02
:1032100009F00401092B0001DFE3A2EC09F004012D
:10322000252B000E26230001C0E3A2EC09F0A2EC3E
:1032300009F0FF0E491A4A1AA2EC09F0010E040126
:1032400013250A6E000E14210B6E0A50660FE96EEC
:10325000010E0B20EA6EEF500A6E49500A5C000125
:10326000D8A4C5D0A2EC09F0020E040113250A6E01
:10327000000E14210B6E0A50660FE96E010E0B2032
:10328000EA6EEF500A6E4A500A5C0001D8A4AFD033
:10329000A2EC09F0A2EC09F0060E0401636FA2ECA7
:1032A00009F0A2EC09F013C460F4A2EC09F00301E8
:1032B000FD31000139E3A2EC09F0A2EC09F000EEC7
:1032C000B9F010EE4DF0080EE75204E0E6CFEEFF45
:1032D000E82EFAD7EF6AA2EC09F0D9EC53F0A2EC91
:1032E00009F004015B31000118E2A2EC09F00B6A5D
:1032F000040160290A6ED8B40B2AA2EC09F00A5026
:10330000660FE96E010E0B20EA6E0D0EEF6EA2EC59
:1033100009F00001EEEF24F006D0A2EC09F0A2ECD7
:1033200009F00401068B0001A2EC09F00301FF5132
:103330000001E8A851D0A2EC09F0A2EC09F00401C8
:10334000069DA2EC09F0A2EC09F0096BA2EC09F0D1
:10335000020E1325086E000E1421096E406B3F6BA0
:1033600004013F51085C40510958000130E3A2ECD0
:1033700009F0040E016E020E046E04013F51660F47
:10338000E96E010E4021EA6EEF504FEC00F0200E86
:1033900055EC01F0A2EC09F0092BA2EC09F0100E9B
:1033A000095D00010BE1A2EC09F0A2EC09F00401B7
:1033B000096BA2EC09F00D0E55EC01F00001A2EC36
:1033C00009F004013F2B000E40230001C9E3A2ECE9
:1033D00009F00D0E55EC01F0A2EC09F00301FF51CC
:1033E0000001E8A204D0A2EC09F026EC27F0A2EC40
:1033F00009F0A2EC09F00401626BA2EC09F00001F3
:1034000081AA0FD0A2EC09F00401622BA2EC09F012
:103410006229000106E0A2EC09F0010EEEEC01F0D9
:10342000EED7A2EC09F0929A899AA2EF09F0A2ECE9
:1034300009F0A2EC09F0F29AA2EC09F0A2EC09F072
:10344000486AA2EC09F0A2EC09F004015D9BA2EC31
:1034500009F0A2EC09F05D9DA2EC09F0096B080EE1
:103460000401095D0001D8B07DD0A2EC09F0A2EC06
:1034700009F0D8904832A2EC09F07BD8A2EC09F010
:10348000A2EC09F00401488E5DAF489EA2EC09F061
:103490005D35000106E2A2EC09F0A2EC09F0436AF6
:1034A0005AD0A2EC09F0432AA2EC09F0050E435CC5
:1034B00052E1A2EC09F05DD8A2EC09F0A2EC09F00F
:1034C000436AA2EC09F004015D35000144E3A2EC7B
:1034D00009F0A2EC09F0D8904832A2EC09F0A2EC75
:1034E00009F00401488E5DAF489EA2EC09F000018E
:1034F00040D8A2EC09F004015D3500011DE2A2EC08
:1035000009F0A2EC09F0D8904832A2EC09F0A2EC44
:1035100009F00401488E5DAF489EA2EC09F0A2ECD0
:1035200009F05D8BA2EC09F0A2EC09F0F28AA2ECA2
:1035300009F0000112000FD0A2EC09F0A2EC09F092
:1035400004015D8DA2EC09F0A2EC09F0F28AA2EC74
:1035500009F000011200A2EC09F00401092B00019E
:10356000D8A07DD7A2EC09F0A2EC09F0F28AA2EF74
:1035700009F0A2EC09F0E86A81BE010F040104BB66
:10358000010800011FE0A2EC09F0A2EC09F004011F
:10359000048B81AE049BA2EC09F0A2EC09F07EC47E
:1035A000BBFFA2EC09F0A2EC09F0BC6AA2EC09F0A6
:1035B000A2EC09F09E92A2EC09F0A2EC09F05D9F4A
:1035C00000011AD0A2EC09F09EA2D3D7A2EC09F018
:1035D000A2EC09F07DC4BBFFA2EC09F0A2EC09F05B
:1035E000BC6AA2EC09F0A2EC09F09E92A2EC09F0F0
:1035F000A2EC09F004015D8F0001A2EF09F0A2EC3A
:1036000009F0010E0301FEB9000E376E010E040130
:1036100002B3000E37160001D8A4A2EF09F0A2EC05
:1036200009F00301FD310001D8A0A2EF09F0A2ECDE
:1036300009F0A2EC09F00401069BA2EC09F0A2EC4F
:1036400009F0069D0001A2EC09F00E0E0401096FBD
:103650003A0E0401095D00012CE2A2EC09F001EE32
:1036600066F004010951E926000EEA22EF500A6EC5
:10367000030E0A5C010ED8A4000E376E0B6A0929EE
:103680000A6ED8B40B2A0A50660FE96E010E0B20A1
:10369000EA6EEF500A6EF00E0A5C010ED8A4000E1E
:1036A0003716000106E1A2EC09F00401092B000124
:1036B000CFE3A2EC09F0A2EC09F004010905636F65
:1036C000A2EC09F0A2EC09F00101735104010B6FA7
:1036D000A2EC09F00D0E635D010ED8A4000E376E4A
:1036E000000E0BB1010E37120001D8A4BFEF21F07C
:1036F000A2EC09F0A2EC09F000EEB9F010EE4DF0EA
:10370000080EE75204E0E6CFEEFFE82EFAD7EF6AA4
:10371000A2EC09F0D9EC53F0A2EC09F004015B3102
:103720000001D8A0BFEF21F0A2EC09F00401005184
:103730000001E8A88CD0A2EC09F0A2EC09F000EEA0
:10374000B9F010EE8CF0080EE75204E0E6CFEEFF81
:10375000E82EFAD7EF6AA2EC09F05EEC54F0A2EC86
:1037600009F004015B310001D8A0BFEF21F0A2EC09
:1037700009F0A2EC09F000EEB9F010EE95F0080E99
:10378000E75204E0E6CFEEFFE82EFAD7EF6AA2ECAC
:1037900009F05EEC54F0A2EC09F004015B31000189
:1037A000D8A0BFEF21F0A2EC09F0A2EC09F000EEE6
:1037B000B9F010EE9EF0080EE75204E0E6CFEEFFFF
:1037C000E82EFAD7EF6AA2EC09F05EEC54F0A2EC16
:1037D00009F004015B310001D8A0BFEF21F0A2EC99
:1037E00009F0A2EC09F000EEB9F010EEA7F0080E17
:1037F000E75204E0E6CFEEFFE82EFAD7EF6AA2EC3C
:1038000009F05EEC54F0A2EC09F004015B31000118
:10381000D8A0BFEF21F0A2EC09F0A2EC09F000EE75
:10382000B9F010EEB0F0080EE75204E0E6CFEEFF7C
:10383000E82EFAD7EF6AA2EC09F05EEC54F0A2ECA5
:1038400009F004015B310001D8A0BFEF21F0A2EC28
:1038500009F004010131000115E3A2EC09F0A2EC2A
:1038600009F00401266B530E256FA2EC09F000014C
:10387000D6EC53F0A2EC09F004015B310001D8A0B2
:10388000BFEF21F0A2EC09F0040101510001E8A210
:1038900015D0A2EC09F0A2EC09F00401266B5A0E37
:1038A000256FA2EC09F00001D6EC53F0A2EC09F070
:1038B00004015B310001D8A0BFEF21F0A2EC09F0B8
:1038C000040101510001E8A415D0A2EC09F0A2EC1A
:1038D00009F00401266B610E256FA2EC09F00001CE
:1038E000D6EC53F0A2EC09F004015B310001D8A042
:1038F000BFEF21F0A2EC09F0040101510001E8A69C
:1039000015D0A2EC09F0A2EC09F00401266B680EB8
:10391000256FA2EC09F00001D6EC53F0A2EC09F0FF
:1039200004015B310001D8A0BFEF21F0A2EC09F047
:10393000040101510001E8A815D0A2EC09F0A2ECA5
:1039400009F00401266B6F0E256FA2EC09F000014F
:10395000D6EC53F0A2EC09F004015B310001D8A0D1
:10396000BFEF21F0A2EC09F0040101510001E8AA27
:1039700015D0A2EC09F0A2EC09F00401266B760E3A
:10398000256FA2EC09F00001D6EC53F0A2EC09F08F
:1039900004015B310001D8A0BFEF21F0A2EC09F0D7
:1039A000040101510001E8AC15D0A2EC09F0A2EC31
:1039B00009F00401266B7D0E256FA2EC09F00001D1
:1039C000D6EC53F0A2EC09F004015B310001D8A061
:1039D000BFEF21F0A2EC09F004010135000115E36D
:1039E000A2EC09F0A2EC09F00401266B840E256F0D
:1039F000A2EC09F00001D6EC53F0A2EC09F00401AE
:103A00005B310001D8A0BFEF21F0A2EC09F0040166
:103A100000510001E8AC15D0A2EC09F0A2EC09F0CD
:103A20000401266B8B0E256FA2EC09F00001D6EC89
:103A300053F0A2EC09F004015B310001D8A0BFEF04
:103A400021F0A2EC09F004010035000115E3A2EC1D
:103A500009F0A2EC09F00401266B920E256FA2EC8E
:103A600009F00001D6EC53F0A2EC09F004015B313F
:103A70000001D8A0BFEF21F0A2EC09F0A2EC09F000
:103A800000EEB9F00A0EF76E0E0EF66EB5EC02F00F
:103A9000EF6AA2EC09F0D9EC53F0A2EC09F00401B2
:103AA0005B31000104E2A2EC09F0A0EC24F0A2ECEE
:103AB00009F0A2EC09F004015E95A2EC09F0A2EC79
:103AC00009F000EEB9F0480EEE6E550EEE6EEF6A9C
:103AD000A2EC09F00001D9EC53F0A2EC09F00401CA
:103AE0005B31000124E2A2EC09F04D500A6E480E51
:103AF0000A5C1CE1A2EC09F04E500A6E410E0A5C11
:103B0000010ED8A4000E376E4E500A6E470E0A5CA6
:103B1000010ED8A4000E371205E0A2EC09F041EC2A
:103B200024F004D0A2EC09F0A0EC24F0DDD0A2EC4B
:103B300009F0A2EC09F000EEB9F0530EEE6E4B0E58
:103B4000EE6EEF6AA2EC09F0D9EC53F0A2EC09F0AA
:103B500004015B3100011DE2A2EC09F04D500A6E38
:103B60004F0E0A5C010ED8A4000E376E4E500A6E3E
:103B70004D0E0A5C010ED8A4000E371605E0A2EC2B
:103B800009F041EC24F004D0A2EC09F0A0EC24F000
:103B9000ABD0A2EC09F0A2EC09F000EEB9F0500EA7
:103BA000EE6E4C0EEE6EEF6AA2EC09F0D9EC53F01B
:103BB000A2EC09F004015B3100012CE2A2EC09F057
:103BC0004D500A6E530E0A5C24E1A2EC09F04E50EF
:103BD0000A6E500E0A5C010ED8A4000E376E4E50CD
:103BE0000A6E510E0A5C010ED8A4000E37124E5018
:103BF0000A6E520E0A5C010ED8A4000E371205E0C0
:103C0000A2EC09F041EC24F004D0A2EC09F0A0EC05
:103C100024F06AD0A2EC09F0A2EC09F000EEB9F0B1
:103C2000410EEE6E540EEE6EEF6AA2EC09F0D9EC86
:103C300053F0A2EC09F004015B3100011DE2A2EC9B
:103C400009F04D500A6E4F0E0A5C010ED8A4000E0A
:103C5000376E4E500A6E450E0A5C010ED8A4000E57
:103C6000371605E0A2EC09F041EC24F004D0A2ECF8
:103C700009F0A0EC24F038D0A2EC09F0A2EC09F095
:103C800000EEB9F0430EEE6E5A0EEE6EEF6AA2EC45
:103C900009F0D9EC53F0A2EC09F004015B3100010A
:103CA00023E2A2EC09F04D500A6E4F0E0A5C1CE1B3
:103CB000A2EC09F04E500A6E4B0E0A5C010ED8A41D
:103CC000000E376E4E500A6E4C0E0A5C010ED8A4E0
:103CD000000E371205E0A2EC09F041EC24F004D00C
:103CE000A2EC09F0A0EC24F0A2EC09F004015E5172
:103CF0000001E8B4BFEF21F0A2EC09F0A2EC09F05A
:103D00000401049F0001A2EC09F0A2EC09F000EE0E
:103D1000B9F0570EEE6E490EEE6E440EEE6E450E85
:103D2000EE6E310EEE6EEF6AA2EC09F0D9EC53F0B4
:103D3000A2EC09F004015B310001D8B06FD0A2EC15
:103D400009F0A2EC09F00B6A060E04010A250A6EBE
:103D5000D8B00B2A0A50660FE96E010E0B20EA6EEE
:103D6000EF500B6FA2EC09F0A2EC09F00B31D8B0C8
:103D70000685D8A00695A2EC09F0096B070E040190
:103D8000095D00013EE2A2EC09F0A2EC09F000EEB0
:103D90004DF004010951EB500A6ED8900A340B6FB4
:103DA000A2EC09F0060E095D000112E1A2EC09F097
:103DB000A2EC09F00401D89206B5D882D8B20B81E2
:103DC000D8A20B91A2EC09F0A2EC09F0600E0B1343
:103DD0000001A2EC09F004010A5109250A6E0B6AE0
:103DE0000B36A2EC09F00A50660FE96E010E0B20AB
:103DF000EA6E0BC4EFFFA2EC09F00401092B0001ED
:103E0000BDE3A2EC09F0A2EC09F00401048FA2ECDE
:103E100009F006510001E8B444D108D0A2EC09F041
:103E2000040100310001D8B0BFEF21F0A2EC09F08D
:103E3000A2EC09F004015E95A2EC09F0A2EC09F0F5
:103E400000EEB9F0570EEE6E490EEE6E440EEE6EB9
:103E5000450EEE6E320EEE6EEF6AA2EC09F0000136
:103E600088EC23F0A2EC09F0A2EC09F000EEB9F026
:103E7000570EEE6E490EEE6E440EEE6E450EEE6E71
:103E8000330EEE6EEF6AA2EC09F088EC23F0A2ECA0
:103E900009F0A2EC09F000EEB9F0570EEE6E490EF3
:103EA000EE6E440EEE6E450EEE6E340EEE6EEF6A62
:103EB000A2EC09F088EC23F0A2EC09F0A2EC09F0E6
:103EC00000EEB9F0570EEE6E490EEE6E440EEE6E39
:103ED000450EEE6E350EEE6EEF6AA2EC09F088EC40
:103EE00023F0A2EC09F0A2EC09F000EEB9F0570EB5
:103EF000EE6E490EEE6E440EEE6E450EEE6E360E12
:103F0000EE6EEF6AA2EC09F088EC23F0A2EC09F067
:103F1000A2EC09F000EEB9F0570EEE6E490EEE6E0F
:103F2000440EEE6E450EEE6E370EEE6EEF6AA2ECAC
:103F300009F088EC23F0A2EC09F004015E510001C5
:103F4000E8B4AFD0A2EC09F0040104350001D8B008
:103F5000A8D0A2EC09F0A2EC09F000EEB9F0570EDF
:103F6000EE6E490EEE6E440EEE6E450EEE6EEF6A8C
:103F7000A2EC09F0D9EC53F0A2EC09F0310E0401E7
:103F8000635D0001D8B08DD0A2EC09F004015B3173
:103F90000001D8B083D0A2EC09F0010E0401406FFB
:103FA0002C0E3F6F0401405304E10A513F5D0001B4
:103FB00023E3A2EC09F0070E04013F250A6E000E70
:103FC00040210B6EA2EC09F03F51660FE96E010E25
:103FD0004021EA6EEFCF0CF00A50660FE96E010E39
:103FE0000B20EA6E0CC0EFFFA2EC09F004013F07C2
:103FF000000E405B0001D6E2A2EC09F00401096B5F
:10400000070E0401095D000133E2A2EC09F0A2EC05
:1040100009F000EE4DF004010951EB500A6ED89002
:104020000A340B6FA2EC09F0060E095D000107E1EE
:10403000A2EC09F0A2EC09F0600E04010B130001E0
:10404000A2EC09F004010A5109250A6E0B6A0B362D
:10405000A2EC09F00A50660FE96E010E0B20EA6E21
:104060000BC4EFFFA2EC09F00401092B0001C8E327
:10407000A2EC09F0A2EC09F00401048FA2EC09F013
:10408000A2EC09F0070E6327A2EC09F0A2EC09F0FC
:10409000070E1327000E1423000103D0A2EC09F031
:1040A0006ED1A2EC09F0040100510001E8A86DD026
:1040B000A2EC09F0A2EC09F000EE8CF010EE95F005
:1040C000080EE75204E0E6CFEEFFE82EFAD7EF6ADB
:1040D000A2EC09F0A2EC09F000EE95F010EE9EF0D3
:1040E000080EE75204E0E6CFEEFFE82EFAD7EF6ABB
:1040F000A2EC09F0A2EC09F000EE9EF010EEA7F0A1
:10410000080EE75204E0E6CFEEFFE82EFAD7EF6A9A
:10411000A2EC09F0A2EC09F000EEA7F010EEB0F06E
:10412000080EE75204E0E6CFEEFFE82EFAD7EF6A7A
:10413000A2EC09F00401096B070E0401095D0001FE
:104140001EE2A2EC09F0A2EC09F00D6A070E0401D0
:1041500009250C6ED8B00D2A0C50660FE96E010EC1
:104160000D20EA6EEFCF0AF000EEB0F009510AC060
:10417000EBFFA2EC09F00401092B0001DDE3A2EC46
:1041800009F0A2EC09F004010E6B0001A2EC09F0A9
:10419000A2EC09F001016C5104010B6FA2EC09F0D3
:1041A000A2EC09F07E0E0B17A2EC09F0A2EC09F0CC
:1041B000E00E0B13A2EC09F0A2EC09F00BC46CF1B9
:1041C000A2EC09F0A2EC09F00101735104010B6F9C
:1041D000A2EC09F0A2EC09F07E0E0B17A2EC09F09C
:1041E000A2EC09F0600E0B13A2EC09F0A2EC09F0AE
:1041F0000BC473F1A2EC09F0140E096F040109510C
:10420000635D000139E3A2EC09F0A2EC09F001EED4
:1042100066F004010951E926000EEA22EF500B6F07
:10422000A2EC09F0000E0BBF010E376E000E00B1BC
:10423000010E37160001D8A4A2D0A2EC09F0A2EC1E
:1042400009F004010B91A2EC09F0A2EC09F0E00ED8
:104250000B13A2EC09F0A2EC09F001EE66F0095193
:10426000E926000EEA220BC4EFFFA2EC09F0070ECC
:10427000040109270001C2E3A2EC09F0A2EC09F055
:1042800001EE66F004016351E926000EEA22EF50C8
:104290000B6FA2EC09F0A2EC09F00B9FA2EC09F065
:1042A000A2EC09F00B8DA2EC09F0A2EC09F00B8B4B
:1042B000A2EC09F0A2EC09F00B81A2EC09F0A2EC4F
:1042C00009F001EE66F06351E926000EEA220BC404
:1042D000EFFFA2EC09F002510001E8A204D0A2EC29
:1042E00009F026EC27F0A2EC09F00301FE510001D1
:1042F000E8A845D0A2EC09F05BD9A2EC09F00401D2
:10430000406B3F6B04013F51135D40511459000154
:104310001AE3A2EC09F0A2EC09F004013F51660F88
:10432000E96E010E4021EA6EEF50476EA2EC09F0F3
:104330000001C8EC15F0A2EC09F004013F2B000EBF
:1043400040230001DFE3A2EC09F0A3D9A2EC09F0BD
:104350000301FF31000106E3A2EC09F0A2EC09F031
:104360000401068D0001A2EC09F00301FF510001D8
:10437000E8A605D0A2EC09F00D0E55EC01F0A2EC78
:1043800009F0A2EC09F00401068FA2EC09F000018B
:104390001200A2EC09F081AA01D1A2EC09F0A2EC72
:1043A00009F004015B91A2EC09F0A2EC09F03E6A6D
:1043B0003D6AA2EC09F0A2EC09F0406A3F6AA2EC67
:1043C00009F0A2EC09F0048B81AE049BA2EC09F089
:1043D0000001E86A81BE010F040104BB010800016D
:1043E000D8B4F6D7A2EC09F0E86A81BE010F040147
:1043F00004BB0108000117E0A2EC09F03D4A3E2A87
:10440000A2EC09F0010E3E5C06E3D8A4C7D0FF0E73
:104410003D5CD8B0C3D0A2EC09F0350EE82EFED733
:1044200000000001E1D7A2EC09F0E86A81BE010FAB
:10443000040104BB0108000117E1A2EC09F03F4AA6
:10444000402AA2EC09F0010E405C06E3D8A4A6D0F5
:10445000FF0E3F5CD8B0A2D0A2EC09F0350EE82EDA
:10446000FED700000001E1D7A2EC09F03E5203E1C3
:104470003C0E3D5C02E3000E01D0010E376E40524F
:1044800004E13C0E3F5C000102E3000E01D0010E8E
:1044900037120001D8A482D0A2EC09F03E5205E107
:1044A000510E3D5C02E2000E01D0010E376E3E520D
:1044B00003E1780E3D5C02E3000E01D0010E3716D9
:1044C0000001D8A46BD0A2EC09F0405205E1510ED6
:1044D0003F5C02E2000E01D0010E376E405203E154
:1044E000780E3F5C02E3000E01D0010E371600018A
:1044F000D8A454D0A2EC09F03E5205E1A10E3D5CD7
:1045000002E2000E01D0010E376E3E5203E1B40EFE
:104510003D5C02E3000E01D0010E37160001D8A465
:104520003DD0A2EC09F0405205E1A10E3F5C02E251
:10453000000E01D0010E376E405203E1B40E3F5C15
:1045400002E3000E01D0010E3716000127E1A2ECB4
:1045500009F0A2EC09F00401266B256BA2EC09F02E
:10456000000181AA19D0A2EC09F00401252B000E4C
:104570002623A2EC09F0010EEEEC01F0A2EC09F00A
:104580000B0E265D000106E309E1B90E0401255D6D
:10459000000104E20001E4D7A2EF09F0A2EC09F067
:1045A000A2EC09F004015B81A2EC09F00001120009
:1045B000A2EC09F0EEDEA2EC09F004015B3100018F
:1045C000F7E3A2EC09F0DCEC01F0A2EC09F0A2ECBC
:1045D00009F0040125518303F4CF26F4F3CF25F429
:1045E000A2EC09F00B6B0401265304E10B51255D8D
:1045F00000010CE3A2EC09F0150EE82EFED7000036
:10460000A2EC09F004010B2B0001EDE3A2EC09F090
:10461000C0DEA2EC09F004015B310001C9E3A2ECA9
:1046200009F00301FF510001E8B604D0A2EC09F043
:1046300094908B80A2EC09F026EC51F0A2EC09F0EA
:10464000A2EC09F04A684968A2EC09F0A2EC09F072
:104650007DC4BBFFA2EC09F0A2EC09F0BC6AA2EC9D
:1046600009F0A2EC09F09E92A2EC09F0A2EC09F08C
:10467000FCC30BF4A2EC09F098EC16F0A2EC09F0E4
:10468000A2EC09F00401166B156BA2EC09F0000115
:104690001200A2EC09F00301FF510001E8A606D0C8
:1046A000A2EC09F00D0E55EC01F02CD0A2EC09F0B3
:1046B000A2EC09F0FF0E4A180401806FA2EC09F089
:1046C000A2EC09F0FF0E4918476EA2EC09F00001B8
:1046D000C8EC15F0A2EC09F0A2EC09F080C447F098
:1046E000A2EC09F0C8EC15F0A2EC09F0A2EC09F07C
:1046F00085C40BF4A2EC09F098EC16F0A2EC09F0DA
:104700009EA2FED7A2EC09F094908B90A2EF09F044
:10471000A2EC09F0D9EC53F0A2EC09F004015B31F2
:104720000001D8B0ACD0A2EC09F0A2EC09F00B6A01
:10473000060E04010A250A6ED8B00B2A0A50660F2D
:10474000E96E010E0B20EA6EEF500B6FA2EC09F040
:10475000A2EC09F00B31D8B00685D8A00695A2ECE2
:1047600009F0A2EC09F0D8900B33A2EC09F0A2EC0E
:1047700009F00F0E0B17A2EC09F00B530001D8A49F
:1047800056D0A2EC09F0040104350001D8B04DD098
:10479000A2EC09F00401096B070E0401095D000198
:1047A0003EE2A2EC09F0A2EC09F000EE4DF00401AB
:1047B0000951EB500A6ED8900A340B6FA2EC09F045
:1047C000060E095D000112E1A2EC09F0A2EC09F06D
:1047D000600E04010B13A2EC09F0A2EC09F0D892D0
:1047E00006B5D882D8B20B81D8A20B910001A2ECF9
:1047F00009F004010A5109250A6E0B6A0B36A2EC76
:1048000009F00A50660FE96E010E0B20EA6E0BC428
:10481000EFFFA2EC09F00401092B0001BDE3A2ECBB
:1048200009F0A2EC09F00401048F000127D0A2ECEA
:1048300009F004010B07A2EC09F0A2EC09F0D890F2
:104840000B37A2EC09F0A2EC09F0D89206B5D88299
:10485000D8B20B81D8A20B91A2EC09F00B6A060E1C
:104860000A250A6ED8B00B2AA2EC09F00A50660F8E
:10487000E96E010E0B20EA6E0BC4EFFF0001A2EF00
:1048800009F0A2EC09F0A2EC09F00B6A060E040193
:104890000A250A6ED8B00B2A0A50660FE96E010E7F
:1048A0000B20EA6EEF500B6FA2EC09F0A2EC09F0BE
:1048B0000B31D8B00685D8A00695A2EC09F0A2EC81
:1048C00009F0D8900B33A2EC09F0A2EC09F00F0E1E
:1048D0000B17A2EC09F00B53000108E1A2EC09F060
:1048E000A2EC09F004015E85000127D0A2EC09F0DA
:1048F00004010B07A2EC09F0A2EC09F0D8900B37E9
:10490000A2EC09F0A2EC09F0D89206B5D882D8B290
:104910000B81D8A20B91A2EC09F00B6A060E0A25B6
:104920000A6ED8B00B2AA2EC09F00A50660FE96EA5
:10493000010E0B20EA6E0BC4EFFF0001A2EF09F09D
:10494000A2EC09F0070E0401135D086E000E145965
:10495000096E406B0AC43FF404013F51085C4051AA
:104960000958000123E3A2EC09F0A2EC09F0070EBC
:1049700004013F250C6E000E40210D6E0C50660F99
:10498000E96E010E0D20EA6EEFCF0AF03F51660F7F
:10499000E96E010E4021EA6E0AC0EFFFA2EC09F0B9
:1049A00004013F2B000E40230001D6E3A2EC09F0E6
:1049B000A2EC09F0070E0401635FA2EC09F0A2EC7F
:1049C00009F0070E135F000E145BA2EC09F0A2ECD5
:1049D00009F05E85A2EC09F000011200A2EC09F0DA
:1049E000A2EC09F00401069BA2EC09F0096B070E8A
:1049F0000401095D00011EE2A2EC09F0A2EC09F03D
:104A00000D6A070E040109250C6ED8B00D2A0C5052
:104A1000660FE96E010E0D20EA6EEFCF0AF000EE90
:104A200084F009510AC0EBFFA2EC09F00401092B44
:104A30000001DDE3A2EC09F0A2EC09F08A510C6E52
:104A40007E0E0C140A6E0AC08AF0A2EC09F0070E62
:104A50000401096F3A0E0401095D00012CE2A2EC89
:104A600009F001EE66F004010951E926000EEA2280
:104A7000EF500A6E030E0A5C010ED8A4000E376ECA
:104A80000B6A09290A6ED8B40B2A0A50660FE96E20
:104A9000010E0B20EA6EEF500A6EF00E0A5C010E5A
:104AA000D8A4000E3716000106E1A2EC09F00401BB
:104AB000092B0001CFE3A2EC09F0A2EC09F0020EF1
:104AC00004010927A2EC09F0180E095D000109E3B1
:104AD000A2EC09F0A2EC09F0020E0401636F0001E0
:104AE00017D0A2EC09F0110E0401095D000109E3E1
:104AF000A2EC09F0A2EC09F0010E0401636F0001C1
:104B000006D0A2EC09F0A2EC09F00401636B0001ED
:104B1000A2EC09F004010A6B0A0E04010A5D00010F
:104B200020E2A2EC09F0040109510A250A6E0B6A81
:104B30000B360A50660FE96E010E0B20EA6EEF503D
:104B40000A6E00EE7AF00A51EB500C6E0A500C5CC3
:104B50000001D8A4EDD0A2EC09F004010A2B000159
:104B6000DBE3A2EC09F094988B88A2EC09F04EEC00
:104B70004FF0A2EC09F06BEC2CF0A2EC09F0A2ECE7
:104B800009F00401058FA2EC09F00001F9EC2CF00A
:104B9000A2EC09F0D8EC22F0A2EC09F00401096BB8
:104BA000070E0401095D000115E2A2EC09F0A2EC78
:104BB00009F000EE84F004010951EB50476EA2ECBD
:104BC00009F00001C8EC15F0A2EC09F00401092B72
:104BD0000001E6E3A2EC09F0A2EC09F000EEB9F066
:104BE00010EE4DF0080EE75204E0E6CFEEFFE82E9F
:104BF000FAD7EF6AA2EC09F0A2EC09F0600E4B6E56
:104C0000A2EC09F004016353000107E1A2EC09F0F2
:104C1000A2EC09F0610E4B6E3FD0A2EC09F0E0EC83
:104C20004EF0A2EC09F0A2EC09F000EEB9F00A0E89
:104C3000F76E160EF66EB5EC02F0010EEE6EEE6A31
:104C4000A2EC09F0A2EC09F0E10E4B6EA2EC09F027
:104C5000010E0401635D00011FE0A2EC09F0A2EC6B
:104C600009F0E00E4B6EA2EC09F0E0EC4EF0A2EC85
:104C700009F0A2EC09F000EEB9F00A0EF76E1E0E74
:104C8000F66EB5EC02F0020EEE6EEE6AA2EC09F0E2
:104C9000A2EC09F0E10E4B6EA2EC09F0E0EC4EF054
:104CA000A2EC09F0A2EC09F0030E476EA2EC09F0A9
:104CB000C8EC15F0A2EC09F0A2EC09F0F00E476E7A
:104CC000A2EC09F0C8EC15F0A2EC09F0A2EC09F096
:104CD0000401096BA2EC09F0000101EE66F0040189
:104CE0000951E926000EEA22EF500A6E0A5200012D
:104CF00018E0A2EC09F0A2EC09F001EE66F0040164
:104D00000951E926000EEA22EF50476EA2EC09F0A5
:104D10000001C8EC15F0A2EC09F00401092B000118
:104D2000DBD7A2EC09F049EC23F0A2EC09F020D08B
:104D3000A2EC09F009C40AF404010A51605D000103
:104D400012E3A2EC09F001EE66F004010A51E92633
:104D5000000EEA22EF5055EC01F0A2EC09F004013C
:104D60000A2B0001E9E3A2EC09F00D0E55EC01F06D
:104D7000A2EC09F0A2EC09F00401068FA2EC09F004
:104D8000A2EC09F0059FA2EC09F0A2EC09F0069D47
:104D9000A2EC09F094988B98A2EC09F00001F7EFCF
:104DA00019F0A2EC09F0C00E55EC01F0040182519B
:104DB00055EC01F0A2EC09F0406B3F6B04013F5150
:104DC000135D4051145900013AE3A2EC09F00401CB
:104DD0003F51660FE96E010E4021EA6EEF500A6EF8
:104DE000C00E0A5C010ED8A4000E376E3F51660F4C
:104DF000E96E010E4021EA6EEF500A6EDB0E0A5C8E
:104E0000010ED8A4000E3712000105E0A2EC09F053
:104E1000DB0E55EC01F0A2EC09F004013F51660FE6
:104E2000E96E010E4021EA6EEF5055EC01F0A2EC64
:104E300009F004013F2B000E40230001BFE3A2EC68
:104E400009F0C00E55EC01F0A2EF09F0A2EC09F058
:104E5000A2EC09F00401069DA2EC09F0010E030189
:104E6000FFB1000E376E010EFFB3000E3716010EB4
:104E7000040102B3000E371600010AE0A2EC09F0AB
:104E8000A2EC09F00401068FA2EC09F00001120067
:104E9000A2EC09F0000E0301FFB5010E376E010E02
:104EA000040102B3000E371600010DE0A2EC09F078
:104EB00078DFA2EC09F0A2EC09F00401068FA2EC65
:104EC00009F000011200A2EC09F00E0E0401096FB6
:104ED0003A0E0401095D00012CE2A2EC09F001EE9A
:104EE00066F004010951E926000EEA22EF500A6E2D
:104EF000030E0A5C010ED8A4000E376E0B6A092956
:104F00000A6ED8B40B2A0A50660FE96E010E0B2008
:104F1000EA6EEF500A6EF00E0A5C010ED8A4000E85
:104F20003716000109E1A2EC09F00401092B000188
:104F3000CFE3A2EC09F070D1A2EC09F0A2EC09F0E9
:104F400004010905636FA2EC09F0096B070E040167
:104F5000095D000125E2A2EC09F0A2EC09F00B6A60
:104F6000070E040109250A6ED8B00B2A0A50660FF5
:104F7000E96E010E0B20EA6EEF500B6FA2EC09F008
:104F8000A2EC09F0D8900B310A6E00EEB9F009518D
:104F90000AC0EBFFA2EC09F00401092B0001D6E3E3
:104FA000A2EC09F0A2EC09F0BF510C6E0F0E0C142C
:104FB0000A6E0AC0BFF0A2EC09F012EC4FF0A2ECAE
:104FC00009F03E0E55EC01F0A2EC09F00401096B6A
:104FD000070E0401095D00011BE2A2EC09F0A2EC3E
:104FE00009F001EE66F004010951E926000EEA22FB
:104FF000EF500C6ED8900C300A6E00EEB9F00951EB
:105000000AC0EBFFA2EC09F00401092B0001E0E368
:10501000A2EC09F0A2EC09F0BF510C6E0F0E0C14BB
:105020000A6E0AC0BFF0A2EC09F012EC4FF0A2EC3D
:1050300009F0A2EC09F00D0E04010A6FA2EC09F0D0
:10504000A2EC09F001EE66F00A51E926000EEA2210
:10505000EF500B6FA2EC09F00B310001D8B057D024
:10506000A2EC09F02C0E55EC01F0A2EC09F00401C1
:10507000096B070E0401095D00011EE2A2EC09F0B4
:1050800004010A2BA2EC09F0A2EC09F001EE66F093
:105090000A51E926000EEA22EF500C6ED8900C302F
:1050A0000A6E00EEB9F009510AC0EBFFA2EC09F05C
:1050B0000401092B0001DDE3A2EC09F0A2EC09F0E8
:1050C000BF510C6E0F0E0C140A6E0AC0BFF0A2EC9A
:1050D00009F012EC4FF0A2EC09F001EE66F00401C9
:1050E0000A51E926000EEA22EF500A6E800E0A5C91
:1050F000000105E3A2EC09F02A0E55EC01F0A2EC48
:1051000009F0040163510A5D0001D8A0A9D7A2ECFF
:1051100009F0A2EC09F0030E040163250A6FA2EC6A
:1051200009F03A0E55EC01F0A2EC09F0406B0AC40C
:105130003FF404013F51135D405114590001D8A0C0
:105140006BD0A2EC09F0040100510001E8A44ED09C
:10515000A2EC09F004013F51660FE96E010E4021F7
:10516000EA6EEF500A6E200E0A5C000102E2000EA9
:1051700001D0010E376E04013F51660FE96E010E3A
:105180004021EA6EEF500A6E0D0E0A5C010ED8A4A3
:10519000000E37123F51660FE96E010E4021EA6E94
:1051A000EF500A6E0A0E0A5C010ED8A4000E3712E8
:1051B0003F51660FE96E010E4021EA6EEF500A6E14
:1051C000080E0A5C010ED8A4000E371200010CE094
:1051D000A2EC09F004013F51660FE96E010E402177
:1051E000EA6EEF5055EC01F000010CD0A2EC09F092
:1051F00004013F51660FE96E010E4021EA6EEF5047
:1052000055EC01F00001A2EC09F004013F2B000E67
:1052100040230001D8A08DD7A2EC09F00D0E55EC6B
:1052200001F0A2EC09F0A2EC09F00401068FA2EC57
:1052300009F000011200A2EC09F0A2EC09F004014F
:105240000485A2EC09F0A2EC09F00301FF93A2ECA3
:1052500009F0A2EC09F0FF91A2EC09F0A2EC09F030
:10526000FE9DA2EC09F0A2EC09F004010599A2EC64
:1052700009F0A2EC09F0630E086FA2EC09F0A2ECB1
:1052800009F00A0E656FA2EC09F0A2EC09F0069194
:10529000A2EC09F0A2EC09F0068FA2EC09F0A2EC56
:1052A00009F00097A2EC09F0A2EC09F00587A2EC46
:1052B00009F0000181A010D0A2EC09F0A2EC09F0E5
:1052C0000301FF8BA2EC09F0A2EC09F0FF9FA2EC16
:1052D00009F0A2EC09F0FF9D0001A2EC09F082B6F2
:1052E00006D0A2EC09F0A2EC09F0090E536EA2EC74
:1052F00009F0010E136EF40EEFEC01F0A2EC09F0D0
:10530000A2EC09F004010A6BA2EC09F0A2EC09F08E
:105310005D93A2EC09F0A2EC09F0266BAA0E256FB2
:10532000A2EC09F00301FD35000130E3A2EC09F025
:10533000630E04010A5D000129E2A2EC09F0A2EC6F
:1053400009F004010A512525A96E000E2621AA6E36
:10535000B0EC01F00B6FA2EC09F00D0E0B5D00013B
:1053600015E0A2EC09F05C0E04010B5D000108E100
:10537000A2EC09F0A2EC09F004015D83000106D063
:10538000A2EC09F004010A2B0001D2D7A2EC09F02B
:10539000A3EF10F0A2EC09F0A2EC09F00401059DC6
:1053A000A2EC09F00301FF510001E8AC2ED0A2EC01
:1053B00009F0A2EC09F001EE66F0470EEE6E500E19
:1053C000EE6E470EEE6E4C0EEE6EEE6EEF6AA2ECD7
:1053D00009F0130E056E880E026E27EC01F0D8A0BE
:1053E000CAD14708FAE127EC01F0D8A0C4D14C0893
:1053F000F4E127EC01F0D8A0BED14C08EEE127EC97
:1054000001F0D8A0B8D104010B6F0001A2EC09F0A3
:105410000301FF3500012EE3A2EC09F0A2EC09F034
:1054200001EE66F0470EEE6E500EEE6E470EEE6E1B
:10543000EE6E410EEE6EEF6AA2EC09F0130E056EF1
:10544000880E026E27EC01F0D8A095D14708FAE14A
:1054500027EC01F0D8A08FD14708F4E127EC01F048
:10546000D8A089D14108EEE127EC01F0D8A083D182
:1054700004010B6F0001A2EC09F00301FF510001D0
:10548000E8AA2FD0A2EC09F0A2EC09F001EE66F038
:10549000470EEE6E500EEE6E520EEE6E4D0EEE6E2E
:1054A000430EEE6EEF6AA2EC09F0130E056E880E45
:1054B000026E27EC01F0D8A05ED15208FAE127EC89
:1054C00001F0D8A058D14D08F4E127EC01F0D8A0A4
:1054D00052D14308EEE127EC01F0D8A04CD10401F1
:1054E0000B6F0001A2EC09F0A2EC09F0060E456E6C
:1054F000A2EC09F0A2EC09F00BC46BF1A2EC09F0EC
:10550000056AC80E026E27EC01F0D8A043D704014B
:105510000B6FA2EC09F0A2EC09F001EE66F0455029
:10552000E926000EEA220BC4EFFFA2EC09F0452A9F
:10553000A2EC09F02A0E04010B5D010ED8A4000EA6
:10554000376E500E455C010ED8A4000E37120001D4
:10555000D5E0A2EC09F0010E366E020E046E05ECE9
:1055600000F00401606FA2EC09F0A2EC09F001EE7A
:1055700066F04550E926000EEA22EF6AA2EC09F037
:10558000A2EC09F0096BA2EC09F0A2EC09F08C6B1B
:10559000A2EC09F0000101EE66F004010951E926D0
:1055A000000EEA22EF500A6E2A0E0A5C000113E098
:1055B000A2EC09F0A2EC09F001EE66F00401095139
:1055C000E926000EEA22EF500A6E8C1BA2EC09F0CD
:1055D000092B0001DFD7A2EC09F0040160514B5CFC
:1055E000000107E0A2EC09F0949A8B9AA2EC09F072
:1055F000D1D6A2EC09F0949A8B8AA2EC09F0A2EC25
:1056000009F004010A6BA2EC09F000017AEC5EF0EB
:10561000A2EC09F001EE66F004010A51E926000E41
:10562000EA22EF500A6E410E0A5C00010CE1A2EC86
:1056300009F0A2EC09F004015D85A2EC09F0949850
:105640008B8800010AD0A2EC09F0A2EC09F0040159
:105650005D95A2EC09F094988B980001A2EC09F0FA
:1056600004015D510001E8A47CD0A2EC09F0000E19
:105670000301FEBB010E376E000E04015DB3010E87
:105680003716000104E0A2EC09F0F3EC54F0A2ECB0
:1056900009F0A3EC5EF0A2EC09F081A005D0A2EC29
:1056A00009F01EEC57F053D0A2EC09F0A2EC09F07F
:1056B00004010A6BA2EC09F0000101EE66F004019E
:1056C0000A51E926000EEA22EF500A6E2A0E0A5C01
:1056D000D8A4010E376E500E0A5D010ED8B0000E30
:1056E0003716000106E0A2EC09F004010A2B0001C4
:1056F000E3D7A2EC09F0500E04010A5D000108E3B3
:10570000A2EC09F0A2EC09F004015D8100011ED0B9
:10571000A2EC09F00B6A04010A290A6ED8B40B2A1C
:10572000A2EC09F00A50660FE96E010E0B20EA6E3A
:105730000D0EEF6EA2EC09F0A2EC09F03E6BAA0E82
:105740003D6FA2EC09F0A2EC09F05D910001A2EC22
:1057500009F004015D31000104E2A2EC09F03FEC24
:1057600015F0A2EC09F0A2EC09F00401068FA2ECFE
:1057700009F000011200A2EC09F094988B98A2ECB9
:1057800009F0949A8B9AA2EF09F0A2EC09F0056A4D
:10579000010E026E27EC01F00AE3466EA2EC09F05E
:1057A00008D8A2EC09F097D8A2EC09F022D9A2EF10
:1057B00009F0A2EC09F0040100510001E8A605D0AF
:1057C000A2EC09F0465055EC01F0A2EC09F00D0EE8
:1057D000465C010ED8A4000E376E0A0E465C010E20
:1057E000D8A4000E3712D8A4A2EF09F0A2EC09F059
:1057F000A2EC09F0010E456EA2EC09F0A2EC09F052
:1058000046C066F1A2EC09F0130E056E880E026E1A
:1058100027EC01F0D8A051D0466EA2EC09F00401AB
:1058200000510001E8A605D0A2EC09F0465055EC65
:1058300001F0A2EC09F0080E465C0AE1A2EC09F0C6
:10584000455203E0A2EC09F04506A2EC09F0DAD7D4
:10585000A2EC09F00D0E465C010ED8A4000E376EC6
:105860000A0E465C010ED8A4000E37124528010E20
:10587000D8A4000E37120FE0A2EC09F0A2EC09F058
:1058800001EE66F04550E926000EEA220D0EEF6E9D
:10589000A2EF09F00CD0A2EC09F0A2EC09F001EEA5
:1058A00066F04550E926000EEA2246C0EFFFA2EC62
:1058B00009F0452AA2EC09F0A5D7A2EC09F0A2EC68
:1058C00009F001EE66F04550E926000EEA220D0EC1
:1058D000EF6EA2EF09F0A2EC09F0A2EC09F00401CE
:1058E0000A6BA2EC09F0000101EE66F004010A5116
:1058F000E926000EEA22EF500A6E200E0A5CD8A4B8
:10590000010E376E01EE66F00A51E926000EEA221A
:10591000EF500A6E0D0E0A5CD8A4010E3716FD0E6C
:105920000A5D010ED8B0000E37160001D8B452D06F
:10593000A2EC09F001EE66F004010A51E926000E1E
:10594000EA22EF500A6E610E0A5C000ED8B0010E1A
:10595000376E01EE66F00A51E926000EEA22EF509A
:105960000A6E7B0E0A5C000102E3000E01D0010EFC
:10597000371618E0A2EC09F0A2EC09F001EE66F08F
:1059800004010A51E926000EEA22EF500C6EDF0EE8
:105990000C140A6E01EE66F00A51E926000EEA22A6
:1059A0000AC0EFFF0001A2EC09F0A2EC09F001EE41
:1059B00066F004010A51E926000EEA22EFCF0AF050
:1059C00000EEB9F00A510AC0EBFFA2EC09F00A2B75
:1059D000000189D7A2EC09F0A2EC09F0F36A00EE0D
:1059E000B9F004010A51F3CFEBFFA2EC09F000017A
:1059F0001200A2EC09F0A2EC09F00401068FA2EC5F
:105A000009F0010166510A6E0A0E0A5C010ED8A463
:105A1000000E376E66510A6E0D0E0A5C010ED8A498
:105A2000000E37120001D8A4A2EF09F0A2EC09F091
:105A30000A0EF76E260EF66E00EEB9F0CFEC02F00D
:105A400009E00A0EF76E2A0EF66E00EEB9F0CFEC02
:105A500002F005E1A2EC09F0D1EF2FF080D20A0E9E
:105A6000F76E320EF66E00EEB9F0CFEC02F005E103
:105A7000A2EC09F04DEF31F072D20A0EF76E380E3B
:105A8000F66E00EEB9F0CFEC02F005E1A2EC09F001
:105A9000B0EF33F064D20A0EF76E3C0EF66E00EEF5
:105AA000B9F0CFEC02F005E1A2EC09F0E4EF46F02A
:105AB00056D20A0EF76E400EF66E00EEB9F0CFEC3D
:105AC00002F005E1A2EC09F09EEF46F048D20A0E82
:105AD000F76E480EF66E00EEB9F0CFEC02F005E17D
:105AE000A2EC09F0A2EF36F03AD20A0EF76E4E0E93
:105AF000F66E00EEB9F0CFEC02F005E1A2EC09F091
:105B000048EF37F02CD20A0EF76E540EF66E00EE08
:105B1000B9F0CFEC02F005E1A2EC09F075EF37F037
:105B20001ED20A0EF76E5C0EF66E00EEB9F0CFECE8
:105B300002F005E1A2EC09F000EF39F010D20A0EF4
:105B4000F76E600EF66E00EEB9F0CFEC02F009E0F1
:105B50000A0EF76E640EF66E00EEB9F0CFEC02F0AE
:105B600005E1A2EC09F001EF38F0F9D10A0EF76E69
:105B70006C0EF66E00EEB9F0CFEC02F009E00A0E02
:105B8000F76E700EF66E00EEB9F0CFEC02F005E1A4
:105B9000A2EC09F0A6EF39F0E2D10A0EF76E780E0A
:105BA000F66E00EEB9F0CFEC02F009E00A0EF76EE7
:105BB0007C0EF66E00EEB9F0CFEC02F005E1A2EC3F
:105BC00009F07BEF34F0CBD10A0EF76E820EF66E41
:105BD00000EEB9F0CFEC02F005E1A2EC09F061EFC4
:105BE00033F0BDD10A0EF76E880EF66E00EEB9F0F6
:105BF000CFEC02F009E00A0EF76E8C0EF66E00EEA6
:105C0000B9F0CFEC02F005E1A2EC09F054EF35F069
:105C1000A6D10A0EF76E940EF66E00EEB9F0CFEC38
:105C200002F009E00A0EF76E980EF66E00EEB9F07B
:105C3000CFEC02F005E1A2EC09F095EF3DF08FD139
:105C40000A0EF76EA00EF66E00EEB9F0CFEC02F081
:105C500005E1A2EC09F033EF3FF081D10A0EF76EB7
:105C6000A60EF66E00EEB9F0CFEC02F005E1A2EC64
:105C700009F090EF4BF073D10A0EF76EAC0EF66E92
:105C800000EEB9F0CFEC02F005E1A2EC09F0BEEFB6
:105C900035F065D10A0EF76EB40EF66E00EEB9F06F
:105CA000CFEC02F005E1A2EC09F0E9EF35F057D1B5
:105CB0000A0EF76EBC0EF66E00EEB9F0CFEC02F0F5
:105CC00005E1A2EC09F0B9EF32F049D10A0EF76E06
:105CD000C20EF66E00EEB9F0CFEC02F004E1A2ECD9
:105CE00009F0FCD13CD10A0EF76EC80EF66E00EE3C
:105CF000B9F0CFEC02F005E1A2EC09F062EF47F059
:105D00002ED10A0EF76ED00EF66E00EEB9F0CFEC83
:105D100002F005E1A2EC09F0CAEF47F020D10A0E2B
:105D2000F76ED60EF66E00EEB9F0CFEC02F009E099
:105D30000A0EF76EDA0EF66E00EEB9F0CFEC02F056
:105D400005E1A2EC09F0A3EF47F009D10A0EF76EC6
:105D5000E20EF66E00EEB9F0CFEC02F005E1A2EC37
:105D600009F08BEF47F0FBD00A0EF76EE80EF66EE7
:105D700000EEB9F0CFEC02F005E1A2EC09F0F1EF92
:105D800047F0EDD00A0EF76EEC0EF66E00EEB9F0AD
:105D9000CFEC02F005E1A2EC09F02FEF48F0DFD0E4
:105DA0000A0EF76EF00EF66E00EEB9F0CFEC02F0D0
:105DB00005E1A2EC09F06EEF48F0D1D00A0EF76EC3
:105DC000F40EF66E00EEB9F0CFEC02F005E1A2ECB5
:105DD00009F0ADEF48F0C3D00A0EF76EF80EF66E7C
:105DE00000EEB9F0CFEC02F005E1A2EC09F0ECEF27
:105DF00048F0B5D00A0EF76EFE0EF66E00EEB9F062
:105E0000CFEC02F005E1A2EC09F0FFEF48F0A7D0DB
:105E10000B0EF76E040EF66E00EEB9F0CFEC02F04A
:105E200005E1A2EC09F012EF49F099D00B0EF76EE4
:105E30000A0EF66E00EEB9F0CFEC02F005E1A2EC2E
:105E400009F025EF49F08BD00B0EF76E100EF66EB1
:105E500000EEB9F0CFEC02F005E1A2EC09F00AEF98
:105E60004AF07DD00B0EF76E160EF66E00EEB9F00E
:105E7000CFEC02F005E1A2EC09F006EF3AF06FD0AA
:105E80000B0EF76E1C0EF66E00EEB9F0CFEC02F0C2
:105E900005E1A2EC09F0F5EF36F061D00B0EF76EDC
:105EA000220EF66E00EEB9F0CFEC02F005E1A2ECA6
:105EB00009F022EF37F053D00B0EF76E280EF66E76
:105EC00000EEB9F0CFEC02F005E1A2EC09F0DCEF56
:105ED0004AF045D00B0EF76E2C0EF66E00EEB9F0C0
:105EE000CFEC02F005E1A2EC09F0C8EF36F037D0B4
:105EF0000B0EF76E320EF66E00EEB9F0CFEC02F03C
:105F000005E1A2EC09F03EEF4BF029D00B0EF76E45
:105F1000380EF66E00EEB9F0CFEC02F005E1A2EC1F
:105F200009F06BEF4BF01BD00B0EF76E3C0EF66ECC
:105F300000EEB9F0CFEC02F005E1A2EC09F0A3EF1E
:105F400037F00DD00B0EF76E420EF66E00EEB9F084
:105F5000CFEC02F004E1A2EC09F095EF35F0A2ECF1
:105F600009F00D0E55EC01F00B0EF76E460EF66EB5
:105F70004DEC01F00D0E55EC01F0630E55EC01F007
:105F80006D0E55EC01F0640E55EC01F03E0E55EC33
:105F900001F0A2EC09F0A2EC09F0AECF0BF4A2EFF5
:105FA00009F0A2EC09F08CEC53F0A2EC09F004012A
:105FB0005B310001D8A070D0A2EC09F0010166515C
:105FC0000A6E450E0A5C0001D8A461D0A2EC09F06B
:105FD00045EC50F0A2EC09F00401265304E13D0E1B
:105FE000255D000108E3A2EC09F0A2EC09F0040130
:105FF000266B3C0E256F0001A2EC09F0A2EC09F023
:1060000025C408F4A2EC09F00401085300010EE1D4
:10601000A2EC09F0A2EC09F00301FE9DA2EC09F04C
:10602000A2EC09F00401059900012FD0A2EC09F0BF
:10603000040105510001E8B80DD0A2EC09F0A2EC72
:1060400009F004010581A2EC09F0A2EC09F0059326
:1060500000010BD0A2EC09F0A2EC09F004010583C9
:10606000A2EC09F0A2EC09F005910001A2EC09F004
:10607000AA6A390EA96E04010851B7EC01F0A2EC2E
:1060800009F0A2EC09F00301FE8D000104D0A2EC9E
:1060900009F0C2EF4FF00DD0A2EC09F0A2EC09F02C
:1060A0000401D8925EB7D8820301D8B2FE8DD8A27F
:1060B000FE9D0001A2EC09F0A2EC09F004017A6B4C
:1060C000A2EC09F0AA6A240EA96E0301FE51B7ECF6
:1060D00001F0A2EC09F000010AEF50F0A2EC09F087
:1060E0008CEC53F0A2EC09F004015B31000142E3B7
:1060F000A2EC09F0010166510A6E450E0A5C00012E
:1061000034E1A2EC09F04EEC4FF0A2EC09F0A2EC65
:1061100009F0010166510A6E0F0E0A140401796F2D
:10612000A2EC09F0AA6A3E0EA96E7951B7EC01F013
:10613000A2EC09F0795300010DE1A2EC09F0A2EC08
:1061400009F00301FE9BA2EC09F0A2EC09F0FD9D11
:1061500000010AD0A2EC09F0A2EC09F00301FE8BC9
:10616000A2EC09F0000148D804D0A2EC09F0C2EF7B
:106170004FF034D0A2EC09F0A2EC09F00401D8925F
:106180005EB7D8820301D8B2FE8BD8A2FE9BA2ECE8
:1061900009F0FE510001E8BA08D0A2EC09F0A2EC27
:1061A00009F00301FD9D000119D0A2EC09F0A2EC59
:1061B00009F03E0EAEEC01F00401796FA2EC09F09B
:1061C0007953000107E1A2EC09F0A2EC09F0050EF9
:1061D0000401796F0001A2EC09F00ED8A2EC09F0DD
:1061E000AA6A240EA96E0301FE51B7EC01F0A2ECDD
:1061F00009F000010AEF50F0A2EC09F0A2EC09F05E
:1062000004010585A2EC09F0A2EC09F0020EAA6EC9
:10621000170EA96EB0EC01F00B6FA2EC09F00D0E99
:106220000B5DD8A4010E376E0B29000ED8A4010E09
:106230003716000106E0A2EC09F0A2EC09F0030118
:10624000FD8D0001A2EC09F0040105510001E8B840
:106250000DD0A2EC09F0A2EC09F004010581A2EC3A
:1062600009F0A2EC09F0059300010BD0A2EC09F0B3
:10627000A2EC09F004010583A2EC09F0A2EC09F0FC
:1062800005910001A2EC09F0A2EC09F004017905E6
:106290007A6FA2EC09F000011200A2EC09F00101F2
:1062A0006B510A6E0D0E0A5C00010FE1A2EC09F0C1
:1062B000A2EC09F00301FD9BA2EC09F0A2EC09F0AD
:1062C000FD9DA2EC09F000013DD1A2EC09F04EECDD
:1062D0004FF0A2EC09F0A2EC09F0010E0401266FC8
:1062E0004C0E256FA2EC09F0010166510A6E310EC9
:1062F0000A5C000132E1A2EC09F0A2EC09F0010E07
:106300000401266F4C0E256FA2EC09F001016751C4
:106310000A6E0D0E0A5C010ED8A4000E376E68518D
:106320000A6E0D0E0A5C010ED8A4000E3712000191
:1063300013E0A2EC09F0010EAA6E4C0EA96E0D0E30
:10634000B7EC01F0A2EC09F0A2EC09F00301FD9B0F
:10635000A2EC09F00001F6D072D0A2EC09F0010124
:1063600066510A6E320E0A5C000132E1A2EC09F0BD
:10637000A2EC09F0020E0401266F170E256FA2ECA5
:1063800009F0010167510A6E0D0E0A5C010ED8A4D6
:10639000000E376E68510A6E0D0E0A5C010ED8A40D
:1063A000000E3712000113E0A2EC09F0020EAA6EF3
:1063B000170EA96E0D0EB7EC01F0A2EC09F0A2ECDD
:1063C00009F00301FD9DA2EC09F00001BBD037D01C
:1063D000A2EC09F0010EAA6E4C0EA96E0D0EB7ECE0
:1063E00001F0A2EC09F0020EAA6E170EA96E0D0EB6
:1063F000B7EC01F0A2EC09F0A2EC09F00301FD9B5F
:10640000A2EC09F0A2EC09F0FD9DA2EC09F0A2ECCF
:1064100009F0FE9DA2EC09F0A2EC09F0040105913F
:10642000A2EC09F00B0EF76E5C0EF66E4DEC01F06F
:106430000D0E55EC01F0A2EC09F0000183D0A2ECA6
:1064400009F00401096BC80E0401095D000135E281
:10645000A2EC09F0A2EC09F00B6A020E0401092576
:106460000A6ED8B00B2A0A50660FE96E010E0B2097
:10647000EA6EEF500B6FA2EC09F00D0E0B5D010EF2
:10648000D8A4000E376E0A0E0B5D010ED8A4000EC4
:106490003712000112E1A2EC09F00401095125258F
:1064A000A96E000E2621AA6E0B51B7EC01F0A2ECEA
:1064B00009F00401092B0001C6E3A2EC09F0040174
:1064C00009512525A96E000E2621AA6E0D0EB7ECE6
:1064D00001F0A2EC09F0010166510A6E310E0A5C6E
:1064E00000010CE1A2EC09F0A2EC09F00301FD8B24
:1064F000A2EC09F0A2EC09F004017A6B0001A2EC15
:1065000009F0010166510A6E320E0A5C00010DE1CC
:10651000A2EC09F0A2EC09F00301FD8DA2EC09F058
:10652000A2EC09F0040179057A6F0001A2EC09F0F0
:10653000A2EC09F00301FE8DA2EC09F0A2EC09F037
:10654000040105810001A2EC09F0AA6A230EA96EDC
:106550000301FD51B7EC01F0A2EC09F0AA6A240E88
:10656000A96EFE51B7EC01F0A2EC09F000010AEFB0
:1065700050F0A2EC09F001016B510A6E0D0E0A5C9D
:106580000001D8B4A2EF09F0A2EC09F04EEC4FF0F4
:10659000A2EC09F0A2EC09F00401266BAA0E256F0B
:1065A000A2EC09F0010166510A6E0D0E0A5C0001B1
:1065B0001CE1A2EC09F026C4AAFF25C4A9FF0D0E18
:1065C000B7EC01F0A2EC09F0A2EC09F00301FD9F89
:1065D000A2EC09F0A2EC09F0FE9BA2EC09F0A2ECFF
:1065E00009F004010595000155D0A2EC09F0040161
:1065F000096B640E0401095D00012FE2A2EC09F0B1
:10660000A2EC09F001EE66F004010951E926000E42
:10661000EA22EF500B6FA2EC09F00D0E0B5D010E9C
:10662000D8A4000E376E0A0E0B5D010ED8A4000E22
:106630003712000112E1A2EC09F0040109512525ED
:10664000A96E000E2621AA6E0B51B7EC01F0A2EC48
:1066500009F00401092B0001CCE3A2EC09F00401CC
:1066600009512525A96E000E2621AA6E0D0EB7EC44
:1066700001F0A2EC09F0A2EC09F00301FD8FA2ECFD
:1066800009F0A2EC09F0FE8BA2EC09F0A2EC09F0F3
:10669000040105850001A2EC09F0AA6A230EA96E87
:1066A0000301FD51B7EC01F0A2EC09F0AA6A240E37
:1066B000A96EFE51B7EC01F0A2EC09F000010AEF5F
:1066C00050F0A2EC09F04EEC4FF0A2EC09F0A2EC75
:1066D00009F0260EAEEC01F00401006FA2EC09F007
:1066E000A2EC09F0010166510A6EDF0E0A140401E2
:1066F0000C6FA2EC09F0460E0C5D000108E1A2EC63
:1067000009F0A2EC09F00401008300011BD0A2EC07
:1067100009F0430E04010C5D000108E1A2EC09F050
:10672000A2EC09F00401009300010CD0A2EC09F0E6
:10673000A2EC09F0430E04010C6FA2EC09F0000179
:10674000C2EF4FF0A2EC09F0AA6A260EA96E04016E
:106750000051B7EC01F0A2EC09F000010AEF50F093
:10676000A2EC09F0040105350001D8B00AEF50F0A1
:10677000A2EC09F00D0E55EC01F00B0EF76E700E49
:10678000F66E4DEC01F00D0E55EC01F00B0EF76EB0
:106790007E0EF66E4DEC01F00D0E55EC01F0A2EC04
:1067A00009F00B0EF76EA20EF66E4DEC01F00D0E19
:1067B00055EC01F0A2EC09F0030E136EE80EEFECBD
:1067C00001F0A2EC09F094908B80A2EC09F0A2EC0D
:1067D00009F004010499A2EC09F000019EA2FDD782
:1067E000A2EC09F0A2EC09F0040104B9818C04A91F
:1067F000819CA2EC09F0A2EC09F09E92A2EC09F0B7
:10680000A2EC09F07DC4BBFFA2EC09F0A2EC09F0F8
:106810000489A2EC09F000019EA2FDD7A2EC09F0C8
:10682000A2EC09F0040104B9818C04A9819CA2ECBA
:1068300009F0A2EC09F09E92A2EC09F0A2EC09F09A
:106840007DC4BBFFA2EC09F0056A010E026E27ECC5
:1068500001F00001BAE304010B6FA2EC09F0A2EC15
:1068600009F00B9BA2EC09F0440E0B5D000111E155
:10687000A2EC09F0AA0E04017D5D000106E2A2EC83
:1068800009F0A2EC09F004017D2B0001A2EC09F053
:106890009CD7A2EC09F0550E04010B5D000111E13B
:1068A000A2EC09F0470E04017D5D000106E3A2ECB5
:1068B00009F0A2EC09F004017D070001A2EC09F047
:1068C00084D7A2EC09F0450E04010B5D0001D8A4A9
:1068D0007CD7A2EC09F094908B90A2EC09F0AA6A04
:1068E0003F0EA96E04017D51B7EC01F0A2EC09F056
:1068F00000010AEF50F0A2EC09F04EEC4FF0A2ECD0
:1069000009F06BEC2CF0A2EC09F0A2EC09F0250EDA
:10691000AEEC01F00301FF6FA2EC09F0010166513A
:106920000A6E4F0E0A5C010ED8A4000E376E675136
:106930000A6E460E0A5C010ED8A4000E371600013E
:106940000DE0A2EC09F0A2EC09F00301FF97A2EC24
:1069500009F0A2EC09F0FF99000198D0A2EC09F02F
:10696000010166510A6E580E0A5C010ED8A4000E91
:10697000376E67510A6E4D0E0A5C010ED8A4000EE8
:10698000371668510A6E490E0A5C010ED8A4000E33
:10699000371669510A6E540E0A5C010ED8A4000E17
:1069A000371600010DE0A2EC09F0A2EC09F003019A
:1069B000FF87A2EC09F0A2EC09F0FF99000166D074
:1069C000A2EC09F0010166510A6E520E0A5C010E3A
:1069D000D8A4000E376E67510A6E430E0A5C010E92
:1069E000D8A4000E371668510A6E560E0A5C010EC6
:1069F000D8A4000E371600010DE0A2EC09F0A2ECBD
:106A000009F00301FF97A2EC09F0A2EC09F0FF895D
:106A100000013CD0A2EC09F00401053500011BE2A5
:106A2000A2EC09F00D0E55EC01F00B0EF76EC40E42
:106A3000F66E4DEC01F00D0E55EC01F0630E55ECC9
:106A400001F06D0E55EC01F0640E55EC01F03E0EB8
:106A500055EC01F019D0A2EC09F0A2EC09F001EE1E
:106A600066F00D0EEE6E0B0EF76EC40EF66EB5EC04
:106A700002F00D0EEE6E630EEE6E6D0EEE6E640E97
:106A8000EE6E3E0EEE6EEE6AA2EF09F0A2EC09F099
:106A9000AA6A250EA96E0301FF51B7EC01F0A2EC22
:106AA00009F000010AEF50F0A2EC09F045EC50F0BB
:106AB000A2EC09F00401265304E1650E255D0001F6
:106AC00008E3A2EC09F0A2EC09F00401266B640EC5
:106AD000256F0001A2EC09F0A2EC09F00401255198
:106AE000800DF3CF20F0F4CF21F02651800DF3502C
:106AF000212625512126800E2024256F000E2120DD
:106B0000266FA2EC09F0A2EC09F026C4FCF3A2EC7B
:106B100009F0AA6A380EA96E0301FC51B7EC01F026
:106B2000A2EC09F000010AEF50F0A2EC09F045ECEC
:106B300050F0A2EC09F00401265304E1100E255D8B
:106B4000000107E3A2EC09F0A2EC09F00401266BB6
:106B5000256B0001A2EC09F0A2EC09F025C482F437
:106B6000A2EC09F0AA6A9A0EA96E04018251B7EC50
:106B700001F0A2EC09F000010AEF50F0A2EC09F0DC
:106B800044D8A2EC09F00A0E04010B5D00010BE2EF
:106B9000A2EC09F0AA6A3B0EA96E04010B51B7ECF6
:106BA00001F0000104D0A2EC09F0C2EF4FF0A2EC1A
:106BB00009F00D0E55EC01F00B0EF76EDA0EF66EC5
:106BC0004DEC01F00D0E55EC01F0A2EC09F00AEFCE
:106BD00050F0A2EC09F019D8A2EC09F00A0E040159
:106BE0000B5D00010BE2A2EC09F0AA6A3A0EA96E55
:106BF00004010B51B7EC01F0000104D0A2EC09F044
:106C0000C2EF4FF0A2EC09F0D2D7A2EC09F045ECAC
:106C100050F0A2EC09F004012551300A26110001C0
:106C200008E004012651120AC00ED8B4251900014B
:106C300008E1A2EC09F0A2EC09F004010B6B0001E1
:106C40007FD004012551600A2611000108E00401EB
:106C50002651250A800ED8B42519000109E1A2ECBD
:106C600009F0A2EC09F0010E04010B6F000168D0DD
:106C700004012551C00A2611000106E00401265135
:106C80004B0A2511000109E1A2EC09F0A2EC09F080
:106C9000020E04010B6F000153D004012651010ABA
:106CA000800ED8B42519000106E004012651960A89
:106CB0002511000109E1A2EC09F0A2EC09F0030E94
:106CC00004010B6F00013CD004012651020A400E62
:106CD000D8B42519000106E004012651E10A251166
:106CE000000109E1A2EC09F0A2EC09F0040E040194
:106CF0000B6F000125D004012551730A26110001F4
:106D00000EE004012651040A800ED8B425190001B2
:106D100006E0040126512D0A2511000109E1A2EC2B
:106D200009F0A2EC09F0050E04010B6F000107D079
:106D3000A2EC09F0A2EC09F00A0E04010B6F0001AD
:106D4000A2EF09F0A2EC09F08CEC53F0A2EC09F0F0
:106D500004015B310001D8B0C2EF4FF0A2EC09F0A2
:106D6000A2EC09F00401D8925EB7D8820301D8B230
:106D7000FE89D8A2FE99A2EC09F0AA6A240EA96E97
:106D8000FE51B7EC01F0A2EC09F000010AEF50F05F
:106D9000A2EC09F08CEC53F0A2EC09F004015B3199
:106DA0000001D8B0C2EF4FF0A2EC09F0A2EC09F05C
:106DB000260EAEEC01F00401006FA2EC09F0A2EC8B
:106DC00009F0D8925EB7D882D8B20081D8A20091DB
:106DD000A2EC09F0AA6A260EA96E0051B7EC01F0E8
:106DE000A2EC09F000010AEF50F0A2EC09F08CECE3
:106DF00053F0A2EC09F004015B310001D8B0C2EFFE
:106E00004FF0A2EC09F0A2EC09F0260EAEEC01F076
:106E10000401006FA2EC09F0A2EC09F0D8925EB771
:106E2000D882D8B20089D8A20099A2EC09F0AA6A47
:106E3000260EA96E0051B7EC01F0A2EC09F000019A
:106E40000AEF50F0A2EC09F08CEC53F0A2EC09F040
:106E500004015B310001D8B0C2EF4FF0A2EC09F0A1
:106E6000A2EC09F00401D8925EB7D8820301D8B22F
:106E7000FE8FD8A2FE9FA2EC09F0AA6A240EA96E8A
:106E8000FE51B7EC01F0A2EC09F000010AEF50F05E
:106E9000A2EC09F08CEC53F0A2EC09F004015B3198
:106EA0000001D8B0C2EF4FF0A2EC09F0A2EC09F05B
:106EB000260EAEEC01F00401006FA2EC09F0A2EC8A
:106EC00009F0D8925EB7D882D8B20087D8A20097CE
:106ED000A2EC09F0AA6A260EA96E0051B7EC01F0E7
:106EE000A2EC09F000010AEF50F0A2EC09F08CECE2
:106EF00053F0A2EC09F004015B310001D8B0C2EFFD
:106F00004FF0A2EC09F0A2EC09F0260EAEEC01F075
:106F10000401006FA2EC09F0A2EC09F0E86A5EB788
:106F2000010E010AD8B40095D8A40085A2EC09F09E
:106F3000AA6A260EA96E0051B7EC01F0A2EC09F086
:106F400000010AEF50F0A2EC09F08CEC53F0A2EC37
:106F500009F004015B310001D8B0C2EF4FF0A2ECA0
:106F600009F0A2EC09F0250EAEEC01F00301FF6F71
:106F7000A2EC09F0A2EC09F0260EAEEC01F004013F
:106F8000006FA2EC09F0A2EC09F0D8925EB7D882AB
:106F9000D8B20283D8A20293A2EC09F002510001F8
:106FA000E8A220D0A2EC09F0A2EC09F00301FF91C5
:106FB000A2EC09F0A2EC09F0FF93A2EC09F0A2EC1C
:106FC00009F0FF95A2EC09F0A2EC09F0FF97A2EC02
:106FD00009F0A2EC09F0FF99A2EC09F0A2EC09F08B
:106FE000040100950001A2EC09F0AA6A990EA96EAD
:106FF00004010251B7EC01F0A2EC09F000010AEF24
:1070000050F0A2EC09F04EEC4FF0A2EC09F06BEC62
:107010002CF0A2EC09F0A2EC09F0250EAEEC01F088
:107020000301FF6FA2EC09F00B0EF76EF40EF66E83
:1070300000EEB9F0CFEC02F0000112E1A2EC09F091
:10704000A2EC09F00301FF81A2EC09F0A2EC09F027
:10705000FF83A2EC09F0A2EC09F0FF950001C2D079
:107060000B0EF76EF80EF66E00EEB9F0CFEC02F0F4
:107070000DE1A2EC09F0A2EC09F00301FF81A2EC02
:1070800009F0A2EC09F0FF930001ACD00B0EF76EF3
:10709000FE0EF66E00EEB9F0CFEC02F012E1A2ECBB
:1070A00009F0A2EC09F00301FF91A2EC09F0A2ECB7
:1070B00009F0FF93A2EC09F0A2EC09F0FF950001A2
:1070C00091D00C0EF76E020EF66E00EEB9F0CFEC1A
:1070D00002F00DE1A2EC09F0A2EC09F00301FF912E
:1070E000A2EC09F0A2EC09F0FF8300017BD00C0EAA
:1070F000F76E060EF66E00EEB9F0CFEC02F01CE172
:10710000A2EC09F0000E0301FFB1010E376E000E74
:10711000FFB3010E3716000106E0A2EC09F0A2EC65
:1071200009F00301FF910001A2EC09F0A2EC09F0C3
:107130000301FF85000156D00C0EF76E0A0EF66EA5
:1071400000EEB9F0CFEC02F009E00C0EF76E0E0E77
:10715000F66E00EEB9F0CFEC02F008E1A2EC09F017
:10716000A2EC09F00301FF9500013CD0A2EC09F06C
:107170000401053500011BE2A2EC09F00D0E55ECEF
:1071800001F00C0EF76E140EF66E4DEC01F00D0EC4
:1071900055EC01F0630E55EC01F06D0E55EC01F06D
:1071A000640E55EC01F03E0E55EC01F019D0A2EC46
:1071B00009F0A2EC09F001EE66F00D0EEE6E0C0E79
:1071C000F76E140EF66EB5EC02F00D0EEE6E630E59
:1071D000EE6E6D0EEE6E640EEE6E3E0EEE6EEE6AAE
:1071E000A2EF09F0A2EC09F0AA6A250EA96E03012C
:1071F000FF51B7EC01F0A2EC09F000010AEF50F0EA
:10720000A2EC09F0470E55EC01F0500E55EC01F0E0
:10721000530E55EC01F00D0E55EC01F0A2EC09F007
:107220004EEC4FF0A2EC09F06BEC2CF0A2EC09F064
:10723000A2EC09F0250EAEEC01F00301FF6FA2EC09
:1072400009F0010166510A6E240E0A5C0001D8A4FF
:107250006BD0A2EC09F0010169510A6E520E0A5C72
:10726000000112E1A2EC09F0A2EC09F00301FF8B8E
:10727000A2EC09F0A2EC09F0FF9FA2EC09F0A2EC4D
:1072800009F0FF9D00014FD0A2EC09F00101665109
:107290000A6E240E0A5C010ED8A4000E376E6951E6
:1072A0000A6E470E0A5C010ED8A4000E37160001C4
:1072B0003AE0A2EC09F001016A510A6E470E0A5C3D
:1072C000000112E1A2EC09F0A2EC09F00301FF8F2A
:1072D000A2EC09F0A2EC09F0FF9DA2EC09F0A2ECEF
:1072E00009F0FF9B00011FD0A2EC09F001016A51D7
:1072F0000A6E4C0E0A5C000112E1A2EC09F0A2EC4D
:1073000009F00301FF8DA2EC09F0A2EC09F0FF9F48
:10731000A2EC09F0A2EC09F0FF9B000104D0A2EC62
:1073200009F0C2EF4FF004D0A2EC09F0C2EF4FF029
:10733000A2EC09F0AA6A250EA96E0301FF51B7EC71
:1073400001F0A2EC09F000010AEF50F0A2EC09F004
:107350004EEC4FF0A2EC09F004015D3100010EE3A8
:10736000A2EC09F0A2EC09F000EEB9F0EE6AEE6AC8
:10737000EE6AEE6AEE6AEE6AEE6A04D0A2EC09F0FA
:107380005AEC4DF0A2EC09F00401096B070E040160
:10739000095D000120E2A2EC09F0A2EC09F000EE88
:1073A000B9F004010951EBCF0AF000EE4DF009519C
:1073B0000AC0EBFFA2EC09F0AA6A09C4A9FF00EE1B
:1073C000B9F00951EB50B7EC01F0A2EC09F004015F
:1073D000092B0001DBE3A2EC09F0A2EC09F0E86A5A
:1073E00004015DB1010E010A0301D8B4FD91D8A4D6
:1073F000FD81A2EC09F0AA6A230EA96EFD51B7EC3B
:1074000001F0A2EC09F000010AEF50F0A2EC09F043
:107410004EEC4FF0A2EC09F0A2EC09F001EE66F0A0
:10742000BDEC02F0A2EC09F0A2EC09F0260EAEECE5
:1074300001F00401006FA2EC09F011EE66F0030EFA
:1074400004EE8DF0E6CFEEFFE82EFCD7EE6A0C0ED0
:10745000F76E360EF66E04EE8DF0CFEC02F0000102
:10746000D8A444D2A2EC09F0010169510A6E410E80
:107470000A5C000135E1A2EC09F0A2EC09F004017C
:107480000191A2EC09F0A2EC09F00193A2EC09F041
:10749000A2EC09F00195A2EC09F0A2EC09F0019729
:1074A000A2EC09F0A2EC09F00199A2EC09F0A2EC1F
:1074B00009F0019BA2EC09F0A2EC09F0019DA2ECFD
:1074C00009F0A2EC09F0019FA2EC09F0A2EC09F08E
:1074D000009DA2EC09F0A2EC09F0009F000105D28A
:1074E000A2EC09F0010169510A6E310E0A5C010E2D
:1074F000D8A4000E376E6A510A6E300E0A5C010E77
:10750000D8A4000E3716000109E0A2EC09F0A2ECA5
:1075100009F0090E04010B6F00010ED0A2EC09F076
:10752000A2EC09F0010169510A6E0F0E0A14040160
:107530000B6FA2EC09F00B070001A2EC09F00401AB
:107540000B53000108E1A2EC09F0A2EC09F00401E0
:107550000191000174D0010E04010B5D000108E1EE
:10756000A2EC09F0A2EC09F004010193000167D03C
:10757000020E04010B5D000108E1A2EC09F0A2EC8F
:1075800009F00401019500015AD0030E04010B5DBE
:10759000000108E1A2EC09F0A2EC09F00401019756
:1075A00000014DD0040E04010B5D000108E1A2ECC6
:1075B00009F0A2EC09F004010199000140D0050E88
:1075C00004010B5D000108E1A2EC09F0A2EC09F056
:1075D0000401019B000133D0060E04010B5D000184
:1075E00008E1A2EC09F0A2EC09F00401019D000100
:1075F00026D0070E04010B5D000108E1A2EC09F0A2
:10760000A2EC09F00401019F000119D0080E040149
:107610000B5D000108E1A2EC09F0A2EC09F0040105
:10762000009D00010CD0090E04010B5D000106E174
:10763000A2EC09F0A2EC09F00401009F0001A2EC09
:1076400009F0010E040101B1000E376E000E01B306
:10765000010E3716000118E0A2EC09F0A2EC09F0C7
:107660000401266B5A0E256FA2EC09F00001C3EC51
:1076700054F0A2EC09F0A2EC09F004010181A2ECA3
:1076800009F0A2EC09F001930001A2EC09F0010E4F
:10769000040101B3000E376E000E01B5010E37165E
:1076A000000118E0A2EC09F0A2EC09F00401266B3D
:1076B000610E256FA2EC09F00001C3EC54F0A2ECBE
:1076C00009F0A2EC09F004010183A2EC09F0A2EC9C
:1076D00009F001950001A2EC09F0010E040101B5C9
:1076E000000E376E000E01B7010E3716000118E0CC
:1076F000A2EC09F0A2EC09F00401266B680E256FDC
:10770000A2EC09F00001C3EC54F0A2EC09F0A2ECE9
:1077100009F004010185A2EC09F0A2EC09F001973F
:107720000001A2EC09F0010E040101B7000E376E52
:10773000000E01B9010E3716000118E0A2EC09F0A5
:10774000A2EC09F00401266B6F0E256FA2EC09F084
:107750000001C3EC54F0A2EC09F0A2EC09F0040122
:107760000187A2EC09F0A2EC09F001990001A2EC5A
:1077700009F0010E040101B9000E376E000E01BBC5
:10778000010E3716000118E0A2EC09F0A2EC09F096
:107790000401266B760E256FA2EC09F00001C3EC04
:1077A00054F0A2EC09F0A2EC09F004010189A2EC6A
:1077B00009F0A2EC09F0019B0001A2EC09F0010E16
:1077C000040101BB000E376E000E01BD010E37161D
:1077D000000118E0A2EC09F0A2EC09F00401266B0C
:1077E0007D0E256FA2EC09F00001C3EC54F0A2EC71
:1077F00009F0A2EC09F00401018BA2EC09F0A2EC63
:1078000009F0019D0001A2EC09F0010E040101BD87
:10781000000E376E000E01BF010E3716000118E092
:10782000A2EC09F0A2EC09F00401266B840E256F8E
:10783000A2EC09F00001C3EC54F0A2EC09F0A2ECB8
:1078400009F00401018DA2EC09F0A2EC09F0019FFE
:107850000001A2EC09F0010E040101BF000E376E19
:10786000000E00BD010E3716000118E0A2EC09F071
:10787000A2EC09F00401266B8B0E256FA2EC09F037
:107880000001C3EC54F0A2EC09F0A2EC09F00401F1
:10789000018FA2EC09F0A2EC09F0009D0001A2EC1E
:1078A00009F0010E040100BD000E376E000E00BF8E
:1078B000010E3716000118E0A2EC09F0A2EC09F065
:1078C0000401266B920E256FA2EC09F00001C3ECB7
:1078D00054F0A2EC09F0A2EC09F00401008DA2EC36
:1078E00009F0A2EC09F0009F000109D1A2EC09F017
:1078F0005AEC4DF0A2EC09F00401013100010FE255
:10790000A2EC09F0A2EC09F00401266B530E256FDE
:10791000A2EC09F0A2EC09F001810001D2D0A2ECA6
:1079200009F0040101510001E8B20FD0A2EC09F006
:10793000A2EC09F00401266B5A0E256FA2EC09F0A7
:10794000A2EC09F001830001BCD0A2EC09F0040113
:1079500001510001E8B40FD0A2EC09F0A2EC09F04B
:107960000401266B610E256FA2EC09F0A2EC09F070
:1079700001850001A6D0A2EC09F00401015100012B
:10798000E8B60FD0A2EC09F0A2EC09F00401266BD6
:10799000680E256FA2EC09F0A2EC09F00187000146
:1079A00090D0A2EC09F0040101510001E8B80FD019
:1079B000A2EC09F0A2EC09F00401266B6F0E256F12
:1079C000A2EC09F0A2EC09F0018900017AD0A2EC46
:1079D00009F0040101510001E8BA0FD0A2EC09F04E
:1079E000A2EC09F00401266B760E256FA2EC09F0DB
:1079F000A2EC09F0018B000164D0A2EC09F00401B3
:107A000001510001E8BC0FD0A2EC09F0A2EC09F092
:107A10000401266B7D0E256FA2EC09F0A2EC09F0A3
:107A2000018D00014ED0A2EC09F0040101350001E6
:107A30000FE2A2EC09F0A2EC09F00401266B840E1F
:107A4000256FA2EC09F0A2EC09F0018F000139D0FA
:107A5000A2EC09F0040100510001E8BC0FD0A2EC37
:107A600009F0A2EC09F00401266B8B0E256FA2EC45
:107A700009F0A2EC09F0008D000123D0A2EC09F07E
:107A80000401003500010FE2A2EC09F0A2EC09F0BC
:107A90000401266B920E256FA2EC09F0A2EC09F00E
:107AA000008F00010ED0A2EC09F00D0E55EC01F094
:107AB0000C0EF76E3A0EF66E4DEC01F00D0E55EC15
:107AC00001F0A2EC09F00401096B070E0401095D45
:107AD000000115E2A2EC09F0040109512525A96E67
:107AE000000E2621AA6E00EEB9F00951EB50B7EC5A
:107AF00001F0A2EC09F00401092B0001E6E3A2EC7D
:107B000009F0AA6A270EA96E04010151B7EC01F031
:107B1000A2EC09F0AA6A260EA96E0051B7EC01F09A
:107B2000A2EC09F000010AEF50F0A2EC09F0A2EC7F
:107B300009F00301FD93A2EC09F0A2EC09F0FD9518
:107B4000A2EC09F0A2EC09F0FD97A2EC09F0A2EC7E
:107B500009F0FD99A2EC09F000014EEC4FF0A2EC07
:107B600009F004015D3100010EE3A2EC09F0A2EC82
:107B700009F000EEB9F0EE6AEE6AEE6AEE6AEE6ABD
:107B8000EE6AEE6A04D0A2EC09F05AEC4DF0A2ECD9
:107B900009F004015D310001D8B0C2EF4FF0A2EC52
:107BA00009F00401096B070E0401095D000123E2DD
:107BB000A2EC09F0A2EC09F000EEB9F004010951C1
:107BC000EBCF0AF000EE56F009510AC0EBFFA2EC31
:107BD00009F0AA6A070E0925A96ED8B0AA2A00EEF4
:107BE000B9F00951EB50B7EC01F0A2EC09F0040137
:107BF000092B0001D8E3A2EC09F0A2EC09F0030183
:107C0000FD83A2EC09F0040104310001D8B002D1D7
:107C1000A2EC09F05AEC4DF0A2EC09F004015D3140
:107C20000001D8B0C2EF4FF0A2EC09F0040104311A
:107C3000000140E2A2EC09F00401096B070E040107
:107C4000095D000123E2A2EC09F0A2EC09F000EECC
:107C5000B9F004010951EBCF0AF000EE5FF00951D1
:107C60000AC0EBFFA2EC09F0AA6A0E0E0925A96E64
:107C7000D8B0AA2A00EEB9F00951EB50B7EC01F0E8
:107C8000A2EC09F00401092B0001D8E3A2EC09F0F1
:107C9000A2EC09F00301FD85A2EC09F000015AEC09
:107CA0004DF0A2EC09F004015D310001D8B0C2EF43
:107CB0004FF01BD0A2EC09F00401096B070E040180
:107CC000095D000112E2A2EC09F0AA6A0E0E04019D
:107CD0000925A96ED8B0AA2A000EB7EC01F0A2ECD3
:107CE00009F00401092B0001E9E3A2EC09F0040109
:107CF0000431000140E2A2EC09F00401096B070E17
:107D00000401095D000123E2A2EC09F0A2EC09F0F4
:107D100000EEB9F004010951EBCF0AF000EE68F073
:107D200009510AC0EBFFA2EC09F0AA6A150E092559
:107D3000A96ED8B0AA2A00EEB9F00951EB50B7EC01
:107D400001F0A2EC09F00401092B0001D8E3A2EC38
:107D500009F0A2EC09F00301FD87A2EC09F0000193
:107D60005AEC4DF0A2EC09F004015D310001D8B0ED
:107D7000C2EF4FF01BD0A2EC09F00401096B070E13
:107D80000401095D000112E2A2EC09F0AA6A150ED5
:107D900004010925A96ED8B0AA2A000EB7EC01F09B
:107DA000A2EC09F00401092B0001E9E3A2EC09F0BF
:107DB0000401096B070E0401095D000123E2A2EC36
:107DC00009F0A2EC09F000EEB9F004010951EBCF83
:107DD0000AF000EE71F009510AC0EBFFA2EC09F0C5
:107DE000AA6A1C0E0925A96ED8B0AA2A00EEB9F01D
:107DF0000951EB50B7EC01F0A2EC09F00401092B9A
:107E00000001D8E3A2EC09F0A2EC09F00301FD891E
:107E100000011BD0A2EC09F00401096B070E04015C
:107E2000095D000112E2A2EC09F0AA6A1C0E04012D
:107E30000925A96ED8B0AA2A000EB7EC01F0A2EC71
:107E400009F00401092B0001E9E3A2EC09F0AA6A98
:107E5000230EA96E0301FD51B7EC01F0A2EC09F06D
:107E600000010AEF50F0A2EC09F004010535000111
:107E7000D8B00AEF50F0A2EC09F00D0E55EC01F06D
:107E80000C0EF76E580EF66E4DEC01F0040E016EFE
:107E9000046A42C417F041C416F069EC00F03A0ECF
:107EA00055EC01F0020E046E0401895167EC00F0FC
:107EB000200E55EC01F0680E55EC01F03A0E55EC31
:107EC00001F06D0E55EC01F0A2EC09F00D0E55EC31
:107ED00001F00C0EF76E6C0EF66E4DEC01F0A2EC9C
:107EE00009F000510001E8A409D0A2EC09F04F0EFE
:107EF00055EC01F04E0E55EC01F00AD0A2EC09F061
:107F00004F0E55EC01F0460E55EC01F055EC01F02A
:107F1000A2EC09F00D0E55EC01F0450E55EC01F008
:107F2000430E55EC01F0480E55EC01F04F0E55ECA8
:107F300001F0200E55EC01F0A2EC09F00401005113
:107F40000001E8A609D0A2EC09F04F0E55EC01F0B3
:107F50004E0E55EC01F00AD0A2EC09F04F0E55EC94
:107F600001F0460E55EC01F055EC01F0A2EC09F0E1
:107F70000D0E55EC01F00C0EF76E740EF66E4DEC16
:107F800001F0A2EC09F0040100510001E8B206D0B2
:107F9000A2EC09F0430E55EC01F005D0A2EC09F07B
:107FA000460E55EC01F0A2EC09F00D0E55EC01F077
:107FB0000C0EF76E820EF66E4DEC01F0040E016EA3
:107FC0000401835166EC00F0A2EC09F0A2EC09F088
:107FD0000301FC51AB0DF3CF25F4F4CF26F4A2EC52
:107FE00009F00D0E55EC01F00C0EF76E900EF66ECA
:107FF0004DEC01F0040E016E0401265166EC00F018
:10800000A2EC09F00D0E55EC01F00C0EF76E9A0E75
:10801000F66E4DEC01F0040E016E855166EC00F039
:10802000A2EC09F00D0E55EC01F0470E55EC01F0F5
:10803000500E55EC01F0530E55EC01F0200E55ECAE
:1080400001F0A2EC09F00301FF510001E8AA08D0F9
:10805000A2EC09F00C0EF76EA20EF66E4DEC01F0DC
:10806000A2EC09F00301FF35000108E3A2EC09F0DE
:108070000C0EF76EAA0EF66E4DEC01F0A2EC09F0B4
:108080000301FF510001E8AC08D0A2EC09F00C0E8E
:10809000F76EB20EF66E4DEC01F0A2EC09F00D0E8B
:1080A00055EC01F00C0EF76EBA0EF66E4DEC01F0C9
:1080B000A2EC09F00301FF510001E8A60FD0A2ECE9
:1080C00009F0580E55EC01F04D0E55EC01F0490E3B
:1080D00055EC01F0540E55EC01F01DD0A2EC09F066
:1080E0000301FF510001E8A80CD0A2EC09F0520EE8
:1080F00055EC01F0430E55EC01F0560E55EC01F035
:108100000AD0A2EC09F04F0E55EC01F0460E55ECEA
:1081100001F055EC01F0A2EC09F00D0E55EC01F068
:108120000C0EF76EC20EF66E4DEC01F0A2EC09F0EB
:10813000000E0301FFB1010E376E000EFFB3010EFA
:10814000371600010BE0A2EC09F0410E55EC01F0EE
:108150004C0E55EC01F055EC01F050D0A2EC09F0BA
:108160000301FF3100011EE3A2EC09F0580E55ECAB
:1081700001F04D0E55EC01F0490E55EC01F0540E96
:1081800055EC01F0A2EC09F00301FF510001E8A455
:1081900008D0A2EC09F00C0EF76ECC0EF66E4DEC8A
:1081A00001F02CD0A2EC09F00301FF510001E8A27C
:1081B0001BD0A2EC09F0520E55EC01F0430E55EC29
:1081C00001F0560E55EC01F0A2EC09F00301FF514D
:1081D0000001E8A408D0A2EC09F00C0EF76ECC0E5A
:1081E000F66E4DEC01F00AD0A2EC09F04F0E55EC02
:1081F00001F0460E55EC01F055EC01F0A2EC09F04F
:108200000D0E55EC01F00C0EF76ED60EF66E4DEC21
:1082100001F0A2EC09F00301FE510001E8A809D029
:10822000A2EC09F04F0E55EC01F04E0E55EC01F0AA
:108230000AD0A2EC09F04F0E55EC01F0460E55ECB9
:1082400001F055EC01F0A2EC09F00D0E55EC01F037
:108250000C0EF76EE00EF66E4DEC01F0A2EC09F09C
:1082600004010031000109E3A2EC09F04F0E55ECC6
:1082700001F04E0E55EC01F00AD0A2EC09F04F0EC1
:1082800055EC01F0460E55EC01F055EC01F0A2EC76
:1082900009F00D0E55EC01F00C0EF76EEE0EF66EB9
:1082A0004DEC01F0A2EC09F0040100510001E8A836
:1082B00009D0A2EC09F04F0E55EC01F04E0E55EC32
:1082C00001F00AD0A2EC09F04F0E55EC01F0460E79
:1082D00055EC01F055EC01F0A2EC09F00D0E55EC57
:1082E00001F00C0EF76EF80EF66E4DEC01F0A2ECFC
:1082F00009F0040100510001E8AA09D0A2EC09F03C
:108300004F0E55EC01F04E0E55EC01F00AD0A2ECE8
:1083100009F04F0E55EC01F0460E55EC01F055EC0E
:1083200001F0A2EC09F00D0E55EC01F00D0EF76E08
:10833000000EF66E4DEC01F0A2EC09F00301FE35E3
:10834000000109E3A2EC09F04F0E55EC01F04E0ECE
:1083500055EC01F00AD0A2EC09F04F0E55EC01F0FB
:10836000460E55EC01F055EC01F0A2EC09F00D0EB3
:1083700055EC01F00D0EF76E080EF66E4DEC01F0A7
:10838000A2EC09F004010231000109E3A2EC09F0BA
:108390004F0E55EC01F04E0E55EC01F00AD0A2EC58
:1083A00009F04F0E55EC01F0460E55EC01F055EC7E
:1083B00001F0A2EC09F00D0E55EC01F00D0EF76E78
:1083C000120EF66E4DEC01F0A2EC09F00301FE5125
:1083D0000001E8AC10D0A2EC09F00D0EF76E1A0EF9
:1083E000F66E4DEC01F0040E016E0401085166ECCE
:1083F00000F000010AD0A2EC09F04F0E55EC01F09C
:10840000460E55EC01F055EC01F0A2EC09F00D0E12
:1084100055EC01F0540E55EC01F0410E55EC01F015
:10842000490E55EC01F04C0E55EC01F0200E55ECC8
:1084300001F0A2EC09F00301FE510001E8AA10D0FE
:10844000A2EC09F00D0EF76E1A0EF66E4DEC01F06F
:10845000040E016E0401795166EC00F000010AD0AF
:10846000A2EC09F04F0E55EC01F0460E55EC01F070
:1084700055EC01F0A2EC09F00D0E55EC01F00D0EDB
:10848000F76E220EF66E4DEC01F004017B5155ECB7
:1084900001F07C5155EC01F0A2EC09F00D0E55EC09
:1084A00001F00D0EF76E2A0EF66E4DEC01F0040E83
:1084B000016E865166EC00F0A2EC09F00D0E55EC51
:1084C00001F00D0EF76E340EF66E4DEC01F0A2ECDD
:1084D00009F002510001E8A209D0A2EC09F04F0E08
:1084E00055EC01F04E0E55EC01F00AD0A2EC09F06B
:1084F0004F0E55EC01F0460E55EC01F055EC01F035
:10850000A2EC09F00D0E55EC01F00D0EF76E3C0ECD
:10851000F66E4DEC01F0040E016E0401825166EC22
:1085200000F0A2EC09F00D0E55EC01F00D0EF76E07
:108530004A0EF66E4DEC01F0A2EC09F0A2EC09F047
:108540003B0EAEEC01F00B6FA2EC09F000011BEC4E
:1085500046F0A2EC09F00D0E55EC01F00D0EF76E91
:10856000520EF66E4DEC01F0A2EC09F0A2EC09F00F
:108570003A0EAEEC01F004010B6FA2EC09F0000121
:108580001BEC46F0A2EC09F00D0E55EC01F00D0EBF
:10859000F76E5A0EF66E4DEC01F0A2EC09F00301F5
:1085A000FD510001E8A286D0A2EC09F0A2EC09F08E
:1085B00000EEB9F010EE56F0080EE75204E0E6CFF8
:1085C000EEFFE82EFAD7EF6AA2EC09F012EC4FF0BA
:1085D000A2EC09F00301FD510001E8A41FD0A2ECB8
:1085E00009F0200E55EC01F0560E55EC01F0200E6E
:1085F00055EC01F0A2EC09F0A2EC09F000EEB9F0A4
:1086000010EE5FF0080EE75204E0E6CFEEFFE82E32
:10861000FAD7EF6AA2EC09F012EC4FF0A2EC09F0E5
:108620000301FD510001E8A61FD0A2EC09F0200EC5
:1086300055EC01F0560E55EC01F0200E55EC01F012
:10864000A2EC09F0A2EC09F000EEB9F010EE68F02F
:10865000080EE75204E0E6CFEEFFE82EFAD7EF6A05
:10866000A2EC09F012EC4FF0A2EC09F00301FD516D
:108670000001E8A81FD0A2EC09F0200E55EC01F093
:10868000560E55EC01F0200E55EC01F0A2EC09F06D
:10869000A2EC09F000EEB9F010EE71F0080EE7520E
:1086A00004E0E6CFEEFFE82EFAD7EF6AA2EC09F07D
:1086B00012EC4FF0A2EC09F00D0E55EC01F00D0E8E
:1086C000F76E640EF66E4DEC01F0A2EC09F0A2EC30
:1086D00009F000EEB9F010EE4DF0080EE75204E09C
:1086E000E6CFEEFFE82EFAD7EF6AA2EC09F012EC23
:1086F0004FF0A2EC09F00D0E55EC01F00D0EF76EE7
:108700006C0EF66E4DEC01F0A2EC09F004010131A3
:1087100000010DE3A2EC09F0A2EC09F00401266BC4
:10872000530E256FA2EC09F000010EEC4FF0A2EC05
:1087300009F0040101510001E8A21BD0A2EC09F0EC
:1087400004010131000108E3A2EC09F02C0E55EC04
:1087500001F0200E55EC01F0A2EC09F0A2EC09F0BA
:108760000401266B5A0E256FA2EC09F000010EECF5
:108770004FF0A2EC09F0040101510001E8A415D06A
:10878000A2EC09F02C0E55EC01F0200E55EC01F096
:10879000A2EC09F0A2EC09F00401266B610E256F32
:1087A000A2EC09F000010EEC4FF0A2EC09F004017C
:1087B00001510001E8A615D0A2EC09F02C0E55ECF1
:1087C00001F0200E55EC01F0A2EC09F0A2EC09F04A
:1087D0000401266B680E256FA2EC09F000010EEC77
:1087E0004FF0A2EC09F0040101510001E8A815D0F6
:1087F000A2EC09F02C0E55EC01F0200E55EC01F026
:10880000A2EC09F0A2EC09F00401266B6F0E256FB3
:10881000A2EC09F000010EEC4FF0A2EC09F004010B
:1088200001510001E8AA15D0A2EC09F02C0E55EC7C
:1088300001F0200E55EC01F0A2EC09F0A2EC09F0D9
:108840000401266B760E256FA2EC09F000010EECF8
:108850004FF0A2EC09F0040101510001E8AC15D081
:10886000A2EC09F02C0E55EC01F0200E55EC01F0B5
:10887000A2EC09F0A2EC09F00401266B7D0E256F35
:10888000A2EC09F000010EEC4FF0A2EC09F004019B
:108890000135000115E3A2EC09F02C0E55EC01F0B6
:1088A000200E55EC01F0A2EC09F0A2EC09F0040155
:1088B000266B840E256FA2EC09F000010EEC4FF040
:1088C000A2EC09F0040100510001E8AC15D0A2ECC3
:1088D00009F02C0E55EC01F0200E55EC01F0A2EC45
:1088E00009F0A2EC09F00401266B8B0E256FA2ECB7
:1088F00009F000010EEC4FF0A2EC09F00401003584
:10890000000115E3A2EC09F02C0E55EC01F0200E4D
:1089100055EC01F0A2EC09F0A2EC09F00401266B81
:10892000920E256FA2EC09F000010EEC4FF0A2ECC4
:1089300009F00D0E55EC01F0440E55EC01F0450E1A
:1089400055EC01F0460E55EC01F0530E55EC01F0DC
:10895000200E55EC01F0A2EC09F00401096B050EA4
:108960000401095D000119E2A2EC09F0A2EC09F092
:10897000AA6A4E0E04010925A96ED8B0AA2AB0EC45
:1089800001F00B6FA2EC09F00B5155EC01F0A2ECD9
:1089900009F00401092B0001E2E3A2EC09F00D0E3D
:1089A00055EC01F0A2EC09F0040105510001E8B812
:1089B00065D0A2EC09F00D0EF76E740EF66E4DEC5C
:1089C00001F0A2EC09F00301FD510001E8AA0ED06C
:1089D000A2EC09F0A2EC09F0010E0401266F4C0E86
:1089E000256FA2EC09F00001F8D805D0A2EC09F03F
:1089F0000D0E55EC01F0A2EC09F00D0EF76E7E0E97
:108A0000F66E4DEC01F0A2EC09F00301FD510001FE
:108A1000E8AC0ED0A2EC09F0A2EC09F0020E0401C1
:108A2000266F170E256FA2EC09F00001D6D805D0ED
:108A3000A2EC09F00D0E55EC01F0A2EC09F00D0EC0
:108A4000F76E880EF66E4DEC01F0A2EC09F0030112
:108A5000FD3500010DE3A2EC09F0A2EC09F00401E0
:108A6000266BAA0E256FA2EC09F00001B6D805D03E
:108A7000A2EC09F00D0E55EC01F0ABD0A2EC09F020
:108A8000500E55EC01F0410E55EC01F0520E55EC34
:108A900001F04D0E55EC01F0200E55EC01F0A2EC6A
:108AA00009F00301FE510001E8A40ED0A2EC09F088
:108AB000A2EC09F0020E0401266FE20E256FA2EC73
:108AC00009F000018AD805D0A2EC09F00D0E55EC92
:108AD00001F0A2EC09F0550E55EC01F04E0E55ECEC
:108AE00001F0490E55EC01F0540E55EC01F0200E4A
:108AF00055EC01F0A2EC09F00301FE510001E8A2DF
:108B00000ED0A2EC09F0A2EC09F0030E0401266FCE
:108B1000410E256FA2EC09F000015FD805D0A2EC50
:108B200009F00D0E55EC01F0A2EC09F0450E55ECE4
:108B300001F0510E55EC01F04E0E55EC01F0530EC4
:108B400055EC01F0200E55EC01F0A2EC09F0030108
:108B5000FE510001E8A60ED0A2EC09F0A2EC09F04B
:108B6000030E0401266FA00E256FA2EC09F0000190
:108B700034D805D0A2EC09F00D0E55EC01F0A2ECB2
:108B800009F0420E55EC01F0490E55EC01F0540E7F
:108B900055EC01F0530E55EC01F0200E55EC01F0B0
:108BA000A2EC09F00301FE3100010EE3A2EC09F092
:108BB000A2EC09F0010E0401266F0F0E256FA2EC46
:108BC00009F000010AD805D0A2EC09F00D0E55EC11
:108BD00001F0A2EC09F00AEF50F0A2EC09F0040158
:108BE000626BC80E0401625D000123E2A2EC09F091
:108BF000A2EC09F026C4AAFF25C4A9FFB0EC01F03D
:108C000004010B6FA2EC09F00B5155EC01F0A2EC42
:108C100009F00D0E0B5D00010CE0A2EC09F004015F
:108C2000252B000E2623A2EC09F00401622B000183
:108C3000D8E3A2EF09F0A2EC09F004010B53000104
:108C40000EE1A2EC09F0340E55EC01F0380E55ECB3
:108C500001F0300E55EC01F055EC01F062D0010E40
:108C600004010B5D00010EE1A2EC09F0390E55EC98
:108C700001F0360E55EC01F0300E55EC01F055ECDC
:108C800001F04FD0020E04010B5D000111E1A2ECD6
:108C900009F0310E55EC01F0390E55EC01F0320EB1
:108CA00055EC01F0300E55EC01F055EC01F039D0E7
:108CB000030E04010B5D000111E1A2EC09F0330E7B
:108CC00055EC01F0380E55EC01F0340E55EC01F086
:108CD000300E55EC01F055EC01F023D0040E0401E8
:108CE0000B5D000111E1A2EC09F0350E55EC01F02D
:108CF000370E55EC01F0360E55EC01F0300E55EC08
:108D000001F055EC01F00DD0050E04010B5D0001E2
:108D100008E1A2EC09F00D0EF76E900EF66E4DEC28
:108D200001F0A2EC09F0200E55EC01F0420E55ECDA
:108D300001F0640E55EC01F0A2EF09F0A2EC09F08D
:108D4000040105350001D8B00AEF50F0A2EC09F09B
:108D50004EEC4FF0A2EC09F06BEC2CF0A2EC09F019
:108D60000401096B0A0E0401095D000129E2A2EC6D
:108D700009F001EE66F004010951E926000EEA222D
:108D8000EF500A6E0D0E0A5C0001D8B4C2EF4FF02E
:108D9000A2EC09F0A2EC09F001EE66F00401095121
:108DA000E926000EEA22EFCF0AF000EE7AF0095130
:108DB0000AC0EBFFA2EC09F00401092B0001D2E389
:108DC000A2EC09F00AEF50F0A2EC09F0040105351D
:108DD0000001D8B00AEF50F0A2EC09F04EEC4FF0D1
:108DE000A2EC09F06BEC2CF0A2EC09F00101665149
:108DF0000A6E4F0E0A5C000132E1A2EC09F001019B
:108E000067510A6E4E0E0A5C000127E1A2EC09F0E0
:108E1000A2EC09F004010683A2EC09F0A2EC09F02F
:108E20000301FE9DA2EC09F0A2EC09F0FE99A2EC70
:108E300009F0A2EC09F004010691A2EC09F0A2EC01
:108E400009F0069DA2EC09F0A2EC09F00301FF91E4
:108E5000A2EC09F0A2EC09F0FF93000104D0A2EC0F
:108E600009F0C2EF4FF0A2EC09F0A2EC09F0230EDA
:108E7000AEEC01F00301FD6FA2EC09F0A2EC09F0E9
:108E8000240EAEEC01F0FE6FA2EC09F0A2EC09F0AA
:108E9000250EAEEC01F0FF6FA2EC09F0A2EC09F098
:108EA000260EAEEC01F00401006FA2EC09F0A2EC7A
:108EB00009F0270EAEEC01F0016FA2EC09F0000101
:108EC0000AEF50F0A2EC09F04EEC4FF0A2EC09F0E2
:108ED000A2EC09F00101665104017B6FA2EC09F0DC
:108EE000A2EC09F00101675104017C6FA2EC09F0CA
:108EF000AA6A3C0EA96E7B51B7EC01F0A2EC09F016
:108F0000AA6A3D0EA96E7C51B7EC01F0A2EC09F003
:108F100000010AEF50F0A2EC09F045EC50F0A2EC91
:108F200009F0A2EC09F025C483F4A2EC09F0AA6AC6
:108F3000400EA96E04018351B7EC01F0A2EC09F0D8
:108F400000010AEF50F0A2EC09F045EC50F0A2EC61
:108F500009F0A2EC09F025C485F4A2EC09F0020E98
:108F60000401855D000107E2A2EC09F0A2EC09F022
:108F7000020E0401856F0001A2EC09F0AA6A420EFC
:108F8000A96E04018551B7EC01F0A2EC09F00001D3
:108F90000AEF50F0A2EC09F045EC50F0A2EC09F019
:108FA000A2EC09F025C486F4A2EC09F00A0E040133
:108FB000865D000107E2A2EC09F0A2EC09F00A0EBE
:108FC0000401866F0001A2EC09F0AA6A430EA96EA3
:108FD00004018651B7EC01F0A2EC09F000010AEFA0
:108FE00050F0A2EC09F0A2EC09F004010F6BA2EC26
:108FF00009F000015EEC51F0A2EC09F0A2EC09F0DE
:109000001EC433F01DC432F01CC431F01BC430F058
:1090100020C42DF01FC42CF07FEC04F070EC03F0A2
:109020002FC01AF42EC019F42DC018F42CC017F458
:10903000A2EC09F0AA6A280EA96E04011751B7EC38
:1090400001F01851B7EC01F01951B7EC01F01A51C9
:10905000B7EC01F0A2EC09F000010AEF50F0A2EC2D
:1090600009F0A2EC09F0010E04010F6FA2EC09F067
:1090700000015EEC51F0A2EC09F0A2EC09F01EC474
:1090800033F01DC432F01CC431F01BC430F020C4D6
:109090002DF01FC42CF07FEC04F070EC03F02FC017
:1090A0001AF42EC019F42DC018F42CC017F4A2EC39
:1090B00009F0AA6A2C0EA96E04011751B7EC01F051
:1090C0001851B7EC01F01951B7EC01F01A51B7EC97
:1090D00001F0A2EC09F000010AEF50F0A2EC09F057
:1090E000A2EC09F0020E04010F6FA2EC09F00001DE
:1090F0005EEC51F0A2EC09F0A2EC09F01EC433F0D2
:109100001DC432F01CC431F01BC430F020C42DF05B
:109110001FC42CF07FEC04F070EC03F02FC01AF4A5
:109120002EC019F42DC018F42CC017F4A2EC09F0CD
:10913000AA6A300EA96E04011751B7EC01F018515C
:10914000B7EC01F01951B7EC01F01A51B7EC01F08E
:10915000A2EC09F000010AEF50F0A2EC09F0A2EC39
:1091600009F0030E04010F6FA2EC09F000015EECA0
:1091700051F0A2EC09F0A2EC09F01EC433F01DC4BA
:1091800032F01CC431F01BC430F020C42DF01FC4D9
:109190002CF07FEC04F070EC03F02FC01AF42EC01A
:1091A00019F42DC018F42CC017F4A2EC09F0AA6A27
:1091B000340EA96E04011751B7EC01F01851B7EC49
:1091C00001F01951B7EC01F01A51B7EC01F0A2EC23
:1091D00009F000010AEF50F0A2EC09F0A2EC09F04E
:1091E0000301FE85A2EC09F0A2EC09F0020E0401D5
:1091F000266FE20E256FA2EC09F000013FD0A2EC31
:1092000009F0A2EC09F00301FE83A2EC09F0A2EC44
:1092100009F0030E0401266F410E256FA2EC09F040
:1092200000012CD0A2EC09F0A2EC09F00301FE87AA
:10923000A2EC09F0A2EC09F0030E0401266FA00EC7
:10924000256FA2EC09F0000119D0A2EC09F0A2EC04
:1092500009F00301FE81A2EC09F0A2EC09F0010E75
:109260000401266F0F0E256FA2EC09F0A2EC09F0A5
:10927000370E646FA2EC09F0000107D0A2EC09F0F0
:10928000A2EC09F04F0E0401646F0001A2EC09F09A
:1092900001016B510A6E0D0E0A5C0001D8A450D07A
:1092A000A2EC09F004012651020AE20ED8B42519F5
:1092B000000106E1A2EC09F0A2EC09F00301FE9521
:1092C0000001A2EC09F004012651030A410ED8B4B2
:1092D0002519000106E1A2EC09F0A2EC09F0030156
:1092E000FE930001A2EC09F004012651030AA00E2E
:1092F000D8B42519000106E1A2EC09F0A2EC09F0AE
:109300000301FE970001A2EC09F004012651010AB5
:109310000F0ED8B42519000106E1A2EC09F0A2EC69
:1093200009F00301FE910001A2EC09F026C4AAFF96
:1093300025C4A9FF0D0EB7EC01F0A2EC09F05CD03A
:10934000A2EC09F04EEC4FF0A2EC09F001016651DD
:109350000A6E0D0E0A5C00010AE1A2EC09F026C4B7
:10936000AAFF25C4A9FF0D0EB7EC01F044D0A2EC72
:1093700009F00401096B04010951645D00012FE348
:10938000A2EC09F0A2EC09F001EE66F0040109512B
:10939000E926000EEA22EF500B6FA2EC09F00D0E49
:1093A0000B5D010ED8A4000E376E0A0E0B5D010E88
:1093B000D8A4000E3712000112E1A2EC09F004015A
:1093C00009512525A96E000E2621AA6E0B51B7EC76
:1093D00001F0A2EC09F00401092B0001CCE3A2EC9E
:1093E00009F0040109512525A96E000E2621AA6E57
:1093F0000D0EB7EC01F00001A2EC09F0AA6A240EF0
:10940000A96E0301FE51B7EC01F0A2EC09F00001D6
:109410000AEF50F0A2EC09F001016A510A6E0D0E3C
:109420000A5C0001D8B40AEF50F0A2EC09F04EEC4F
:109430004FF0A2EC09F0010166510A6E0D0E0A5CB4
:10944000000115E1A2EC09F0AA6A4E0EA96E300ED9
:10945000B7EC01F0300EB7EC01F0300EB7EC01F0D4
:10946000300EB7EC01F0300EB7EC01F0A1D0A2EC59
:1094700009F00401096B050E0401095D0001D8B073
:1094800097D0A2EC09F0A2EC09F001EE66F004011D
:109490000951E926000EEA22EF500B6FA2EC09F009
:1094A0003A0E0B5D000106E3A2EC09F0A2EC09F014
:1094B00004010B9B0001A2EC09F0410E04010B5DBD
:1094C000010ED8A4000E376E540E0B5D010ED8A409
:1094D000000E3712300E0B5D010ED8A4000E3712AD
:1094E00000010EE0A2EC09F0AA6A4E0E0401092563
:1094F000A96ED8B0AA2A0B51B7EC01F0000151D0E7
:10950000A2EC09F0040E0401095D010ED8A4000EBE
:10951000376E410E0B5D010ED8A4000E3716000108
:109520003CE0A2EC09F00401053500011BE2A2ECCD
:1095300009F00D0E55EC01F00D0EF76E980EF66E5B
:109540004DEC01F00D0E55EC01F0630E55EC01F001
:109550006D0E55EC01F0640E55EC01F03E0E55EC2D
:1095600001F019D0A2EC09F0A2EC09F001EE66F0CE
:109570000D0EEE6E0D0EF76E980EF66EB5EC02F057
:109580000D0EEE6E630EEE6E6D0EEE6E640EEE6EF2
:109590003E0EEE6EEE6AA2EF09F0A2EC09F0C2EF09
:1095A0004FF0A2EC09F00401092B0001D8A063D709
:1095B000A2EC09F00AEF50F0A2EC09F00401053525
:1095C000000122E2A2EC09F00D0E55EC01F00D0EA7
:1095D000F76EB00EF66E4DEC01F0040E016E046AEB
:1095E000176A166E69EC00F02E0E55EC01F0010EB4
:1095F000046E310E67EC00F00D0E55EC01F0A2EC9C
:1096000009F00AEF50F032D0A2EC09F0A2EC09F018
:1096100001EE66F00D0EEE6E0D0EF76EB00EF66EEC
:10962000B5EC02F0020E016E046A176A040E166EA3
:1096300069EC00F02E0EEE6E020E016E010E046E4D
:10964000310E67EC00F00D0EEE6E4F0EEE6E4B0E0F
:10965000EE6E0D0EEE6E630EEE6E6D0EEE6E640E21
:10966000EE6E3E0EEE6E0D0EEE6EEE6AA2EC09F0A0
:10967000A2EC09F0AECF0BF4A2EF09F0A2EC09F0D6
:109680008CEC53F0A2EC09F004015B310001D8B07E
:10969000C2EF4FF0A2EC09F0A2EC09F0260EAEECFE
:1096A00001F00401006FA2EC09F0A2EC09F0D892DD
:1096B0005EB7D882D8B2008BD8A2009BA2EC09F08A
:1096C000AA6A260EA96E0051B7EC01F0A2EC09F0CF
:1096D00000010AEF50F0A2EC09F08CEC53F0A2EC80
:1096E00009F004015B310001D8B0C2EF4FF0A2ECE9
:1096F00009F0A2EC09F00401D8925EB7D882D8B282
:109700000281D8A20291A2EC09F0AA6A990EA96E70
:109710000251B7EC01F0A2EC09F000010AEF50F0A1
:10972000A2EC09F0040105350001D8B00AEF50F0B1
:10973000A2EC09F00D0E55EC01F00D0EF76EC20E05
:10974000F66E4DEC01F00D0E55EC01F00D0E55ECE2
:1097500001F0A2EC09F00D0EF76EDC0EF66E4DEC8A
:1097600001F00D0E55EC01F0A2EC09F00D0EF76EB4
:10977000F60EF66E4DEC01F00D0E55EC01F0A2EC7C
:1097800009F00E0EF76E2A0EF66E4DEC01F00D0E7E
:1097900055EC01F0A2EC09F00E0EF76E420EF66EDB
:1097A0004DEC01F00D0E55EC01F0A2EC09F00E0E9F
:1097B000F76E5A0EF66E4DEC01F00D0E55EC01F001
:1097C000A2EC09F00E0EF76EB20EF66E4DEC01F043
:1097D0000D0E55EC01F0A2EC09F00E0EF76ED40E52
:1097E000F66E4DEC01F00D0E55EC01F0A2EC09F017
:1097F0000E0EF76EF20EF66E4DEC01F00D0E55ECFE
:1098000001F0A2EC09F00F0EF76E000EF66E4DECB3
:1098100001F00D0E55EC01F0A2EC09F00F0EF76E01
:10982000120EF66E4DEC01F00D0E55EC01F0A2ECAF
:1098300009F00F0EF76E260EF66E4DEC01F00D0ED0
:1098400055EC01F0A2EC09F00F0EF76E340EF66E37
:109850004DEC01F00D0E55EC01F0A2EC09F00F0EED
:10986000F76E520EF66E4DEC01F00D0E55EC01F058
:10987000A2EC09F00F0EF76E860EF66E4DEC01F0BD
:109880000D0E55EC01F0A2EC09F00F0EF76EA60ECE
:10989000F66E4DEC01F00D0E55EC01F0A2EC09F066
:1098A0000F0EF76ECA0EF66E4DEC01F00D0E55EC74
:1098B00001F0A2EC09F00F0EF76EE20EF66E4DEC21
:1098C00001F00D0E55EC01F0A2EC09F00F0EF76E51
:1098D000F40EF66E4DEC01F00D0E55EC01F0A2EC1D
:1098E00009F0100EF76E1C0EF66E4DEC01F00D0E29
:1098F00055EC01F0A2EC09F0100EF76E340EF66E86
:109900004DEC01F00D0E55EC01F0A2EC09F0100E3B
:10991000F76E5A0EF66E4DEC01F00D0E55EC01F09F
:10992000A2EC09F0100EF76E7A0EF66E4DEC01F017
:109930000D0E55EC01F0A2EC09F0100EF76EAA0E18
:10994000F66E4DEC01F00D0E55EC01F0A2EC09F0B5
:10995000100EF76EE60EF66E4DEC01F00D0E55ECA6
:1099600001F0A2EC09F0110EF76E0A0EF66E4DEC46
:1099700001F00D0E55EC01F0A2EC09F0110EF76E9E
:10998000360EF66E4DEC01F00D0E55EC01F0A2EC2A
:1099900009F0110EF76E640EF66E4DEC01F00D0E2F
:1099A00055EC01F0A2EC09F0110EF76E900EF66E78
:1099B0004DEC01F00D0E55EC01F0A2EC09F0110E8A
:1099C000F76EB60EF66E4DEC01F00D0E55EC01F093
:1099D000A2EC09F0110EF76EC20EF66E4DEC01F01E
:1099E0000D0E55EC01F0A2EC09F0110EF76ECE0E43
:1099F000F66E4DEC01F00D0E55EC01F0A2EC09F005
:109A0000110EF76EDA0EF66E4DEC01F00D0E55EC00
:109A100001F0A2EC09F0110EF76EEE0EF66E4DECB1
:109A200001F00D0E55EC01F0A2EC09F0110EF76EED
:109A3000FE0EF66E4DEC01F00D0E55EC01F0A2ECB1
:109A400009F0120EF76E340EF66E4DEC01F00D0EAD
:109A500055EC01F0A2EC09F0120EF76E5E0EF66EF8
:109A60004DEC01F00D0E55EC01F0A2EC09F0120ED8
:109A7000F76E9E0EF66E4DEC01F00D0E55EC01F0FA
:109A8000A2EC09F0120EF76EBC0EF66E4DEC01F072
:109A90000D0E55EC01F0A2EC09F0120EF76EEC0E73
:109AA000F66E4DEC01F00D0E55EC01F0A2EC09F054
:109AB0000AEF50F0A2EC09F0A2EC09F004015D916C
:109AC000A2EC09F000016BEC2CF0A2EC09F0A2EC86
:109AD00009F004010491A2EC09F0A2EC09F0096B71
:109AE000A2EC09F0000101EE66F004010951E9263B
:109AF000000EEA22EF500A6E2D0E0A5CD8A4010E69
:109B0000376E01EE66F00951E926000EEA22EF50A9
:109B10000A6E200E0A5CD8A4010E371601EE66F01C
:109B20000951E926000EEA22EF500A6E0D0E0A5C7A
:109B3000D8A4010E37160A0E095D010ED8B0000E2A
:109B40003716000117E0A2EC09F0A2EC09F001EED3
:109B500066F004010951E926000EEA22EFCF0AF06F
:109B600000EEB9F009510AC0EBFFA2EC09F0092B95
:109B70000001B8D7A2EC09F0060E0401095D00014E
:109B80001EE2A2EC09F0A2EC09F009C40AF4A2EC6E
:109B900009F0060E04010A5D000111E2A2EC09F0D1
:109BA000A2EC09F0200EF36E00EEB9F004010A51A8
:109BB000F3CFEBFFA2EC09F00A2B0001EAD7A2ECED
:109BC00009F001EE66F004010951E926000EEA22CF
:109BD000EF500A6E200E0A5C000105E1A2EC09F0CC
:109BE000A2EC09F0BF6BA2EC09F001EE66F00401F3
:109BF0000951E926000EEA22EF500A6E0D0E0A5CAA
:109C000000010EE1A2EC09F0A2EC09F004010481CC
:109C1000A2EC09F0A2EC09F00001BF6BA2EF09F081
:109C2000A2EC09F001EE66F004010951E926000EEC
:109C3000EA22EF500A6E2D0E0A5C0001D8A48CD0E7
:109C4000A2EC09F00401092BA2EC09F0A2EC09F046
:109C500001EE66F00951E926000EEA22EF500A6E85
:109C60000F0E0A144B6EA2EC09F0092BA2EC09F0BE
:109C700001EE66F00951E926000EEA22EF500A6E65
:109C8000300E0A5C000ED8B0010E376E01EE66F0A1
:109C90000951E926000EEA22EF500A6E3A0E0A5CDC
:109CA000000102E3000E01D0010E371635E0A2ECF0
:109CB00009F0A2EC09F0216A0A0E206E21C00EF014
:109CC0004B502002F3CF20F0F4CF21F00E02F350DE
:109CD000212601EE66F004010951E926000EEA2270
:109CE000EF500A6E256A0AC024F00F0E2416000EEB
:109CF0002516205024244B6EA2EC09F0100E4B5C6C
:109D0000000106E3A2EC09F0A2EC09F00F0E4B6E85
:109D1000A2EC09F00401092B0001A2EC09F0A2EC6D
:109D200009F04BC0BFF0A2EC09F001EE66F00401AF
:109D30000951E926000EEA22EF500A6E0D0E0A5C68
:109D400000010AE1A2EC09F0A2EC09F0040104818F
:109D5000A2EC09F000011200A2EC09F00401092BA9
:109D6000A2EC09F001EE66F00951E926000EEA22A4
:109D7000EF500A6E560E0A5C010ED8A4000E376E24
:109D800001EE66F00951E926000EEA22EF500A6E54
:109D9000760E0A5C010ED8A4000E3712000107E00F
:109DA000A2EC09F07BD8A2EC09F078D806D0A2EC9E
:109DB00009F0A2EC09F004015D810001A2EF09F0B5
:109DC000A2EC09F00401096B070E0401095D000112
:109DD00023E2A2EC09F0A2EC09F000EEB9F00401D4
:109DE0000951EB500A6ED8900A34476EA2EC09F084
:109DF000060E095D000106E1A2EC09F0A2EC09F0F3
:109E00004B504712A2EC09F0C8EC15F0A2EC09F097
:109E10000401092B0001D8E3A2EF09F0A2EC09F03C
:109E200096EC54F0A2EC09F0A2EC09F00401096BE5
:109E3000A2EC09F0000100EEB9F004010951EB5069
:109E40000A6E200E0A5CD8A4010E376E060E095D5C
:109E5000010ED8B0000E371600010EE0A2EC09F09A
:109E600000EEB9F004010951EB5055EC01F0A2EC01
:109E700009F0092B0001DED7A2EC09F0BF510A6EF0
:109E80000A520AE0A2EC09F02D0E55EC01F0040E86
:109E9000016EBF5166EC00F0A2EF09F0A2EC09F0F0
:109EA000A2EC09F004015D91A2EC09F0A2EC09F02A
:109EB000626BA2EC09F0000101EE66F00401625150
:109EC000E926000EEA22EF500A6E200E0A5CD8A4A2
:109ED000010E376EFD0E625D010ED8B0000E371612
:109EE00000011FE0A2EC09F001EE66F004016251EE
:109EF000E926000EEA22EF500A6E0D0E0A5C000100
:109F00000AE1A2EC09F0A2EC09F004015D81A2ECE7
:109F100009F000011200A2EC09F00401622B00011B
:109F2000CAD7A2EC09F00401622BA2EC09F062513D
:109F3000FF08086E0A6B04010A51085C000120E367
:109F4000A2EC09F0A2EC09F004010A5162250C6EA2
:109F50000D6A0D360C50660FE96E010E0D20EA6E8B
:109F6000EFCF0AF001EE66F00A51E926000EEA2270
:109F70000AC0EFFFA2EC09F004010A2B0001DBE3A9
:109F8000A2EF09F0A2EC09F004010535000120E27E
:109F9000A2EC09F0450E55EC01F0520E55EC01F023
:109FA00055EC01F04F0E55EC01F0520E55EC01F05E
:109FB0000D0E55EC01F0630E55EC01F06D0E55ECF5
:109FC00001F0640E55EC01F03E0E55EC01F01AD094
:109FD000A2EC09F0A2EC09F001EE66F0450EEE6E7F
:109FE000520EEE6EEE6E4F0EEE6E520EEE6E0D0EC9
:109FF000EE6E630EEE6E6D0EEE6E640EEE6E3E0E47
:10A00000EE6EEE6AA2EC09F0A2EC09F0AECF0BF412
:10A01000A2EF09F0A2EC09F004010535000118E2F5
:10A02000A2EC09F04F0E55EC01F04B0E55EC01F08F
:10A030000D0E55EC01F0630E55EC01F06D0E55EC74
:10A0400001F0640E55EC01F03E0E55EC01F015D018
:10A05000A2EC09F0A2EC09F001EE66F04F0EEE6EF4
:10A060004B0EEE6E0D0EEE6E630EEE6E6D0EEE6E20
:10A07000640EEE6E3E0EEE6EEE6AA2EC09F0A2ECFD
:10A0800009F0AECF0BF4A2EF09F0A2EC09F006DF65
:10A09000A2EC09F0A2EC09F0010166510A6E0F0E64
:10A0A0000A140401266B256FA2EC09F00101675127
:10A0B0000A6E0D0E0A5C0001D8B4C6D0A2EC09F0FD
:10A0C000A2EC09F0216A0A0E206E21C017F0205080
:10A0D000166E04012503F3CF20F0F4CF21F01750C2
:10A0E0002503F350212616502603F35021260101A3
:10A0F00067510A6E256A0AC024F00F0E2416000E5E
:10A100002516245020240401256F25502120266F78
:10A11000A2EC09F0010168510A6E0D0E0A5C000103
:10A12000D8B492D0A2EC09F0A2EC09F0216A0A0E90
:10A13000206E21C017F02050166E04012503F3CFC6
:10A1400020F0F4CF21F017502503F35021261650AC
:10A150002603F3502126010168510A6E256A0AC0C0
:10A1600024F00F0E2416000E25162450202404017E
:10A17000256F25502120266FA2EC09F001016951BD
:10A180000A6E0D0E0A5C0001D8B45ED0A2EC09F094
:10A19000A2EC09F0216A0A0E206E21C017F02050AF
:10A1A000166E04012503F3CF20F0F4CF21F01750F1
:10A1B0002503F350212616502603F35021260101D2
:10A1C00069510A6E256A0AC024F00F0E2416000E8B
:10A1D0002516245020240401256F25502120266FA8
:10A1E000A2EC09F001016A510A6E0D0E0A5C000131
:10A1F0002AE0A2EC09F0A2EC09F0216A0A0E206E16
:10A2000021C017F02050166E04012503F3CF20F073
:10A21000F4CF21F017502503F350212616502603C2
:10A22000F350212601016A510A6E256A0AC024F002
:10A230000F0E2416000E2516245020240401256F2D
:10A2400025502120266F0001A2EF09F0A2EC09F0B1
:10A25000A2EC09F0426AA2EC09F0A2EC09F0436A10
:10A26000A2EC09F0A2EC09F0446AA2EC09F0A2EC1D
:10A2700009F0456AA2EC09F0A2EC09F0476AA2ECE9
:10A2800009F0A2EC09F0486AA2EC09F0A2EC09F08E
:10A290004A6A496AA2EC09F0A2EC09F04B6AA2EC06
:10A2A00009F0A2EC09F00401816BA2EC09F0A2EC28
:10A2B00009F00489A2EC09F000011200A2EC09F0F7
:10A2C000EDDDA2EC09F0A2EC09F00401206B1F6B9C
:10A2D000A2EC09F0096B0B0E0401095D0001D8B076
:10A2E00064D0A2EC09F001EE66F004010951E92600
:10A2F000000EEA22EF500A6E2E0E0A5C010ED8A460
:10A30000000E376E01EE66F00951E926000EEA22D2
:10A31000EF500A6E2C0E0A5C010ED8A4000E371204
:10A3200001EE66F00951E926000EEA22EF500A6EAE
:10A330000D0E0A5C010ED8A4000E3712000135E1A3
:10A34000A2EC09F0A2EC09F0216A0A0E206E21C0ED
:10A3500017F02050166E04011F03F3CF20F0F4CF46
:10A3600021F017501F03F350212616502003F350FD
:10A37000212601EE66F00951E926000EEA22EF508F
:10A380000A6E256A0AC024F00F0E2416000E251648
:10A39000245020241F6F25502120206FA2EC09F0AB
:10A3A0000401092B0001D8A096D7A2EC09F00A0EEF
:10A3B0000401095D0001D8B4E5D5A2EC09F001EE75
:10A3C00066F004010951E926000EEA22EF500A6EF8
:10A3D0000D0E0A5C000115E1A2EC09F0A2EC09F0F7
:10A3E00020C42DF01FC42CF07FEC04F02FC01EF40D
:10A3F0002EC01DF42DC01CF42CC01BF4A2EC09F0DF
:10A40000C8D0A2EC09F00B6A040109290A6ED8B47D
:10A410000B2A0A50660FE96E010E0B20EA6EEF5010
:10A420000A6E0D0E0A5C000133E0A2EC09F0A2EC0A
:10A4300009F0216A0A0E206E21C017F02050166E16
:10A4400004011F03F3CF20F0F4CF21F017501F03B6
:10A45000F350212616502003F35021260D6A0929B6
:10A460000C6ED8B40D2A0C50660FE96E010E0D204B
:10A47000EA6EEF500A6E256A0AC024F00F0E241609
:10A48000000E2516245020241F6F25502120206FF8
:10A490000001A2EC09F00B6A020E040109250A6E04
:10A4A000D8B00B2A0A50660FE96E010E0B20EA6E37
:10A4B000EF500A6E0D0E0A5C0001D8B450D0A2EC29
:10A4C00009F0A2EC09F0216A0A0E206E21C017F0F3
:10A4D0002050166E04011F03F3CF20F0F4CF21F0BB
:10A4E00017501F03F350212616502003F350212646
:10A4F0000D6A020E09250C6ED8B00D2A0C50660F9D
:10A50000E96E010E0D20EA6EEF500A6E256A0AC050
:10A5100024F00F0E2416000E2516245020241F6F41
:10A5200025502120206FA2EC09F0A2EC09F0336A3B
:10A53000326A480E316E850E306E20C42DF01FC475
:10A540002CF07FEC04F070EC03F02FC01EF42EC052
:10A550001DF42DC01CF42CC01BF400011AD0A2EC79
:10A5600009F0A2EC09F0336A326A200E316E820ED5
:10A57000306E20C42DF01FC42CF07FEC04F070EC82
:10A5800003F02FC01EF42EC01DF42DC01CF42CC0EF
:10A590001BF4A2EC09F0A2EC09F00401206B1F6B84
:10A5A000A2EC09F0616B060E0401615D000119E285
:10A5B000A2EC09F0A2EC09F004010F51C6EC01F085
:10A5C000256F21C026F4A2EC09F0A2EC09F0255178
:10A5D0001F2726512023A2EC09F00401612B000162
:10A5E000E2E3A2EF09F0A2EC09F0D3DFA2EC09F05C
:10A5F00004010F53000114E1A2EC09F0A2EC09F0F0
:10A60000280EAEEC01F00401176FB0EC01F0186FEA
:10A61000B0EC01F0196FB0EC01F01A6F00014AD0F4
:10A62000010E04010F5D000114E1A2EC09F0A2EC9F
:10A6300009F02C0EAEEC01F00401176FB0EC01F044
:10A64000186FB0EC01F0196FB0EC01F01A6F000157
:10A6500031D0020E04010F5D000114E1A2EC09F0FB
:10A66000A2EC09F0300EAEEC01F00401176FB0EC73
:10A6700001F0186FB0EC01F0196FB0EC01F01A6F37
:10A68000000118D0030E04010F5D000112E1A2ECDD
:10A6900009F0A2EC09F0340EAEEC01F00401176FE2
:10A6A000B0EC01F0186FB0EC01F0196FB0EC01F0F4
:10A6B0001A6F0001A2EC09F0A2EC09F01AC433F001
:10A6C00019C432F018C431F017C430F020C42DF092
:10A6D0001FC42CF07FEC04F070EC03F02FC024F4C6
:10A6E0002EC023F42DC022F42CC021F4A2EC09F0DA
:10A6F000A2EC09F000EEB9F0020E016E24C423F0C2
:10A7000023C422F022C421F021C420F0010EA2ECC7
:10A7100000F0EE6AA2EF09F0A2EC09F04EEC4FF067
:10A72000A2EC09F06BEC2CF0A2EC09F0A2EC09F021
:10A7300004015B91A2EC09F0010166510A6E4F0E13
:10A740000A5C00012AE1A2EC09F0010167510A6EDE
:10A750004E0E0A5C000108E1A2EC09F0A2EC09F03F
:10A7600004015E87000118D0A2EC09F001016751D5
:10A770000A6E460E0A5C000108E1A2EC09F0A2ECA8
:10A7800009F004015E97000106D0A2EC09F0A2ECEA
:10A7900009F004015B81000106D0A2EC09F0A2ECF3
:10A7A00009F004015B810001A2EF09F0A2EC09F0BD
:10A7B000BDD8A2EC09F0A2EC09F004015B81A2EC87
:10A7C00009F0380E635D000107E3A2EC09F0A2EC8A
:10A7D00009F0370E0401636F0001A2EC09F00401D7
:10A7E0000A6B04010A51635D0001D8A05BD0A2ECA2
:10A7F00009F0A2EC09F00401096BA2EC09F00001D8
:10A8000000EEB9F004010951EB500A6E0A52000142
:10A8100037E0A2EC09F0A2EC09F004010A51092585
:10A820000A6E0B6A0B360A50660FE96E010E0B209A
:10A83000EA6EEF500B6FA2EC09F0A2EC09F0D89091
:10A840000B33A2EC09F0060E095D000107E1A2EC52
:10A8500009F0A2EC09F00F0E04010B170001A2ECA5
:10A8600009F000EEB9F004010951EB500A6E0B5DDE
:10A87000000110E1A2EC09F00401092B0001BFD78F
:10A88000A2EC09F0A2EC09F004015B91A2EC09F042
:10A89000000108D0A2EC09F0070E04010A2700010C
:10A8A000D8A09FD7A2EC09F0A2EC09F0040109514D
:10A8B0000A25456EA2EC09F000011200A2EC09F095
:10A8C000A2EC09F004015B91A2EC09F0096B070E00
:10A8D0000401095D000128E2A2EC09F000EEB9F0E4
:10A8E00004010951EB500A6E0D6A070E09250C6E22
:10A8F000D8B00D2A0C50660FE96E010E0D20EA6EDD
:10A90000EF500C6E0A500C5C000108E0A2EC09F05C
:10A91000A2EC09F004015B81000106D0A2EC09F071
:10A920000401092B0001D3E3A2EF09F0A2EC09F026
:10A930000401096B070E0401095D00011DE2A2EC90
:10A9400009F0A2EC09F0040109512525A96E000EB9
:10A950002621AA6EB0EC01F00B6FA2EC09F0A2EC7C
:10A9600009F000EEB9F009510BC4EBFFA2EC09F0BD
:10A970000401092B0001DEE3A2EC09F0A2EC09F0CE
:10A98000C06BA2EF09F0A2EC09F00401096B070EFD
:10A990000401095D000125E2A2EC09F0A2EC09F036
:10A9A000040109512525A96E000E2621AA6EB0ECDE
:10A9B00001F00B6FA2EC09F009512525206E000E65
:10A9C0002621216E070E205CA96E000E2158AA6E6A
:10A9D0000B51B7EC01F0A2EC09F00401092B0001C6
:10A9E000D6E3A2EF09F0A2EC09F0A2EC09F03E6A6E
:10A9F000AA0E3D6EA2EC09F0A2EC09F0630E3D2414
:10AA00003F6E000E3E20406EA2EC09F020D0A2EC7A
:10AA100009F0A2EC09F0010E3E6E4C0E3D6EA2EC68
:10AA200009F004015E31000108E3A2EC09F0A2EC98
:10AA300009F0020E3E6E170E3D6EA2EC09F0A2EC7C
:10AA400009F0FE0E3D243F6E000E3E20406EA2EC4B
:10AA500009F03EC014F43DC013F4040113513F5CEF
:10AA6000145140580001D8A0E7D1A2EC09F0A2ECA3
:10AA700009F014C4AAFF13C4A9FFB0EC01F004014B
:10AA80000B6FA2EC09F00D0E0B5D0001D8B4A2EF24
:10AA900009F0A2EC09F05C0E04010B5D0001D8A4E2
:10AAA000C2D1A2EC09F0A2EC09F0010E04011325B9
:10AAB000A96E000E1421AA6EB0EC01F00B6FA2EC8F
:10AAC00009F0A2EC09F00B9BA2EC09F0550E0B5D0E
:10AAD000010ED8A4000E376E560E0B5D010ED8A4E1
:10AAE000000E3712570E0B5D010ED8A4000E371260
:10AAF000580E0B5D010ED8A4000E3712590E0B5DD7
:10AB0000010ED8A4000E3712000105E0A2EC09F0F6
:10AB100043EC63F088D1A2EC09F0520E04010B5D06
:10AB200000011BE1A2EC09F0A2EC09F001EE5BF0E0
:10AB3000020E016E046A42C417F041C416F069ECBB
:10AB400000F03A0EEE6E020E016E046E04018951A1
:10AB500067EC00F0EE6A000166D1A2EC09F0040196
:10AB60005C510001E8A85FD1A2EC09F04C0E040191
:10AB70000B5D0001D8A466D0A2EC09F0A2EC09F0AC
:10AB8000CFC033F4D0C034F4A2EC09F0010E0401BC
:10AB9000616F0F0E0401615D00012FE2A2EC09F06C
:10ABA00000EECFF0D89004016135E926000EEA22CC
:10ABB000EECF0AF0EFCF0BF033510A5C34510B5853
:10ABC0000B503419D8B0800A000110E6A2EC09F04D
:10ABD000A2EC09F000EECFF0D89004016135E9262F
:10ABE000000EEA22EECF33F4EFCF34F40001A2ECF2
:10ABF00009F00401612B0001CCE3A2EC09F0A2EC06
:10AC000009F001EE45F0020E016E046A34C41DF035
:10AC100033C41CF0176A0A0E166E4BEC02F0166E67
:10AC20000FC017F064EC00F02E0EEE6E020E016EF7
:10AC3000010E046E34C417F033C416F069EC00F052
:10AC4000EE6AF1D0A2EC09F0480E04010B5D0001A0
:10AC5000D8A466D0A2EC09F0A2EC09F0CFC033F47E
:10AC6000D0C034F4A2EC09F0010E0401616F0F0EA4
:10AC70000401615D00012FE2A2EC09F000EECFF0CB
:10AC8000D89004016135E926000EEA22EECF0AF0E1
:10AC9000EFCF0BF00A50335D0B5034590B50341981
:10ACA000D8B0800A000110E6A2EC09F0A2EC09F08D
:10ACB00000EECFF0D89004016135E926000EEA22BB
:10ACC000EECF33F4EFCF34F40001A2EC09F004012D
:10ACD000612B0001CCE3A2EC09F0A2EC09F001EE3B
:10ACE00050F0020E016E046A34C41DF033C41CF02F
:10ACF000176A0A0E166E4BEC02F0166E0FC017F0B4
:10AD000064EC00F02E0EEE6E020E016E010E046E6B
:10AD100034C417F033C416F069EC00F0EE6A83D047
:10AD2000A2EC09F0530E04010B5D0001D8A460D021
:10AD3000A2EC09F0A2EC09F00401346B336BA2EC35
:10AD400009F0616B0F0E0401615D00011AE2A2ECD3
:10AD500009F0A2EC09F000EECFF0D89004016135C3
:10AD6000E926000EEA22EECF0AF0EFCF0BF00A50F0
:10AD700033270B503423A2EC09F00401612B0001AE
:10AD8000E1E3A2EC09F0A2EC09F034C41DF033C4F5
:10AD90001CF0176A0F0E166E4BEC02F00401336FB5
:10ADA0000FC034F4A2EC09F0A2EC09F001EE3AF085
:10ADB000020E016E046A34C41DF033C41CF0176A1D
:10ADC0000A0E166E4BEC02F0166E0FC017F064EC14
:10ADD00000F02E0EEE6E020E016E010E046E34C4F3
:10ADE00017F033C416F069EC00F0EE6A00011BD0D6
:10ADF000A2EC09F0540E04010B5D000114E1A2EC79
:10AE000009F0A2EC09F000EEF8F0020E016E30C479
:10AE100023F02FC422F02EC421F02DC420F0010E07
:10AE2000A2EC00F0EE6AA2EC09F00401132B000E74
:10AE300014230001D8A011D6A2EF09F0A2EC09F06A
:10AE4000A2EC09F004015D91A2EC09F0A2EC09F07A
:10AE5000666BA2EC09F0A2EC09F0676BA2EC09F0BA
:10AE6000A2EC09F0686BA2EC09F0A2EC09F0696BA6
:10AE7000A2EC09F0A2EC09F06A6BA2EC09F0A2ECDA
:10AE800009F06B6BA2EC09F0A2EC09F00A6BA2ECE2
:10AE900009F0000177EC5EF0A2EC09F0A2EC09F0F9
:10AEA00001EE66F004010A51E926000EEA22EF5095
:10AEB000706FA2EC09F00A2BA2EC09F0A2EC09F0E9
:10AEC00001EE66F00A51E926000EEA22EF50716F9A
:10AED000A2EC09F00A2BA2EC09F0A2EC09F001EEB9
:10AEE00066F00A51E926000EEA22EF50726FA2ECDA
:10AEF00009F00A2BA2EC09F0A2EC09F001EE66F0D1
:10AF00000A51E926000EEA22EF50736FA2EC09F015
:10AF10000A2BA2EC09F001EE66F00A51E926000EB8
:10AF2000EA22EF500A6E2E0E0A5C0001D8A45BEFF5
:10AF30005EF0A2EC09F004010A2BA2EC09F0A2ECED
:10AF400009F001EE66F00A51E926000EEA22EF5000
:10AF5000746FA2EC09F00A2BA2EC09F0A2EC09F044
:10AF600001EE66F00A51E926000EEA22EF50756FF5
:10AF7000A2EC09F000017DEC5EF0A2EC09F001EE1C
:10AF800066F004010A51E926000EEA22EF500A6E2B
:10AF90004E0E0A5C000108E1A2EC09F0A2EC09F0F7
:10AFA00004015C8D00011BD0A2EC09F001EE66F0FB
:10AFB00004010A51E926000EEA22EF500A6E530EF0
:10AFC0000A5C000108E1A2EC09F0A2EC09F004011E
:10AFD0005C9D000104D0A2EC09F05BEF5EF0A2ECF6
:10AFE00009F0A2EC09F0020E04010A27A2EC09F014
:10AFF000A2EC09F001EE66F00A51E926000EEA2201
:10B00000EF500A6E0F0E0A14766FA2EC09F00A2BAD
:10B01000A2EC09F0A2EC09F0216A76C420F02150DC
:10B020000A0DF3CF21F020500A0DF3CF20F0F45099
:10B03000212601EE66F00A51E926000EEA22EF50C1
:10B040000A6E256A0AC024F00F0E2416000E25167B
:10B0500020502424766FA2EC09F00A2BA2EC09F010
:10B06000A2EC09F0216A76C420F021500A0DF3CF3A
:10B0700021F020500A0DF3CF20F0F450212601EEEC
:10B0800066F00A51E926000EEA22EF500A6E256AA0
:10B090000AC024F00F0E2416000E2516205024247A
:10B0A000766FA2EC09F00A2BA2EC09F0A2EC09F0F1
:10B0B00001EE66F00A51E926000EEA22EF500A6E10
:10B0C0000F0E0A14776FA2EC09F00A2BA2EC09F01C
:10B0D000A2EC09F0216A77C420F021500A0DF3CFC9
:10B0E00021F020500A0DF3CF20F0F450212601EE7C
:10B0F00066F00A51E926000EEA22EF500A6E256A30
:10B100000AC024F00F0E2416000E25162050242409
:10B11000776FA2EC09F0A2EC09F0020E0A27A2EC6C
:10B1200009F0A2EC09F001EE66F00A51E926000EE2
:10B13000EA22EF500A6E0F0E0A14786FA2EC09F0A3
:10B140000A2BA2EC09F0A2EC09F0216A78C420F0E5
:10B1500021500A0DF3CF21F020500A0DF3CF20F03B
:10B16000F450212601EE66F00A51E926000EEA228B
:10B17000EF500A6E256A0AC024F00F0E2416000E46
:10B18000251620502424786FA2EC09F000017DECF4
:10B190005EF0A2EC09F001EE66F004010A51E92626
:10B1A000000EEA22EF500A6E450E0A5C000108E12B
:10B1B000A2EC09F0A2EC09F004015C9F00011BD095
:10B1C000A2EC09F001EE66F004010A51E926000E36
:10B1D000EA22EF500A6E570E0A5C000108E1A2EC69
:10B1E00009F0A2EC09F004015C8F000104D0A2EC8C
:10B1F00009F05BEF5EF0A2EC09F0A2EC09F0030E9F
:10B2000004010A27A2EC09F001EE66F00A51E926D2
:10B21000000EEA22EF500A6E2E0E0A5C000115E1C4
:10B22000A2EC09F0A2EC09F0FF0E04010A250A6E57
:10B230000B6AFF0E0B220A50660FE96E010E0B20FF
:10B24000EA6EEF50686F000188D0A2EC09F00401AB
:10B250000A2BA2EC09F001EE66F00A51E926000E75
:10B26000EA22EF500A6E2E0E0A5C000127E1A2ECE2
:10B2700009F0A2EC09F0FE0E04010A250A6E0B6A21
:10B28000FF0E0B220A50660FE96E010E0B20EA6ECC
:10B29000EF50676FA2EC09F0A2EC09F0FF0E0A254F
:10B2A0000A6E0B6AFF0E0B220A50660FE96E010E42
:10B2B0000B20EA6EEF50686F00014FD0A2EC09F04E
:10B2C00004010A2BA2EC09F001EE66F00A51E9260E
:10B2D000000EEA22EF500A6E2E0E0A5C000139E1E0
:10B2E000A2EC09F0A2EC09F0FD0E04010A250A6E99
:10B2F0000B6AFF0E0B220A50660FE96E010E0B203F
:10B30000EA6EEF50666FA2EC09F0A2EC09F0FE0EB7
:10B310000A250A6E0B6AFF0E0B220A50660FE96EB1
:10B32000010E0B20EA6EEF50676FA2EC09F0A2EC61
:10B3300009F0FF0E0A250A6E0B6AFF0E0B220A5057
:10B34000660FE96E010E0B20EA6EEF50686F000188
:10B3500004D0A2EC09F05BEF5EF0A2EC09F07DEC0A
:10B360005EF0A2EC09F001EE66F004010A51E92654
:10B37000000EEA22EF500A6E2C0E0A5C000117E163
:10B38000A2EC09F0A2EC09F0300E04016B6FA2EC04
:10B3900009F0A2EC09F0300E6A6FA2EC09F0A2EC01
:10B3A00009F0300E696FA2EC09F00001BFD0A2ECE9
:10B3B00009F004010A2BA2EC09F001EE66F00A5133
:10B3C000E926000EEA22EF500A6E2E0E0A5C0001FA
:10B3D00015E1A2EC09F0A2EC09F0FF0E04010A2528
:10B3E0000A6E0B6AFF0E0B220A50660FE96E010E01
:10B3F0000B20EA6EEF506B6F000198D0A2EC09F0C1
:10B4000004010A2BA2EC09F001EE66F00A51E926CC
:10B41000000EEA22EF500A6E2E0E0A5C000127E1B0
:10B42000A2EC09F0A2EC09F0FE0E04010A250A6E56
:10B430000B6AFF0E0B220A50660FE96E010E0B20FD
:10B44000EA6EEF506A6FA2EC09F0A2EC09F0FF0E71
:10B450000A250A6E0B6AFF0E0B220A50660FE96E70
:10B46000010E0B20EA6EEF506B6F00015FD0A2EC73
:10B4700009F004010A2BA2EC09F001EE66F00A5172
:10B48000E926000EEA22EF500A6E2E0E0A5C000139
:10B4900039E1A2EC09F0A2EC09F0FD0E04010A2545
:10B4A0000A6E0B6AFF0E0B220A50660FE96E010E40
:10B4B0000B20EA6EEF50696FA2EC09F0A2EC09F0E4
:10B4C000FE0E0A250A6E0B6AFF0E0B220A50660F4B
:10B4D000E96E010E0B20EA6EEF506A6FA2EC09F0E4
:10B4E000A2EC09F0FF0E0A250A6E0B6AFF0E0B2272
:10B4F0000A50660FE96E010E0B20EA6EEF506B6F7B
:10B50000000113D0A2EC09F0A2EC09F0300E040106
:10B510006B6FA2EC09F0A2EC09F0300E6A6FA2EC9E
:10B5200009F0A2EC09F0300E696F0001A2EC09F0FD
:10B53000A2EC09F0216A67C420F00F0E2016000E5D
:10B540002116256A0A0E246E276A66C426F00F0E9D
:10B550002616000E271625C017F02450166E260258
:10B56000F3CF24F0F4CF25F017502602F350252610
:10B5700016502702F3502526205024240401676F1B
:10B58000A2EC09F0140E675D000109E2A2EC09F0DB
:10B59000A2EC09F06C0E04016727000107D0A2ECB1
:10B5A00009F0A2EC09F0300E040167270001A2ECBB
:10B5B00009F0A2EC09F0216A69C420F00F0E2016F0
:10B5C000000E2116256A0A0E246E276A68C426F02A
:10B5D0000F0E2616000E271625C017F02450166EE3
:10B5E0002602F3CF24F0F4CF25F017502602F350B3
:10B5F000252616502702F350252620502424040126
:10B60000696FA2EC09F0A2EC09F0200E6927A2EC08
:10B6100009F0A2EC09F0216A6AC420F00F0E20168E
:10B62000000E2116256A0A0E246E276A6BC426F0C6
:10B630000F0E2616000E271625C017F02450166E82
:10B640002602F3CF24F0F4CF25F017502602F35052
:10B65000252616502702F3502526205024246B6FF0
:10B66000A2EC09F0A2EC09F01C0E6B27A2EC09F089
:10B67000A2EC09F0200E7027A2EC09F0000181B6BF
:10B6800007D0A2EC09F0A2EC09F0200E0401722709
:10B690000001A2EC09F081A407D0A2EC09F0A2EC11
:10B6A00009F0200E040171270001A2EC09F0040149
:10B6B0005C510001E8AC07D0A2EC09F0A2EC09F063
:10B6C000200E040173270001A2EC09F0650E0401AD
:10B6D000765D000107E3A2EC09F0A2EC09F0200E70
:10B6E000040174270001A2EC09F004015C3500019B
:10B6F00007E3A2EC09F0A2EC09F0200E0401752783
:10B700000001A2EC09F0650E0401765D000119E369
:10B71000A2EC09F06E0E0401765D000109E2A2ECD4
:10B7200009F0A2EC09F0080E04017627000107D009
:10B73000A2EC09F0A2EC09F0480E0401765F0001CA
:10B7400018D0A2EC09F00A0E0401765D000109E3AD
:10B75000A2EC09F0A2EC09F01C0E0401762700010E
:10B7600007D0A2EC09F0A2EC09F0760E04017627CE
:10B770000001A2EC09F00A0E0401775D000109E264
:10B78000A2EC09F0A2EC09F0580E040177270001A1
:10B7900007D0A2EC09F0A2EC09F01C0E04017727F7
:10B7A0000001A2EC09F081B89DD1A2EC09F0A2EC55
:10B7B00009F00401566B556BA2EC09F0A2EC09F0FC
:10B7C000050E096FA2EC09F0A2EC09F001EE66F09B
:10B7D000470EEE6E500EEE6E470EEE6EEE6E410EA2
:10B7E000EE6EEF6AA2EC09F0130E056E880E026E83
:10B7F000000127EC01F0D8A075D14708F9E127EC4A
:10B8000001F0D8A06FD14708F3E127EC01F0D8A0F0
:10B8100069D14108EDE127EC01F0D8A063D1040122
:10B820000B6FA2EC09F02A0E04010B5D00011DE074
:10B83000A2EC09F0010E056EF40E026E27EC01F089
:10B84000D8A050D104010B6FA2EC09F0A2EC09F0D2
:10B8500001EE66F00951E926000EEA220BC4EFFF63
:10B86000A2EC09F0092B0001DED7A2EC09F0A2EC52
:10B8700009F004010A6BA2EC09F0000126DAA2EC3F
:10B8800009F0A2EC09F001EE66F004010A51E92684
:10B89000000EEA22EF500A6E0F0E0A14566B556F17
:10B8A000A2EC09F00A2BA2EC09F001EE66F00A51B5
:10B8B000E926000EEA22EF500A6E2E0E0A5C000105
:10B8C000D8B410D1A2EC09F0A2EC09F056C421F0D2
:10B8D00055C420F021500A0DF3CF21F020500A0D5D
:10B8E000F3CF20F0F450212601EE66F004010A5156
:10B8F000E926000EEA22EF500A6E256A0AC024F0FB
:10B900000F0E2416000E251624502024556F2550A6
:10B910002120566FA2EC09F00A2BA2EC09F001EEEF
:10B9200066F00A51E926000EEA22EF500A6E2E0E4A
:10B930000A5C0001D8B4D6D0A2EC09F0A2EC09F060
:10B9400056C421F055C420F021500A0DF3CF21F048
:10B9500020500A0DF3CF20F0F450212601EE66F0BE
:10B9600004010A51E926000EEA22EF500A6E256A08
:10B970000AC024F00F0E2416000E25162450202491
:10B98000556F25502120566FA2EC09F00A2BA2EC2E
:10B9900009F001EE66F00A51E926000EEA22EF50A6
:10B9A0000A6E2E0E0A5C0001D8B49CD0A2EC09F0FD
:10B9B000A2EC09F056C421F055C420F021500A0D24
:10B9C000F3CF21F020500A0DF3CF20F0F4502126C0
:10B9D00001EE66F004010A51E926000EEA22EF505A
:10B9E0000A6E256A0AC024F00F0E2416000E2516D2
:10B9F00024502024556F25502120566FA2EC09F0C9
:10BA00000A2BA2EC09F001EE66F00A51E926000EBD
:10BA1000EA22EF500A6E2E0E0A5C0001D8B462D002
:10BA2000A2EC09F0A2EC09F056C421F055C420F0B4
:10BA300021500A0DF3CF21F020500A0DF3CF20F052
:10BA4000F450212601EE66F004010A51E926000EA9
:10BA5000EA22EF500A6E256A0AC024F00F0E24165F
:10BA6000000E251624502024556F25502120566F96
:10BA7000A2EC09F00A2BA2EC09F001EE66F00A51E3
:10BA8000E926000EEA22EF500A6E2E0E0A5C000133
:10BA900028E0A2EC09F0A2EC09F056C421F055C44C
:10BAA00020F021500A0DF3CF21F020500A0DF3CFE2
:10BAB00020F0F450212601EE66F004010A51E92637
:10BAC000000EEA22EF500A6E256A0AC024F00F0E1B
:10BAD0002416000E251624502024556F25502120B1
:10BAE000566F0001A2EC09F0A2EC09F01C0E040153
:10BAF0007827A2EC09F0A2EC09F070C456F0A2EC91
:10BB000009F0A2EC09F071C457F0A2EC09F0A2EC24
:10BB100009F072C458F0A2EC09F0A2EC09F073C469
:10BB200059F0A2EC09F0A2EC09F074C45AF0A2ECAE
:10BB300009F0A2EC09F075C45BF0A2EC09F0A2ECEC
:10BB400009F05C6AA2EC09F0A2EC09F076C466F197
:10BB5000A2EC09F0A2EC09F077C467F1A2EC09F0BD
:10BB6000A2EC09F078C468F1A2EC09F0A2EC09F0AB
:10BB700067C469F1A2EC09F0A2EC09F069C46AF1AA
:10BB8000A2EC09F0A2EC09F06BC46BF1A2EC09F095
:10BB9000A2EC09F07CC46CF1A2EC09F0A2EC09F073
:10BBA0007BC46DF1A2EC09F0000181A809D0A2ECE0
:10BBB00009F0A2EC09F00D0E01016E6F000169D0D1
:10BBC000A2EC09F0A2EC09F0100E04015527270E93
:10BBD0005623A2EC09F0A2EC09F056C40FF055C4AC
:10BBE0000EF0200E136E590E126E34EC02F0206E21
:10BBF0000FC021F0210E20240A6E0AC06EF1A2ECC3
:10BC000009F0A2EC09F056C40FF055C40EF0200E56
:10BC1000136E590E126E34EC02F017C056F416C0B3
:10BC200055F4A2EC09F0A2EC09F056C40FF055C48B
:10BC30000EF0136A5B0E126E34EC02F0206E0FC031
:10BC400021F0210E20240A6E0AC06FF1A2EC09F047
:10BC5000A2EC09F056C40FF055C40EF0136A5B0E47
:10BC6000126E34EC02F017C021F016C020F0210E45
:10BC700020240A6E0AC070F1A2EC09F0A2EC09F0CF
:10BC80007D0E0101716FA2EC09F0A2EC09F00D0E1E
:10BC9000726F0001A2EC09F0A2EC09F004013E6B06
:10BCA000AA0E3D6FA2EC09F0A2EC09F00599A2ECF6
:10BCB00009F000011200A2EC09F0A2EC09F0040165
:10BCC0005D81A2EC09F000011200A2EC09F015D888
:10BCD000A2EC09F012D8A2EC09F00FD8A2EC09F0FE
:10BCE0000CD8A2EC09F009D8A2EC09F006D8A2EC15
:10BCF00009F003D8A2EC09F000D8A2EC09F001EE9B
:10BD000066F004010A51E926000EEA22EF500A6E9D
:10BD10002C0E0A5CD8A4010E376E500E0A5D010E7F
:10BD2000D8B0000E3716000106E0A2EC09F00401BD
:10BD30000A2B0001E4D7A2EC09F004010A2BA2ECC3
:10BD400009F000011200A2EC09F081B207D0A2ECC8
:10BD500009F0A2EC09F086C465F4E9D1A2EC09F07F
:10BD6000A2EC09F004010A6BA2EC09F00001B3DFB8
:10BD7000A2EC09F0A2EC09F001EE66F004010A5110
:10BD8000E926000EEA22EF500A6E0F0E0A14266B07
:10BD9000256FA2EC09F00A2BA2EC09F001EE66F087
:10BDA0000A51E926000EEA22EF500A6E2E0E0A5CB6
:10BDB0000001D8B46ED0A2EC09F0A2EC09F0216A1F
:10BDC0000A0E206E21C017F02050166E04012503C4
:10BDD000F3CF20F0F4CF21F017502503F3502126A4
:10BDE00016502603F350212601EE66F00A51E9268B
:10BDF000000EEA22EF500A6E256A0AC024F00F0EE8
:10BE00002416000E251624502024256F25502120AD
:10BE1000266FA2EC09F00A2BA2EC09F001EE66F005
:10BE20000A51E926000EEA22EF500A6E2E0E0A5C35
:10BE300000012EE0A2EC09F0A2EC09F0216A0A0E42
:10BE4000206E21C017F02050166E04012503F3CF99
:10BE500020F0F4CF21F017502503F350212616507F
:10BE60002603F350212601EE66F00A51E926000E62
:10BE7000EA22EF500A6E256A0AC024F00F0E24163B
:10BE8000000E251624502024256F25502120266FD2
:10BE90000001A2EC09F031DFA2EC09F0A2EC09F0FC
:10BEA00001EE66F004010A51E926000EEA22EF5085
:10BEB0000A6E0F0E0A146D6B6C6FA2EC09F00A2B60
:10BEC000A2EC09F001EE66F00A51E926000EEA2222
:10BED000EF500A6E2E0E0A5C0001D8B462D0A2ECBC
:10BEE00009F0A2EC09F06DC421F06CC420F02150DF
:10BEF0000A0DF3CF21F020500A0DF3CF20F0F450BB
:10BF0000212601EE66F004010A51E926000EEA221C
:10BF1000EF500A6E256A0AC024F00F0E2416000E98
:10BF20002516245020246C6F255021206D6FA2EC23
:10BF300009F00A2BA2EC09F001EE66F00A51E9269D
:10BF4000000EEA22EF500A6E2E0E0A5C000128E075
:10BF5000A2EC09F0A2EC09F06DC421F06CC420F051
:10BF600021500A0DF3CF21F020500A0DF3CF20F01D
:10BF7000F450212601EE66F004010A51E926000E74
:10BF8000EA22EF500A6E256A0AC024F00F0E24162A
:10BF9000000E2516245020246C6F255021206D6F33
:10BFA0000001A2EC09F0A2EC09F0680E04016C2774
:10BFB000010E6D23A2EC09F0265304E1060E255D67
:10BFC00000013AE3A2EC09F004016E516C5D0E6EC3
:10BFD0006F516D590F6EA5EC02F00A6E0FC00BF099
:10BFE0000B5204E1290E0A5C000108E3A2EC09F0FF
:10BFF000A2EC09F00401266B320E256F0001A2ECC1
:10C0000009F004016E516C5D0E6E6F516D590F6E2B
:10C01000A5EC02F00A6E0FC00BF00B5204E13D0ECE
:10C020000A5C000108E3A2EC09F0A2EC09F00401AB
:10C03000266B460E256F0001A2EC09F0A2EC09F078
:10C040006DC46FF46CC46EF4A2EC09F004012653C5
:10C0500004E1420E255D000109E3A2EC09F0A2EC27
:10C0600009F00A0E0401656F000161D0A2EC09F02D
:10C070000401265304E12D0E255D000109E3A2EC25
:10C0800009F0A2EC09F0140E0401656F00014FD015
:10C09000A2EC09F00401265304E11C0E255D000109
:10C0A00009E3A2EC09F0A2EC09F01E0E0401656F91
:10C0B00000013DD0A2EC09F00401265304E10E0E6C
:10C0C000255D000109E3A2EC09F0A2EC09F03C0EA9
:10C0D0000401656F00012BD0A2EC09F00401265386
:10C0E00004E1070E255D000109E3A2EC09F0A2ECD2
:10C0F00009F0780E0401656F000119D0A2EC09F077
:10C100000401265304E1030E255D000109E3A2ECBE
:10C1100009F0A2EC09F0C80E0401656F000106D019
:10C12000A2EC09F0A2EC09F0040165690001A2EF9C
:10C1300009F0A2EC09F00301FD310001D8A0A2EF43
:10C1400009F0A2EC09F0A2EC09F001EE66F0130E82
:10C15000F76E060EF66EB5EC02F0020E016E046A82
:10C16000176A040E166E69EC00F02E0EEE6E020ECB
:10C17000016E010E046E310E67EC00F00D0EEE6ED6
:10C18000EE6AA2EC09F0D8EC22F0A2EC09F0A2ECE5
:10C1900009F000EEB9F0130EF76E0E0EF66EB5EC68
:10C1A00002F0EE6AA2EC09F0A2EC09F0600E4B6E10
:10C1B000A2EC09F0E0EC4EF0A2EC09F0A2EC09F0E0
:10C1C00000EEB9F010EE4DF0080EE75204E0E6CFB5
:10C1D000EEFFE82EFAD7EF6AA2EC09F0A2EC09F024
:10C1E000610E4B6EA2EC09F0E0EC4EF0A2EC09F00F
:10C1F000A2EC09F0030E476EA2EC09F0C8EC15F0B2
:10C20000A2EC09F0A2EC09F0F00E476EA2EC09F0E6
:10C21000C8EC15F0A2EC09F00401096B640E0401EE
:10C22000095D00011CE2A2EC09F0A2EC09F001EEAC
:10C2300066F004010951E926000EEA22EF50476E2C
:10C24000A2EC09F0475200010AE0A2EC09F0C8ECA8
:10C2500015F0A2EC09F00401092B0001DFE3A2ECC8
:10C2600009F049EC23F0A2EC09F0A2EC09F004017A
:10C270000597A2EC09F0A2EC09F0068FA2EC09F0F8
:10C28000010E136EF40EEFEC01F0A2EC09F00001C8
:10C290001200A2EC09F0A2EC09F00401069DA2EC48
:10C2A00009F0A2EC09F0069BA2EC09F0A2EC09F05F
:10C2B0000693A2EC09F0A2EC09F00591A2EC09F0BA
:10C2C000A2EC09F00583A2EC09F0A2EC09F00681CA
:10C2D000A2EC09F0A2EC09F00589A2EC09F0A2ECAD
:10C2E00009F079C47AF4A2EC09F000011200A2EC82
:10C2F00009F0C9D9A2EC09F0A2EC09F081CF10F441
:10C30000A2EC09F0A2EC09F001EE66F0540EEE6E1C
:10C31000230EEE6E020E016E030E046E88C417F03B
:10C3200087C416F069EC00F02C0EEE6E11EE03F0EF
:10C330000A0EE75204E0E6CFEEFFE82EFAD72C0E05
:10C34000EE6E11EE0EF00A0EE75204E0E6CFEEFFBD
:10C35000E82EFAD72C0EEE6E11EE19F00A0EE75207
:10C3600004E0E6CFEEFFE82EFAD72C0EEE6E11EECB
:10C3700024F00A0EE75204E0E6CFEEFFE82EFAD7EB
:10C380002C0EEE6E11EE2FF00A0EE75204E0E6CF0F
:10C39000EEFFE82EFAD72C0EEE6E020E016E080E9E
:10C3A000046E040110513DEC00F00D0EEE6EEE6ACD
:10C3B000A2EC09F00001E7EC11F0A2EC09F0A2EC0C
:10C3C00009F00401406B3F6BA2EC09F004013F51FE
:10C3D000660FE96E010E4021EA6EEF500A6E0D0EF7
:10C3E0000A5CD8A4010E376E405304E1FF0E3F5D96
:10C3F000000102E3000E01D0010E371600011AE021
:10C40000A2EC09F0A2EC09F004013F51660FE96EBD
:10C41000010E4021EA6EEF50476EA2EC09F00001D8
:10C42000C8EC15F0A2EC09F004013F2B000E4023EC
:10C430000001CCD7A2EC09F049EC23F0A2EC09F002
:10C44000A2EC09F0010E04018725206E000E882160
:10C45000216E21C00FF020C00EF0030E136EE80E07
:10C46000126E34EC02F017C088F416C087F4A2EC08
:10C4700009F000011200A2EC09F0040105510001CD
:10C48000E8B802D0A2EF09F0A2EC09F030DFA2EC8C
:10C4900009F0A2EC09F004010593A2EC09F07A2B53
:10C4A000A2EC09F079517A5D000ED8B0010E376E1A
:10C4B000000E0301FEBB010E37160001D8B4ABD04D
:10C4C000A2EC09F0A2EC09F00C0E04018A6FA2ECB8
:10C4D00009F004018A53000106E0A2EC09F09EBABB
:10C4E000A2EF09F0F6D7A2EC09F00301FE35000136
:10C4F000D8A07ED0A2EC09F0E7EC11F0A2EC09F094
:10C50000A2EC09F004015D91A2EC09F0A2EC09F0A3
:10C51000020E266FE20E256FA2EC09F000017ED814
:10C52000A2EC09F004018A53000106E0A2EC09F034
:10C530009EBAA2EF09F0F6D7A2EC09F0E7EC11F0F1
:10C54000A2EC09F0A2EC09F0030E0401266F410EE3
:10C55000256FA2EC09F0000161D8A2EC09F00401FA
:10C560008A53000106E0A2EC09F09EBAA2EF09F09E
:10C57000F6D7A2EC09F0E7EC11F0A2EC09F0A2EC7E
:10C5800009F0030E0401266FA00E256FA2EC09F03E
:10C59000000144D8A2EC09F004018A53000106E02E
:10C5A000A2EC09F09EBAA2EF09F0F6D7A2EC09F0CE
:10C5B000E7EC11F0A2EC09F0A2EC09F0010E040185
:10C5C000266F0F0E256FA2EC09F0A2EC09F07A6B32
:10C5D000A2EC09F0000122D8A2EC09F004018A5370
:10C5E000000106E0A2EC09F09EBAA2EF09F0F6D72E
:10C5F000A2EC09F00301FD35000107E3A2EC09F00C
:10C60000A4EC12F0A2EC09F033D8A2EC09F0A2ECF1
:10C6100009F004017A6B0001A2EF09F0A2EC09F025
:10C62000A2EC09F0456AA2EC09F0C80E455C1CE2D8
:10C63000A2EC09F0A2EC09F0455004012525A96EF1
:10C64000000E2621AA6EB0EC01F0476EA2EC09F0B4
:10C650000D0E475C000108E0A2EC09F0C8EC15F0F3
:10C66000A2EC09F0452AE1D7A2EC09F049EC23F04D
:10C67000A2EC09F0A2EC09F00C0E04018A6FA2EC06
:10C6800009F000011200A2EC09F0A2EC09F004018B
:10C690005D97A2EC09F0096B050E0401095D00012C
:10C6A000D8B08ED0A2EC09F0A2EC09F0AA6A4E0E26
:10C6B00004010925A96ED8B0AA2AB0EC01F00B6FCD
:10C6C000A2EC09F0540E0B5D0001D8A472D0A2ECCC
:10C6D00009F0A2EC09F004015D87A2EC09F009530E
:10C6E000000110E1A2EC09F0800E026E010E056E51
:10C6F000076E9CEC01F0CC0E85EC01F0440E85EC4D
:10C7000001F057D0010E0401095D000111E1A2EC16
:10C7100009F0800E026E020E056E010E076E9CEC93
:10C7200001F0CC0E85EC01F0440E85EC01F041D017
:10C73000020E0401095D000111E1A2EC09F0800E76
:10C74000026E040E056E010E076E9CEC01F0CC0E1D
:10C7500085EC01F0440E85EC01F02BD0030E0401B2
:10C76000095D000111E1A2EC09F0800E026E080ED5
:10C77000056E010E076E9CEC01F0CC0E85EC01F00D
:10C78000440E85EC01F015D0040E0401095D000192
:10C7900010E1A2EC09F0800E026E100E056E010E83
:10C7A000076E9CEC01F0CC0E85EC01F0440E85EC9C
:10C7B00001F0A2EC09F00401092B0001D8A06CD70C
:10C7C000A2EC09F004015D510001E8A62BD0A2EC17
:10C7D00009F00401266B256B030E0401265D0001A0
:10C7E00006E320E1210E0401255D00011BE2A2EC1D
:10C7F00009F0000E9EBA010E376E000E82B2010ED5
:10C8000037160001D8A4A2EF09F0A2EC09F0010E3E
:10C81000EEEC01F0A2EC09F00401252B000E26231A
:10C820000001DAE3A2EC09F0A2EC09F04E0EAEEC46
:10C8300001F004010B6FA2EC09F0410E0B5D000149
:10C84000D8A45ED0A2EC09F0A2EC09F004010F6BB1
:10C85000A2EC09F000510001E8AA3DD0A2EC09F0D9
:10C86000C9EC52F0A2EC09F0A2EC09F020C40FF0E0
:10C870001FC40EF0136A060E126E34EC02F00401AF
:10C880001F6F0FC020F4A2EC09F0030E205D000121
:10C890000FE305E1E80E04011F5D000109E3A2ECCE
:10C8A00009F0A2EC09F0030E0401206FE70E1F6FE0
:10C8B0000001A2EC09F0A2EC09F001EE03F0020E77
:10C8C000016E030E046E20C417F01FC416F069EC4D
:10C8D00000F0EE6A14D0A2EC09F0F3EC52F0A2ECF6
:10C8E00009F0A2EC09F001EE03F010EEB9F00F0E22
:10C8F000E75204E0E6CFEEFFE82EFAD7EF6A84D0E5
:10C90000A2EC09F0540E04010B5D010ED8A4000E38
:10C91000376E000E5CB1010E37160001D8B46BD033
:10C92000A2EC09F0800E026E010E056E076E9CEC03
:10C9300001F0CC0E85EC01F0BE0E85EC01F0A2EC0E
:10C9400009F0800E026E010E056E076A67EC01F0B9
:10C950000401396F67EC01F03A6FA2EC09F0A2EC28
:10C9600009F0D8925BB5D882D8B25E89D8A25E9918
:10C97000A2EC09F0000185EC68F0A2EC09F00401DA
:10C9800000510001E8AA22D0A2EC09F0A2EC09F0C3
:10C9900038C42FF037C42EF036C42DF035C42CF037
:10C9A000D8EC02F00401336F2DC034F4A2EC09F08E
:10C9B000A2EC09F001EE03F0020E016E030E046E0C
:10C9C000335167EC00F0EE6A000114D0A2EC09F0DC
:10C9D000A2EC09F001EE03F0020E016E38C423F060
:10C9E00037C422F036C421F035C420F0010EA2EC89
:10C9F00000F0EF6A09D0A2EC09F0A2EC09F001EE18
:10CA000003F0300EEE6EEF6AA2EC09F0A2EC09F032
:10CA1000AA6A4F0EA96EB0EC01F004010B6FA2ECF4
:10CA200009F0410E0B5D0001D8A45FD0A2EC09F023
:10CA3000A2EC09F0010E04010F6FA2EC09F0005105
:10CA40000001E8AA3DD0A2EC09F0C9EC52F0A2EC3A
:10CA500009F0A2EC09F020C40FF01FC40EF0136A15
:10CA6000060E126E34EC02F004011F6F0FC020F4AA
:10CA7000A2EC09F0030E205D00010FE305E1E80ED2
:10CA800004011F5D000109E3A2EC09F0A2EC09F02A
:10CA9000030E0401206FE70E1F6F0001A2EC09F0E6
:10CAA000A2EC09F001EE0EF0020E016E030E046E10
:10CAB00020C417F01FC416F069EC00F0EE6A14D021
:10CAC000A2EC09F0F3EC52F0A2EC09F0A2EC09F0B0
:10CAD00001EE0EF010EEB9F00F0EE75204E0E6CFD3
:10CAE000EEFFE82EFAD7EF6A85D0A2EC09F0540EDB
:10CAF00004010B5D010ED8A4000E376E000E5CB36E
:10CB0000010E37160001D8B46CD0A2EC09F0800EEB
:10CB1000026E020E056E010E076E9CEC01F0CC0E4B
:10CB200085EC01F0BE0E85EC01F0A2EC09F0800E60
:10CB3000026E020E056E076A67EC01F00401396FA0
:10CB400067EC01F03A6FA2EC09F0A2EC09F0D89280
:10CB50005BB7D882D8B25E89D8A25E99A2EC09F000
:10CB6000000185EC68F0A2EC09F00401005100011D
:10CB7000E8AA22D0A2EC09F0A2EC09F038C42FF008
:10CB800037C42EF036C42DF035C42CF0D8EC02F0AA
:10CB90000401336F2DC034F4A2EC09F0A2EC09F0CB
:10CBA00001EE0EF0020E016E030E046E335167ECBF
:10CBB00000F0EE6A000114D0A2EC09F0A2EC09F03A
:10CBC00001EE0EF0020E016E38C423F037C422F0DD
:10CBD00036C421F035C420F0010EA2EC00F0EF6A5B
:10CBE00009D0A2EC09F0A2EC09F001EE0EF0300E33
:10CBF000EE6EEF6AA2EC09F0A2EC09F0AA6A500E00
:10CC0000A96EB0EC01F004010B6FA2EC09F0410E2B
:10CC10000B5D0001D8A45FD0A2EC09F0A2EC09F0F2
:10CC2000020E04010F6FA2EC09F000510001E8AA06
:10CC30003DD0A2EC09F0C9EC52F0A2EC09F0A2EC54
:10CC400009F020C40FF01FC40EF0136A060E126E16
:10CC500034EC02F004011F6F0FC020F4A2EC09F0C5
:10CC6000030E205D00010FE305E1E80E04011F5DE6
:10CC7000000109E3A2EC09F0A2EC09F0030E0401A3
:10CC8000206FE70E1F6F0001A2EC09F0A2EC09F083
:10CC900001EE19F0020E016E030E046E20C417F0AF
:10CCA0001FC416F069EC00F0EE6A14D0A2EC09F093
:10CCB000F3EC52F0A2EC09F0A2EC09F001EE19F04D
:10CCC00010EEB9F00F0EE75204E0E6CFEEFFE82ECB
:10CCD000FAD7EF6A84D0A2EC09F0540E04010B5D80
:10CCE000010ED8A4000E376E000E5CB5010E37168B
:10CCF0000001D8B46BD0A2EC09F0800E026E040ED5
:10CD0000056E010E076E9CEC01F0CC0E85EC01F077
:10CD1000BE0E85EC01F0A2EC09F0800E026E040E4E
:10CD2000056E076A67EC01F00401396F67EC01F0EA
:10CD30003A6FA2EC09F0A2EC09F0D8925BB9D88264
:10CD4000D8B25E89D8A25E99A2EC09F00001DDD9C3
:10CD5000A2EC09F0040100510001E8AA22D0A2ECE3
:10CD600009F0A2EC09F038C42FF037C42EF036C415
:10CD70002DF035C42CF0D8EC02F00401336F2DC037
:10CD800034F4A2EC09F0A2EC09F001EE19F0020E65
:10CD9000016E030E046E335167EC00F0EE6A000181
:10CDA00014D0A2EC09F0A2EC09F001EE19F0020E89
:10CDB000016E38C423F037C422F036C421F035C4E4
:10CDC00020F0010EA2EC00F0EF6A09D0A2EC09F00D
:10CDD000A2EC09F001EE19F0300EEE6EEF6AA2EC53
:10CDE00009F0A2EC09F0AA6A510EA96EB0EC01F0AC
:10CDF00004010B6FA2EC09F0410E0B5D0001D8A4F9
:10CE00005FD0A2EC09F0A2EC09F0030E04010F6F51
:10CE1000A2EC09F000510001E8AA3DD0A2EC09F013
:10CE2000C9EC52F0A2EC09F0A2EC09F020C40FF01A
:10CE30001FC40EF0136A060E126E34EC02F00401E9
:10CE40001F6F0FC020F4A2EC09F0030E205D00015B
:10CE50000FE305E1E80E04011F5D000109E3A2EC08
:10CE600009F0A2EC09F0030E0401206FE70E1F6F1A
:10CE70000001A2EC09F0A2EC09F001EE24F0020E90
:10CE8000016E030E046E20C417F01FC416F069EC87
:10CE900000F0EE6A14D0A2EC09F0F3EC52F0A2EC30
:10CEA00009F0A2EC09F001EE24F010EEB9F00F0E3B
:10CEB000E75204E0E6CFEEFFE82EFAD7EF6A84D01F
:10CEC000A2EC09F0540E04010B5D010ED8A4000E73
:10CED000376E000E5CB7010E37160001D8B46BD068
:10CEE000A2EC09F0800E026E080E056E010E076EB0
:10CEF0009CEC01F0CC0E85EC01F0BE0E85EC01F04F
:10CF0000A2EC09F0800E026E080E056E076A67EC4F
:10CF100001F00401396F67EC01F03A6FA2EC09F0FF
:10CF2000A2EC09F0D8925BBBD882D8B25E89D8A2B5
:10CF30005E99A2EC09F00001E8D8A2EC09F0040126
:10CF400000510001E8AA22D0A2EC09F0A2EC09F0FD
:10CF500038C42FF037C42EF036C42DF035C42CF071
:10CF6000D8EC02F00401336F2DC034F4A2EC09F0C8
:10CF7000A2EC09F001EE24F0020E016E030E046E25
:10CF8000335167EC00F0EE6A000114D0A2EC09F016
:10CF9000A2EC09F001EE24F0020E016E38C423F079
:10CFA00037C422F036C421F035C420F0010EA2ECC3
:10CFB00000F0EF6A09D0A2EC09F0A2EC09F001EE52
:10CFC00024F0300EEE6EEF6AA2EC09F0A2EC09F04C
:10CFD000AA6A520EA96EB0EC01F004010B6F0001B9
:10CFE000A2EC09F0540E04010B5D010ED8A4000E52
:10CFF000376E000E5CB9010E37160001D8B46AD046
:10D00000A2EC09F0800E026E100E056E010E076E86
:10D010009CEC01F0CC0E85EC01F0BE0E85EC01F02D
:10D02000A2EC09F0800E026E100E056E076A67EC26
:10D0300001F00401396F67EC01F03A6FA2EC09F0DE
:10D04000A2EC09F05B35E836D8B05E89D8A05E99CD
:10D05000A2EC09F0000159D8A2EC09F0040100513A
:10D060000001E8AA22D0A2EC09F0A2EC09F038C431
:10D070002FF037C42EF036C42DF035C42CF0D8EC88
:10D0800002F00401336F2DC034F4A2EC09F0A2ECDD
:10D0900009F001EE2FF0020E016E030E046E335103
:10D0A00067EC00F0EE6A000114D0A2EC09F0A2ECEB
:10D0B00009F001EE2FF0020E016E38C423F037C4E0
:10D0C00022F036C421F035C420F0010EA2EC00F0AD
:10D0D000EF6A09D0A2EC09F0A2EC09F001EE2FF002
:10D0E000300EEE6EEF6AA2EC09F0A2EC09F000EE51
:10D0F000F8F011EE2FF00A0EE75204E0E6CFEEFF53
:10D10000E82EFAD7EF6AA2EF09F0A2EC09F00401C9
:10D110005E510001E8A812D0A2EC09F0A2EC09F0DF
:10D120003AC41BF039C41AF0136AA00E126E86ECD2
:10D1300002F017C033F40EC034F40FD0A2EC09F0A3
:10D14000A2EC09F004013A51050DF3CF34F4395142
:10D15000050DF3CF33F4F45034270001A2EC09F0AD
:10D16000A2EC09F0336A326A200E316E820E306E04
:10D1700034C42DF033C42CF077EC04F070EC03F0E1
:10D180002FC038F42EC037F42DC036F42CC035F43F
:10D19000A2EC09F0040100510001E8A262D0A2EC67
:10D1A00009F0A2EC09F02F6A2E6A100E2D6E820E85
:10D1B0002C6E38C433F037C432F036C431F035C485
:10D1C00030F0D6EC03F02FC023F02EC022F02DC09B
:10D1D00021F02CC020F0336A326A200E316E810EAD
:10D1E000306E23C02FF022C02EF021C02DF020C0C1
:10D1F0002CF070EC03F0336A326A7E0E306E800ED3
:10D200002DAE000E316EE2EC02F024EC04F02FBEE5
:10D2100003D081EC04F002D083EC04F02FC038F48A
:10D220002EC037F42DC036F42CC035F4A2EC09F032
:10D23000A2EC09F02F6A2E6A2D6A840E2C6E38C477
:10D2400033F037C432F036C431F035C430F0E2EC9C
:10D2500002F02FC038F42EC037F42DC036F42CC0A5
:10D2600035F4A2EF09F0A2EC09F0A2EC09F00401F8
:10D270005B93A2EC09F0A2EC09F05B9FA2EC09F031
:10D28000100E5F5D010ED8A4000E376E280E5F5D94
:10D29000010ED8A4000E3712220E5F5D010ED8A435
:10D2A000000E3712000111E0A2EC09F0A2EC09F027
:10D2B00004015B8FA2EC09F0A2EC09F0D8925FBBED
:10D2C000D882D8B25B83D8A25B930001A2EF09F0A9
:10D2D000A2EC09F00301FD350001D8A08CEF6CF041
:10D2E000A2EC09F0A2EC09F004010A6BA2EC09F02F
:10D2F000A2EC09F08B6BA2EC09F0A2EC09F05D93B3
:10D30000A2EC09F0A2EC09F05D97A2EC09F0FA0E8C
:10D3100004010A5D0001D8B00DD2A2EC09F0A2EC24
:10D3200009F0AA6AAA0E04010A25A96ED8B0AA2A91
:10D33000B0EC01F00B6FA2EC09F00D0E0B5D0001DB
:10D34000D8B4F8D1A2EC09F05C0E04010B5D000129
:10D35000D8A4EAD1A2EC09F0A2EC09F004015D83A3
:10D36000A2EC09F00A2BA2EC09F0A2EC09F0AA6ADF
:10D37000AA0E0A25A96ED8B0AA2AB0EC01F00B6F4C
:10D38000A2EC09F0A2EC09F00B9BA2EC09F0550EFF
:10D390000B5D000106E1A2EC09F0A2EC09F004012A
:10D3A0008B810001A2EC09F0560E04010B5D000117
:10D3B00006E1A2EC09F0A2EC09F004018B83000164
:10D3C000A2EC09F0570E04010B5D000106E1A2EC8E
:10D3D00009F0A2EC09F004018B850001A2EC09F030
:10D3E000580E04010B5D000106E1A2EC09F0A2EC6D
:10D3F00009F004018B870001A2EC09F0590E040129
:10D400000B5D010ED8A4000E376E540E0B5D010E9D
:10D41000D8A4000E3712000106E0A2EC09F0A2EC3D
:10D4200009F004018B890001A2EC09F0520E0401FD
:10D430000B5D00011BE1A2EC09F0A2EC09F001EE8A
:10D440005BF0020E016E046A42C417F041C416F08C
:10D4500069EC00F03A0EEE6E020E016E046E0401ED
:10D46000895167EC00F0EE6A00015ED1A2EC09F090
:10D4700004015C510001E8A857D1A2EC09F04C0E60
:10D4800004010B5D0001D8A471D0A2EC09F0A2EC5C
:10D4900009F0090E0401346FC40E336FA2EC09F0D9
:10D4A000616B0F0E0401615D00012FE2A2EC09F037
:10D4B00000EECFF0D89004016135E926000EEA2293
:10D4C000EECF0AF0EFCF0BF033510A5C34510B581A
:10D4D0000B503419D8B0800A000110E6A2EC09F014
:10D4E000A2EC09F000EECFF0D89004016135E926F6
:10D4F000000EEA22EECF33F4EFCF34F40001A2ECB9
:10D5000009F00401612B0001CCE3A2EC09F0A2ECCC
:10D5100009F001EE45F0020E016E046A34C41DF0FC
:10D5200033C41CF0176A0A0E166E4BEC02F0206E24
:10D530000FC021F021C01DF020C01CF0176A0A0E98
:10D54000166E4BEC02F0166E0FC017F064EC00F094
:10D550002E0EEE6E020E016E010E046E34C417F034
:10D5600033C416F064EC00F0EE6ADED0A2EC09F0F1
:10D57000480E04010B5D0001D8A46FD0A2EC09F0A5
:10D58000A2EC09F00401346B336BA2EC09F0616B7F
:10D590000F0E0401615D00012FE2A2EC09F000EE24
:10D5A000CFF0D89004016135E926000EEA22EECFD3
:10D5B0000AF0EFCF0BF00A50335D0B5034590B508B
:10D5C0003419D8B0800A000110E6A2EC09F0A2ECF0
:10D5D00009F000EECFF0D89004016135E926000E85
:10D5E000EA22EECF33F4EFCF34F40001A2EC09F0DD
:10D5F0000401612B0001CCE3A2EC09F0A2EC09F0DC
:10D6000001EE50F0020E016E046A34C41DF033C402
:10D610001CF0176A0A0E166E4BEC02F0206E0FC05B
:10D6200021F021C01DF020C01CF0176A0A0E166EF2
:10D630004BEC02F0166E0FC017F064EC00F02E0EEB
:10D64000EE6E020E016E010E046E34C417F033C488
:10D6500016F064EC00F0EE6A67D0A2EC09F0530E0D
:10D6600004010B5D0001D8A45ED0A2EC09F0A2EC8D
:10D6700009F00401346B336BA2EC09F0616B0F0EFF
:10D680000401615D00011AE2A2EC09F0A2EC09F0CC
:10D6900000EECFF0D89004016135E926000EEA22B1
:10D6A000EECF0AF0EFCF0BF00A5033270B503423A4
:10D6B000A2EC09F00401612B0001E1E3A2EC09F006
:10D6C000A2EC09F034C41DF033C41CF0176A0F0E2D
:10D6D000166E4BEC02F00401336F0FC034F4A2EC71
:10D6E00009F0A2EC09F001EE3AF0020E016E046AB4
:10D6F00034C41DF033C41CF0176A0A0E166E4BECCE
:10D7000002F0166E0FC017F064EC00F02E0EEE6EF5
:10D71000020E016E010E046E34C417F033C416F00D
:10D7200064EC00F0EE6A0001A2EC09F004010A2B9F
:10D730000001EDD5A2EC09F004018B530001D8B42F
:10D74000E7D0A2EC09F004018B31000125E3A2EC43
:10D7500009F0A2EC09F04E0EAEEC01F004010B6FE3
:10D76000A2EC09F0540E0B5D000115E1A2EC09F0EA
:10D77000A2EC09F004015D87A2EC09F0800E026EB4
:10D78000010E056E076E9CEC01F0CC0E85EC01F0ED
:10D79000440E85EC01F00001A2EC09F004018B516C
:10D7A0000001E8A228D0A2EC09F0A2EC09F0AA6AD4
:10D7B0004F0EA96EB0EC01F004010B6FA2EC09F062
:10D7C000540E0B5D000116E1A2EC09F0A2EC09F089
:10D7D00004015D87A2EC09F0800E026E020E056E58
:10D7E000010E076E9CEC01F0CC0E85EC01F0440EAE
:10D7F00085EC01F00001A2EC09F004018B5100015D
:10D80000E8A428D0A2EC09F0A2EC09F0AA6A500E14
:10D81000A96EB0EC01F004010B6FA2EC09F0540EFC
:10D820000B5D000116E1A2EC09F0A2EC09F0040185
:10D830005D87A2EC09F0800E026E040E056E010EEB
:10D84000076E9CEC01F0CC0E85EC01F0440E85ECEB
:10D8500001F00001A2EC09F004018B510001E8A6DF
:10D8600028D0A2EC09F0A2EC09F0AA6A510EA96E28
:10D87000B0EC01F004010B6FA2EC09F0540E0B5D4B
:10D88000000116E1A2EC09F0A2EC09F004015D87A9
:10D89000A2EC09F0800E026E080E056E010E076EF6
:10D8A0009CEC01F0CC0E85EC01F0440E85EC01F00F
:10D8B0000001A2EC09F004018B510001E8A828D076
:10D8C000A2EC09F0A2EC09F0AA6A520EA96EB0EC23
:10D8D00001F004010B6FA2EC09F0540E0B5D000186
:10D8E00016E1A2EC09F0A2EC09F004015D87A2ECBC
:10D8F00009F0800E026E100E056E010E076E9CEC94
:10D9000001F0CC0E85EC01F0440E85EC01F0000135
:10D91000A2EC09F0E0EC63F0A2EF09F0F2A462D10E
:10D920000B0ED76EDB0ED66E0401292B000E2A23B8
:10D930000E2B1153000104E004011107000106D071
:10D9400004011253000102E004010583000E0401EA
:10D9500000B9010E376E010E0EB1000E3716000130
:10D960003AE000EE8CF010EE95F0080EE75204E07D
:10D97000E6CFEEFFE82EFAD7EF6A00EE95F010EE54
:10D980009EF0080EE75204E0E6CFEEFFE82EFAD74D
:10D99000EF6A00EE9EF010EEA7F0080EE75204E0EA
:10D9A000E6CFEEFFE82EFAD7EF6A00EEA7F010EE12
:10D9B000B0F0080EE75204E0E6CFEEFFE82EFAD70B
:10D9C000EF6A00EEB0F0EE6AEE6AEE6AEE6AEE6AB8
:10D9D000EE6AEE6AEE6A2AC40FF029C40EF0136AEA
:10D9E0003C0E126E34EC02F017C00BF016C00AF0B9
:10D9F0000B500A1013E14FCF57F450CF58F40F01DA
:10DA0000506B4F6B0401892B3C0E895D000106E1D0
:10DA10000401896B0587412B000E42230401045148
:10DA20000001E8A40FD004012A5304E16551295DE7
:10DA3000000106E30401058D2A6B296B059105930E
:10DA4000000121D02AC40FF029C40EF0136A3C0E45
:10DA5000126E34EC02F00A6E0FC00BF00B5205E1AF
:10DA6000040108510A5C00010EE304012A6B296BD2
:10DA7000059D05510001E8B804D0040105810001AD
:10DA800002D00401058304015C510001E8A8A9D07B
:10DA90002AC40FF029C40EF0136A3C0E126E34EC47
:10DAA00002F017C00BF016C00AF00A503B0A0B1028
:10DAB00002E0000E01D0010E376E000E04015CB9C9
:10DAC000010E371600010EE0800E026E100E056E7C
:10DAD000010E076E9CEC01F0CC0E85EC01F0440EBB
:10DAE00085EC01F02AC40FF029C40EF0136A3C0E35
:10DAF000126E34EC02F017C00BF016C00AF00B5097
:10DB00000A1002E0000E01D0010E376E000E040173
:10DB10005CB9010E37160001D8B463D0800E026ED6
:10DB2000100E056E010E076E9CEC01F0CC0E85EC1C
:10DB300001F0BE0E85EC01F0800E026E100E056E37
:10DB4000076A67EC01F00401396F67EC01F03A6F86
:10DB50005B35E836D8B05E89D8A05E99000185ECC7
:10DB600068F038C430F437C42FF436C42EF435C40A
:10DB70002DF40401616B0E0E0401615D000118E2D9
:10DB80000401612900EECFF0D890E836EBCF0AF01F
:10DB9000E82AEBCF0BF000EECFF0D89061350AC049
:10DBA000EBFFE82A0BC0EBFF0401612B0001E3E36C
:10DBB0002F6A2E6A200E2D6E820E2C6E38C433F022
:10DBC00037C432F036C431F035C430F0D6EC03F04F
:10DBD00024EC04F00A6E2DC00BF00BC0ECF00AC070
:10DBE000EBF0F29411000001A2EC09F00400FCD764
:08DBF000A2EC09F00400FCD7CF
:020000040030CA
:03000100D80F38DD
:020005003D803C
:060008000FC00FE00F40E5
:0200000400F00A
:1000000000000000000000000000000000000000F0
:1000100000000000000000000000000000000000E0
:100020000000000010221C008448000084480000EA
:100030008448000084480000280F00032F3E058AF2
:10004000401E021E303030303030303030304141D0
:1000500041415400000000000000000000000000CA
:100060000000000000000000000000000000000090
:100070000000000000000000000000000000000080
:100080000000000000000000000000000000000070
:0C00900000000000000000000000000064
:00000001FF
